:100000000C94C9300C94FA300C94FA300C94FA30F9
:100010000C94FA300C94FA300C94FA300C94FA30B8
:100020000C94FA300C94FA300C94FA300C94FA30A8
:100030000C94FA300D94BE020C94FA300C94FA3001
:100040000C94FA300C949EDC0C94FA300C94FA3038
:100050000C94FA300C94FA300C94064B0C947EFEFF
:100060000C94FA300C946CD90C94FA300C94FA304D
:100070000C94FA300C94FA300C94FA300C94FA3058
:100080000C94FA300C94FA300C94FA300C94FA3048
:100090000C94FA300C94FA300C94FA300C94B0FBB7
:1000A0000C94FA300C94FA300C94FA300C94FA3028
:1000B0000C94FA300C94FA300C94FA300C94FA3018
:1000C0000C94FA300C94FA300C94FA300C94FA3008
:1000D0000C94FA300C94FA300C94FA300C94FA30F8
:1000E0000C94FA30534B614B7D4B8B4BA54BB34B70
:1000F000CD4BD14BD34BD74BDF4B02FD07FD0CFD56
:1001000016FD8FFD20FD28FD30FD3AFD44FD4EFD1E
:100110005DFD67FD8FFD71FD7BFD85FDADFDB0FDD6
:10012000A3FDA7FDE7FDB4FDB8FDBEFDC2FDC6FD04
:10013000CCFDD0FDD4FDE7FDDAFDDEFDE2FD084A91
:10014000D73B3BCE016E84BCBFFDC12F3D6C7431EB
:100150009ABD56833DDA3D00C77F11BED9E4BB4C42
:100160003E916BAAAABE000000803F05A84CCDB20C
:10017000D44EB93836A9020C50B9918688083CA6ED
:10018000AAAA2ABE000000803F000D94F3037C3C25
:100190003E5E2B3D3F2F5B5D3B2C2A225C0045726F
:1001A000723A204D415854454D5020424544005428
:1001B000656D7065726174757265206865617465DE
:1001C0006420626564207377697463686564206F76
:1001D00066662E204D415854454D50207472696713
:1001E00067657265642021004572723A204D494E60
:1001F00054454D50003A20457874727564657220FC
:100200007377697463686564206F66662E204D4954
:100210004E54454D5020747269676765726564205D
:1002200021004572723A204D415854454D50003AD4
:100230002045787472756465722073776974636899
:100240006564206F66662E204D415854454D502000
:10025000747269676765726564202100544845526D
:100260004D414C2052554E4157415900202D2049B7
:100270006E76616C6964206578747275646572204D
:100280006E756D626572202100504944204175747D
:100290006F74756E652066696E6973686564212088
:1002A00050757420746865206C617374204B702CD9
:1002B000204B6920616E64204B6420636F6E737401
:1002C000616E74732066726F6D2061626F76652057
:1002D000696E746F20436F6E6669677572617469C9
:1002E0006F6E2E6800504944204175746F74756EAE
:1002F00065206661696C6564212074696D656F7540
:10030000740020403A006F6B20543A006F6B20421B
:100310003A00504944204175746F74756E652066CB
:1003200061696C6564212054656D706572617475D6
:10033000726520746F6F206869676800204B643AAB
:100340002000204B693A2000204B703A20002043C7
:100350006C61737369632050494420002054753ADE
:100360002000204B753A2000206D61783A20002053
:100370006D696E3A200020643A2000206269617342
:100380003A20001000C90210012C01400122017026
:10039000011801B0010E01F00104015002FA00B091
:1003A00002F0003003E600D003DC009004D20070BD
:1003B00005C800A006BE000008B400B009AA00D01D
:1003C0000BA000600E960060118C000015820020CA
:1003D000197800C01D6E00A0226400B0275A00905A
:1003E0002C500000314600E0343C001038320090C0
:1003F0003A2800603C1E00A03D1400803E0A002008
:100400003F000070012C0190012701B0012201C0C2
:10041000011D01F00118011002130130020E0160EC
:1004200002090190020401C002FF000003FA00402B
:1004300003F5008003F000D003EB002004E6007019
:1004400004E100E004DC004005D700C005D2004014
:1004500006CD00D006C8008007C3003008BE00F0FB
:1004600008B900C009B400B00AAF00B00BAA00D0B0
:100470000CA500000EA000500F9B00C0109600506D
:1004800012910000148C00C0158700B0178200B0D4
:10049000197D00D01B7800001E730040206E009074
:1004A000226900F024640040275F0090295A00E090
:1004B0002B5500102E500020304B0010324600E02B
:1004C00033410090353C001037370070383200A0BF
:1004D000392D00B03A2800A03B2300603C1E0010DC
:1004E0003D1900903D1400103E0F00703E0A00C000
:1004F0003E0500003F00004472756B207A20555382
:1005000042202000496D70726573696F6E206465CA
:100510002055534220005374616D70612064612046
:10052000555342005469736B207A20555342202062
:1005300000555342207072696E74696E6720200006
:1005400053746174797374796B61202000457374FE
:100550006164697374696361202000537461746914
:100560007374696368650053746174697374696B4B
:10057000612020005374617469737469637320206F
:100580000053656C6674657374206E69657564618B
:100590006E79004175746F746573742066616C6C5C
:1005A00061646F004175746F746573742066616C6B
:1005B0006C69746F0053656C667465737420736541
:1005C0006C68616C20200053656C667465737420E0
:1005D0006661696C656420200053656C66746573A0
:1005E00074202020202020202020004175746F746A
:1005F000657374004175746F746573740053656C32
:100600006674657374202020202020202020005351
:10061000656C6674657374202020202020202020C3
:100620000057737A7973746B6F204F4B2020202012
:10063000202000546F646F2062696520004E65734E
:1006400073756E206572726F726500567365204F08
:100650004B202020202020202020202000416C6CD6
:1006600020636F7272656374202020202020004B6D
:100670006F6E74726F6C6120626564202020202090
:1006800000436F6E74726F6C2064652063616D61EE
:10069000005665726966696361207069617374727E
:1006A00061004B6F6E74726F6C6120626564202014
:1006B00020202000436865636B696E672062656473
:1006C0002020202020004B6F6E74726F6C61205AC6
:1006D0002061786973202000436F6E74726F6C2004
:1006E00064656C20656A65205A00566572696669A2
:1006F00063612061737365205A004B6F6E74726F73
:100700006C61205A2061786973202000436865631A
:100710006B696E67205A20617869732020004B6FE7
:100720006E74726F6C6120592061786973202000AB
:10073000436F6E74726F6C2064656C20656A65200F
:10074000590056657269666963612061737365203B
:1007500059004B6F6E74726F6C612059206178691B
:1007600073202000436865636B696E6720592061C0
:100770007869732020004B6F6E74726F6C61205823
:100780002061786973202000436F6E74726F6C2053
:1007900064656C20656A65205800566572696669F3
:1007A000636120617373652058004B6F6E74726FC4
:1007B0006C6120582061786973202000436865636C
:1007C0006B696E67205820617869732020004B6F39
:1007D0006E74726F6C6120686F74656E64202000A7
:1007E000436F6E74726F6C20686F74656E64200066
:1007F0005665726966696361206C696D2074656D08
:1008000070004B6F6E74726F6C6120686F74656EF0
:1008100064202000436865636B696E6720686F74AD
:10082000656E642020004B6F6E74726F6C61206582
:100830006E6473746F707300436F6E742E20746FE8
:100840007065732066696E616C00566572696669D1
:100850006361206C696D697469004B6F6E74726FAF
:100860006C6120656E6473746F70730043686563B8
:100870006B696E6720656E6473746F707300536587
:100880006C66207465737420737461727420200028
:100890004175746F746573742073616C6964610071
:1008A000496E697A6961206175746F74657374004B
:1008B00053656C6620746573742073746172742060
:1008C000200053656C6620746573742073746172C4
:1008D00074202000437A6173206472756B75203A2E
:1008E0002020005469656D706F20646520696D700B
:1008F0002E3A0054656D706F207374616D70613AAB
:1009000000436173207469736B75203A2020005096
:1009100072696E742074696D653A20200046696CB6
:10092000616D656E74203A20200046696C616D65CA
:100930006E746F203A20200046696C616D656E749C
:100940006F3A0046696C616D656E74203A20200034
:1009500046696C616D656E7420757365643A20201C
:1009600000437A61732063616C6B6F7769747920DF
:100970003A005469656D706F20746F74616C203A31
:100980000054656D706F207374616D706120746FB9
:10099000743A0043656C6B6F767920636173203A1B
:1009A00000546F74616C207072696E742074696D8C
:1009B00065203A0046696C616D656E74206C6163F8
:1009C0007A6E6965203A0046696C616D656E746F78
:1009D00020746F74616C3A0046696C616D656E7469
:1009E0006F20746F743A0046696C616D656E742097
:1009F00063656C6B656D203A00546F74616C2066A2
:100A0000696C616D656E74203A0053656C66207484
:100A1000657374204F4B0053656C66207465737466
:100A2000204F4B004175746F74657374204F4B00F9
:100A300053656C662074657374204F4B0053656C6E
:100A4000662074657374204F4B00456E6473746F39
:100A500070206E6F742068697400546F7065206632
:100A6000696E2E206E6F20746F632E004C696D2EA0
:100A70002066756F7269706F727461746100456E83
:100A80006473746F70206E6F742068697400456EB3
:100A90006473746F70206E6F742068697400456EA3
:100AA0006473746F7000546F70652066696E616C5A
:100AB000004C696D69746520636F72736100456EE7
:100AC0006473746F7000456E6473746F7000536963
:100AD0006C6E696B004D6F746F72004D6F746F7246
:100AE00065004D6F746F72004D6F746F7200456ECC
:100AF0006473746F707300546F7065732066696EF1
:100B0000616C004C696D69746920636F7273610078
:100B1000456E6473746F707300456E6473746F70A8
:100B20007300426C616420706F6C61637A656E69FA
:100B300061004572726F7220646520636F6E657824
:100B400069C383C692C382C2B36E004572726F726C
:100B500065206361626C616767696F0043687962F1
:100B600061207A61706F6A656E6900576972696E9B
:100B700067206572726F7200426564202F2048659D
:100B8000617465720043616D612F43616C656E74C1
:100B900061646F7200506961737472612F5269737E
:100BA00063616C6461746F726500426564202F201C
:100BB00048656174657200426564202F2048656154
:100BC000746572004865617465722F546865726D52
:100BD0006973746F720043616C656E742E2F546577
:100BE000726D6973746F720052697363616C642E05
:100BF0002F5465726D6973746F7265004865617416
:100C000065722F546865726D6973746F7200486500
:100C1000617465722F546865726D6973746F7200C8
:100C20004E696520706F646C61637A6F6E6F20200F
:100C300020004E6F2068617920636F6E6578696F60
:100C40006E2020004E6F6E20636F6E6E6573736F43
:100C5000004E657A61706F6A656E6F2020202000FB
:100C60004E6F7420636F6E6E656374656400536BC2
:100C70006F6E74726F6C756A203A00436F6E747297
:100C80006F6C61203A0056657269666963613A006B
:100C90005A6B6F6E74726F6C756A7465203A00508F
:100CA0006C6561736520636865636B203A0053650A
:100CB0006C6674657374206572726F72202100C354
:100CC00083E2809AC382C2A14175746F74657374A4
:100CD000206572726F7221004175746F7465737450
:100CE000206E6567617469766F0053656C66746524
:100CF0007374206572726F7220210053656C667484
:100D0000657374206572726F72202100686F77744A
:100D10006F2E707275736133642E637A00686F771B
:100D2000746F2E707275736133642E636F6D00681B
:100D30006F77746F2E707275736133642E636F6D8D
:100D400000686F77746F2E707275736133642E63F1
:100D50007A00686F77746F2E707275736133642ECA
:100D6000636F6D00666F72756D2E7072757361338F
:100D7000642E637A00666F72756D2E707275736182
:100D800033642E636F6D00666F72756D2E707275B1
:100D9000736133642E636F6D00666F72756D2E70B4
:100DA0007275736133642E637A00666F72756D2E8F
:100DB000707275736133642E636F6D00707275733A
:100DC0006133642E637A00707275736133642E63CD
:100DD0006F6D00707275736133642E636F6D007098
:100DE0007275736133642E637A0070727573613348
:100DF000642E636F6D005779626F72206A657A792D
:100E00006B6120202020202020200043616D62693A
:100E100061206C61206C656E677561200053656CA4
:100E2000657A2E206C61206C696E67756100567959
:100E3000626572206A617A796B612020202020200F
:100E400020200053656C656374206C616E6775616A
:100E50006765202020202000506F6C736B6900456F
:100E60007370616E6F6C004974616C69616E6F00C4
:100E700043657374696E6100456E676C69736800E1
:100E80004572726F7220696E206D656E7520737485
:100E900072756374757265004572726F7220696E47
:100EA000206D656E7520737472756374757265005C
:100EB0004572726F7220696E206D656E7520737455
:100EC00072756374757265004572726F7220696E17
:100ED000206D656E7520737472756374757265002C
:100EE0004572726F7220696E206D656E7520737425
:100EF0007275637475726500446F737461766F7692
:100F0000616E69205A0041646A757374696E672066
:100F10005A0041646A757374696E67205A00446FA1
:100F2000737461766F76616E69205A0041646A75E8
:100F30007374696E67205A004261627973746570D8
:100F400070696E67205900426162797374657070D0
:100F5000696E6720590042616279737465707069C7
:100F60006E67205900426162797374657070696EB2
:100F700067205900426162797374657070696E67A9
:100F8000205900426162797374657070696E6720E0
:100F90005800426162797374657070696E67205899
:100FA00000426162797374657070696E67205800E1
:100FB000426162797374657070696E67205800428F
:100FC0006162797374657070696E6720580020746F
:100FD0006F6F206C6F6E6720657874727573696FC0
:100FE0006E2070726576656E7465640020746F6F34
:100FF000206C6F6E6720657874727573696F6E20F0
:1010000070726576656E7465640020746F6F206C15
:101010006F6E6720657874727573696F6E20707279
:101020006576656E7465640020746F6F206C6F6EFA
:101030006720657874727573696F6E20707265765B
:10104000656E7465640020746F6F206C6F6E67202E
:10105000657874727573696F6E2070726576656EEF
:101060007465640020636F6C6420657874727573B6
:10107000696F6E2070726576656E746564002063BA
:101080006F6C6420657874727573696F6E2070720E
:101090006576656E7465640020636F6C64206578A6
:1010A00074727573696F6E2070726576656E7465A3
:1010B000640020636F6C6420657874727573696F67
:1010C0006E2070726576656E7465640020636F6C67
:1010D0006420657874727573696F6E2070726576BE
:1010E000656E74656400656E6473746F70732068F8
:1010F00069743A2000656E6473746F707320686958
:10110000743A2000656E6473746F7073206869743C
:101110003A2000656E6473746F7073206869743A66
:101120002000656E6473746F7073206869743A2070
:1011300000537465707261746520746F6F20686904
:1011400067683A2000537465707261746520746F2B
:101150006F20686967683A20005374657072617423
:101160006520746F6F20686967683A200053746562
:10117000707261746520746F6F20686967683A20C7
:1011800000537465707261746520746F6F206869B4
:1011900067683A200043616E6E6F7420656E7465F7
:1011A00072207375626469723A200043616E6E6FDB
:1011B0007420656E746572207375626469723A207A
:1011C0000043616E6E6F7420656E74657220737576
:1011D000626469723A200043616E6E6F7420656EBE
:1011E000746572207375626469723A200043616E9F
:1011F0006E6F7420656E74657220737562646972B7
:101200003A20006572726F722077726974696E6736
:1012100020746F2066696C65006572726F7220774A
:10122000726974696E6720746F2066696C65006509
:1012300072726F722077726974696E6720746F20A2
:1012400066696C65006572726F7220777269746985
:101250006E6720746F2066696C65006572726F72CC
:101260002077726974696E6720746F2066696C6597
:10127000004E6F74205344207072696E74696E67FB
:10128000004E6F74205344207072696E74696E67EB
:10129000004E6F74205344207072696E74696E67DB
:1012A000004E6F74205344207072696E74696E67CB
:1012B000004E6F74205344207072696E74696E67BB
:1012C000005344207072696E74696E67206279748D
:1012D0006520005344207072696E74696E672062E5
:1012E00079746520005344207072696E74696E676A
:1012F000206279746520005344207072696E7469AD
:101300006E67206279746520005344207072696EA4
:1013100074696E6720627974652000577269746918
:101320006E6720746F2066696C653A200057726999
:1013300074696E6720746F2066696C653A20005787
:10134000726974696E6720746F2066696C653A20F3
:101350000057726974696E6720746F2066696C65E6
:101360003A200057726974696E6720746F2066694D
:101370006C653A200046696C652073656C65637422
:1013800065640046696C652073656C6563746564AB
:101390000046696C652073656C656374656400461E
:1013A000696C652073656C65637465640046696C7F
:1013B000652073656C6563746564002053697A65A4
:1013C0003A20002053697A653A20002053697A65F3
:1013D0003A20002053697A653A20002053697A65E3
:1013E0003A200046696C65206F70656E65643A202E
:1013F0000046696C65206F70656E65643A20004632
:10140000696C65206F70656E65643A200046696C92
:1014100065206F70656E65643A200046696C6520D2
:101420006F70656E65643A20006F70656E2066614E
:10143000696C65642C2046696C653A20006F7065A4
:101440006E206661696C65642C2046696C653A2083
:10145000006F70656E206661696C65642C2046695A
:101460006C653A20006F70656E206661696C65641A
:101470002C2046696C653A20006F70656E206661AD
:10148000696C65642C2046696C653A2000776F7240
:101490006B446972206F70656E206661696C65646B
:1014A00000776F726B446972206F70656E206661A1
:1014B000696C656400776F726B446972206F706548
:1014C0006E206661696C656400776F726B44697247
:1014D000206F70656E206661696C656400776F725D
:1014E0006B446972206F70656E206661696C65641B
:1014F0000053442063617264206F6B005344206387
:10150000617264206F6B0053442063617264206FCA
:101510006B0053442063617264206F6B005344205E
:1015200063617264206F6B006F70656E526F6F74D1
:10153000206661696C6564006F70656E526F6F74D0
:10154000206661696C6564006F70656E526F6F74C0
:10155000206661696C6564006F70656E526F6F74B0
:10156000206661696C6564006F70656E526F6F74A0
:10157000206661696C656400766F6C756D652E69B7
:101580006E6974206661696C656400766F6C756D58
:10159000652E696E6974206661696C656400766F9A
:1015A0006C756D652E696E6974206661696C656421
:1015B00000766F6C756D652E696E69742066616961
:1015C0006C656400766F6C756D652E696E6974204C
:1015D0006661696C656400534420696E69742066B5
:1015E00061696C00534420696E6974206661696C9E
:1015F00000534420696E6974206661696C0053442D
:1016000020696E6974206661696C00534420696EBC
:101610006974206661696C0043616E6E6F74206F3F
:1016200070656E207375626469720043616E6E6FDF
:1016300074206F70656E2073756264697200436117
:101640006E6E6F74206F70656E2073756264697260
:101650000043616E6E6F74206F70656E20737562EB
:101660006469720043616E6E6F74206F70656E20E6
:1016700073756264697200486F74656E64206F668A
:1016800066736574733A00486F74656E64206F66A4
:1016900066736574733A00486F74656E64206F6694
:1016A00066736574733A00486F74656E64206F6684
:1016B00066736574733A00486F74656E64206F6674
:1016C00066736574733A006F70656E006F70656E57
:1016D000006F70656E006F70656E006F70656E00F4
:1016E000545249474745524544005452494747459B
:1016F00052454400545249474745524544005452CC
:101700004947474552454400545249474745524589
:1017100044005265706F7274696E6720656E647301
:10172000746F7020737461747573005265706F729A
:1017300074696E6720656E6473746F702073746172
:10174000747573005265706F7274696E6720656E90
:101750006473746F70207374617475730052657074
:101760006F7274696E6720656E6473746F70207336
:101770007461747573005265706F7274696E67205E
:10178000656E6473746F7020737461747573007A1E
:101790005F6D61783A20007A5F6D61783A20007A57
:1017A0005F6D61783A20007A5F6D61783A20007A47
:1017B0005F6D61783A20007A5F6D696E3A20007A39
:1017C0005F6D696E3A20007A5F6D696E3A20007A2B
:1017D0005F6D696E3A20007A5F6D696E3A2000791C
:1017E0005F6D61783A2000795F6D61783A20007909
:1017F0005F6D61783A2000795F6D61783A200079F9
:101800005F6D61783A2000795F6D696E3A200079EA
:101810005F6D696E3A2000795F6D696E3A200079DC
:101820005F6D696E3A2000795F6D696E3A200078CD
:101830005F6D61783A2000785F6D61783A200078BA
:101840005F6D61783A2000785F6D61783A200078AA
:101850005F6D61783A2000785F6D696E3A2000789C
:101860005F6D696E3A2000785F6D696E3A2000788E
:101870005F6D696E3A2000785F6D696E3A200049AD
:101880006E76616C69642065787472756465720047
:10189000496E76616C6964206578747275646572EE
:1018A00000496E76616C6964206578747275646550
:1018B0007200496E76616C69642065787472756433
:1018C000657200496E76616C696420657874727522
:1018D0006465720041637469766520457874727539
:1018E0006465723A200041637469766520457874B6
:1018F00072756465723A20004163746976652045AB
:10190000787472756465723A200041637469766513
:101910002045787472756465723A20004163746979
:1019200076652045787472756465723A2000556E4C
:101930006B6E6F776E20636F6D6D616E643A2022FF
:1019400000556E6B6E6F776E20636F6D6D616E64A8
:101950003A202200556E6B6E6F776E20636F6D6D4F
:10196000616E643A202200556E6B6E6F776E206355
:101970006F6D6D616E643A202200556E6B6E6F77ED
:101980006E20636F6D6D616E643A20220052657344
:10199000656E643A2000526573656E643A200052A9
:1019A0006573656E643A2000526573656E643A2013
:1019B00000526573656E643A20005072696E7465FA
:1019C000722073746F707065642064756520746F25
:1019D000206572726F72732E204669782074686574
:1019E000206572726F7220616E6420757365204D80
:1019F00039393920746F20726573746172742E20C6
:101A00002854656D70657261747572652069732004
:101A100072657365742E2053657420697420616645
:101A20007465722072657374617274696E672900DF
:101A30005072696E7465722073746F707065642083
:101A400064756520746F206572726F72732E204604
:101A5000697820746865206572726F7220616E64A7
:101A600020757365204D39393920746F2072657384
:101A7000746172742E202854656D7065726174757E
:101A800072652069732072657365742E20536574C6
:101A90002069742061667465722072657374617266
:101AA00074696E6729005072696E74657220737470
:101AB0006F707065642064756520746F2065727244
:101AC0006F72732E20466978207468652065727283
:101AD0006F7220616E6420757365204D393939202D
:101AE000746F20726573746172742E202854656D52
:101AF00070657261747572652069732072657365B3
:101B0000742E205365742069742061667465722098
:101B100072657374617274696E6729005072696EC0
:101B20007465722073746F707065642064756520CD
:101B3000746F206572726F72732E204669782074FC
:101B40006865206572726F7220616E6420757365BE
:101B5000204D39393920746F207265737461727445
:101B60002E202854656D70657261747572652069E8
:101B7000732072657365742E205365742069742018
:101B800061667465722072657374617274696E67E0
:101B900029005072696E7465722073746F7070657D
:101BA000642064756520746F206572726F72732E85
:101BB0002046697820746865206572726F722061B2
:101BC0006E6420757365204D39393920746F207229
:101BD0006573746172742E202854656D706572612E
:101BE000747572652069732072657365742E205355
:101BF00065742069742061667465722072657374FF
:101C0000617274696E6729005072696E7465722022
:101C100068616C7465642E206B696C6C2829206384
:101C2000616C6C656421005072696E746572206825
:101C3000616C7465642E206B696C6C28292063616B
:101C40006C6C656421005072696E74657220686105
:101C50006C7465642E206B696C6C28292063616C40
:101C60006C656421005072696E7465722068616CE5
:101C70007465642E206B696C6C28292063616C6C20
:101C8000656421005072696E7465722068616C74BD
:101C900065642E206B696C6C28292063616C6C650F
:101CA00064210020436F756E7420583A2000204351
:101CB0006F756E7420583A200020436F756E742043
:101CC000583A200020436F756E7420583A20002047
:101CD000436F756E7420583A20004649524D574163
:101CE00052455F4E414D453A4D61726C696E2056CA
:101CF000312E302E323B20537072696E7465722F14
:101D00006772626C206D617368757020666F7220F7
:101D100067656E36204649524D574152455F5552D0
:101D20004C3A68747470733A2F2F676974687562DF
:101D30002E636F6D2F707275736133642F507275DF
:101D400073612D69332D506C75732F2050524F5491
:101D50004F434F4C5F56455253494F4E3A312E3008
:101D6000204D414348494E455F545950453A5072C1
:101D7000757361206933204D4B32204558545255BC
:101D80004445525F434F554E543A312055554944CE
:101D90003A30303030303030302D303030302D303F
:101DA0003030302D303030302D3030303030303039
:101DB00030303030300A004649524D574152455F6D
:101DC0004E414D453A4D61726C696E2056312E3050
:101DD0002E323B20537072696E7465722F67726287
:101DE0006C206D617368757020666F722067656E18
:101DF00036204649524D574152455F55524C3A683C
:101E0000747470733A2F2F6769746875622E636FEC
:101E10006D2F707275736133642F50727573612DFD
:101E200069332D506C75732F2050524F544F434FD0
:101E30004C5F56455253494F4E3A312E30204D415A
:101E40004348494E455F545950453A507275736145
:101E5000206933204D4B3220455854525544455249
:101E60005F434F554E543A3120555549443A30302E
:101E70003030303030302D303030302D3030303068
:101E80002D303030302D3030303030303030303058
:101E900030300A004649524D574152455F4E414D40
:101EA000453A4D61726C696E2056312E302E323BB0
:101EB00020537072696E7465722F6772626C206D48
:101EC000617368757020666F722067656E36204694
:101ED00049524D574152455F55524C3A687474709F
:101EE000733A2F2F6769746875622E636F6D2F7058
:101EF0007275736133642F50727573612D69332D60
:101F0000506C75732F2050524F544F434F4C5F56B7
:101F1000455253494F4E3A312E30204D41434849A6
:101F20004E455F545950453A50727573612069337C
:101F3000204D4B322045585452554445525F434F33
:101F4000554E543A3120555549443A3030303030AE
:101F50003030302D303030302D303030302D30308A
:101F600030302D3030303030303030303030300A9A
:101F7000004649524D574152455F4E414D453A4DFD
:101F800061726C696E2056312E302E323B205370B8
:101F900072696E7465722F6772626C206D6173680E
:101FA000757020666F722067656E36204649524D07
:101FB000574152455F55524C3A68747470733A2FCA
:101FC0002F6769746875622E636F6D2F70727573F9
:101FD0006133642F50727573612D69332D506C75A8
:101FE000732F2050524F544F434F4C5F564552531E
:101FF000494F4E3A312E30204D414348494E455FBE
:10200000545950453A5072757361206933204D4BD5
:10201000322045585452554445525F434F554E5413
:102020003A3120555549443A303030303030303034
:102030002D303030302D303030302D303030302DAC
:102040003030303030303030303030300A004649B7
:10205000524D574152455F4E414D453A4D61726C6C
:10206000696E2056312E302E323B20537072696ECD
:102070007465722F6772626C206D61736875702071
:10208000666F722067656E36204649524D57415241
:10209000455F55524C3A68747470733A2F2F6769D4
:1020A000746875622E636F6D2F707275736133641F
:1020B0002F50727573612D69332D506C75732F20FD
:1020C00050524F544F434F4C5F56455253494F4E19
:1020D0003A312E30204D414348494E455F545950C6
:1020E000453A5072757361206933204D4B3220455B
:1020F000585452554445525F434F554E543A31203F
:10210000555549443A30303030303030302D303051
:1021100030302D303030302D303030302D303030C8
:102120003030303030303030300A0053746F6C69EA
:102130006B204F4B2E0042617365206C6973746F86
:102140002E0050696174746F20666174746F2E0084
:10215000426564204F4B2E0042656420646F6E65BB
:102160000047727A616E69652073746F6C696B6188
:102170002E2E00426173652043616C656E74616E42
:10218000646F0050696174746F2072697363616C6D
:1021900064616D2E005A6168726976616E692062B1
:1021A0006564004265642048656174696E67004734
:1021B000727A616E6965204F4B2E0043616C656ECB
:1021C00074616E646F206C6973746F2E0052697352
:1021D00063616C64616D656E746F20666174746FA9
:1021E0002E005A6168726976616E69204F4B2E002D
:1021F00048656174696E6720646F6E652E00477272
:102200007A616E69652E2E2E0043616C656E746175
:102210006E646F2E2E2E0052697363616C64616D63
:10222000656E746F2E2E2E005A6168726976616E2B
:10223000690048656174696E67004D313039204925
:102240006E76616C6964206578747275646572205D
:10225000004D31303920496E76616C6964206578B3
:1022600074727564657220004D31303920496E7684
:10227000616C696420657874727564657220004DC4
:1022800031303920496E76616C69642065787472EA
:102290007564657220004D31303920496E76616C6D
:1022A000696420657874727564657220004E6F20D1
:1022B000746865726D6973746F7273202D206E6F10
:1022C0002074656D7065726174757265004E6F2063
:1022D000746865726D6973746F7273202D206E6FF0
:1022E0002074656D7065726174757265004E6F2043
:1022F000746865726D6973746F7273202D206E6FD0
:102300002074656D7065726174757265004E6F2022
:10231000746865726D6973746F7273202D206E6FAF
:102320002074656D7065726174757265004E6F2002
:10233000746865726D6973746F7273202D206E6F8F
:102340002074656D7065726174757265004D32320E
:102350003120496E76616C696420657874727564A9
:10236000657220004D32323120496E76616C6964AD
:1023700020657874727564657220004D32323120A8
:10238000496E76616C6964206578747275646572F3
:1023900020004D32323120496E76616C69642065CF
:1023A0007874727564657220004D32323120496E46
:1023B00076616C696420657874727564657220005A
:1023C0004D32313820496E76616C696420657874CD
:1023D000727564657220004D32313820496E766125
:1023E0006C696420657874727564657220004D3282
:1023F000313820496E76616C696420657874727535
:1024000064657220004D32313820496E76616C6906
:102410006420657874727564657220004D323138BD
:1024200020496E76616C69642065787472756465A4
:102430007220004D32303020496E76616C69642024
:10244000657874727564657220004D3230302049B1
:102450006E76616C6964206578747275646572204B
:10246000004D32303020496E76616C6964206578A9
:1024700074727564657220004D32303020496E767A
:10248000616C696420657874727564657220004DB2
:1024900032303020496E76616C69642065787472E0
:1024A0007564657220004D31303520496E76616C5F
:1024B000696420657874727564657220004D3130EE
:1024C0003520496E76616C69642065787472756434
:1024D000657220004D31303520496E76616C69643B
:1024E00020657874727564657220004D3130352036
:1024F000496E76616C696420657874727564657282
:1025000020004D31303520496E76616C696420655C
:102510007874727564657220004D31303420496ED4
:1025200076616C69642065787472756465722000E8
:102530004D31303420496E76616C69642065787461
:10254000727564657220004D31303420496E7661B9
:102550006C696420657874727564657220004D3111
:10256000303420496E76616C6964206578747275C8
:1025700064657220004D31303420496E76616C699B
:10258000642065787472756465722000456E6420FD
:1025900066696C65206C69737400456E64206669B9
:1025A0006C65206C69737400456E642066696C65A7
:1025B000206C69737400456E642066696C65206CDC
:1025C00069737400456E642066696C65206C69737C
:1025D0007400426567696E2066696C65206C69737A
:1025E0007400426567696E2066696C65206C69736A
:1025F0007400426567696E2066696C65206C69735A
:102600007400426567696E2066696C65206C697349
:102610007400426567696E2066696C65206C697339
:102620007400446F6E65207072696E74696E672005
:1026300066696C6500446F6E65207072696E7469BE
:102640006E672066696C6500446F6E652070726904
:102650006E74696E672066696C6500446F6E6520F4
:102660007072696E74696E672066696C6500446F8C
:102670006E65207072696E74696E672066696C653C
:10268000004E6F204C696E65204E756D626572203C
:102690007769746820636865636B73756D2C204C73
:1026A000617374204C696E653A20004E6F204C694E
:1026B0006E65204E756D626572207769746820635F
:1026C0006865636B73756D2C204C617374204C6965
:1026D0006E653A20004E6F204C696E65204E756D18
:1026E000626572207769746820636865636B7375CF
:1026F0006D2C204C617374204C696E653A20004E3D
:102700006F204C696E65204E756D62657220776929
:10271000746820636865636B73756D2C204C6173FE
:1027200074204C696E653A20004E6F204C696E65CE
:10273000204E756D626572207769746820636865E4
:10274000636B73756D2C204C617374204C696E65DE
:102750003A20004E6F20436865636B73756D207778
:10276000697468206C696E65206E756D6265722C87
:10277000204C617374204C696E653A20004E6F20C6
:10278000436865636B73756D2077697468206C6945
:102790006E65206E756D6265722C204C61737420BD
:1027A0004C696E653A20004E6F20436865636B7319
:1027B000756D2077697468206C696E65206E756D23
:1027C0006265722C204C617374204C696E653A20EE
:1027D000004E6F20436865636B73756D2077697475
:1027E00068206C696E65206E756D6265722C204C78
:1027F000617374204C696E653A20004E6F20436807
:1028000065636B73756D2077697468206C696E659C
:10281000206E756D6265722C204C617374204C695A
:102820006E653A2000636865636B73756D206D6932
:10283000736D617463682C204C617374204C696EF5
:10284000653A2000636865636B73756D206D69730D
:102850006D617463682C204C617374204C696E65E3
:102860003A2000636865636B73756D206D69736DE5
:10287000617463682C204C617374204C696E653AF6
:102880002000636865636B73756D206D69736D619E
:102890007463682C204C617374204C696E653A2017
:1028A00000636865636B73756D206D69736D61742A
:1028B00063682C204C617374204C696E653A20006B
:1028C0004C696E65204E756D626572206973206E6D
:1028D0006F74204C617374204C696E65204E756D69
:1028E0006265722B312C204C617374204C696E65CB
:1028F0003A20004C696E65204E756D6265722069E4
:1029000073206E6F74204C617374204C696E652067
:102910004E756D6265722B312C204C617374204CA6
:10292000696E653A20004C696E65204E756D626572
:1029300072206973206E6F74204C617374204C692F
:102940006E65204E756D6265722B312C204C617363
:1029500074204C696E653A20004C696E65204E7596
:102960006D626572206973206E6F74204C617374A0
:10297000204C696E65204E756D6265722B312C207E
:102980004C617374204C696E653A20004C696E6529
:10299000204E756D626572206973206E6F74204CD5
:1029A000617374204C696E65204E756D6265722B83
:1029B000312C204C617374204C696E653A200044C0
:1029C0006F6E6520736176696E672066696C652E2F
:1029D00000446F6E6520736176696E672066696C6E
:1029E000652E00446F6E6520736176696E672066A0
:1029F000696C652E00446F6E6520736176696E6741
:102A00002066696C652E00446F6E6520736176697F
:102A10006E672066696C652E006F6B006F6B006FD0
:102A20006B006F6B006F6B002020506C616E6E65E9
:102A30007242756666657242797465733A20002049
:102A400020506C616E6E6572427566666572427981
:102A50007465733A20002020506C616E6E6572427E
:102A6000756666657242797465733A20002020505D
:102A70006C616E6E657242756666657242797465E8
:102A8000733A20002020506C616E6E65724275664C
:102A900066657242797465733A20002046726565F6
:102AA000204D656D6F72793A200020467265652071
:102AB0004D656D6F72793A20002046726565204D34
:102AC000656D6F72793A20002046726565204D650C
:102AD0006D6F72793A20002046726565204D656DF4
:102AE0006F72793A2000204C6173742055706461D4
:102AF0007465643A2000204C6173742055706461E1
:102B00007465643A2000204C6173742055706461D0
:102B10007465643A2000204C6173742055706461C0
:102B20007465643A2000204C6173742055706461B0
:102B30007465643A2000207C20417574686F723A95
:102B40002000207C20417574686F723A2000207C40
:102B500020417574686F723A2000207C20417574A2
:102B6000686F723A2000207C20417574686F723A59
:102B7000200020536F66747761726520526573651B
:102B8000740020536F6674776172652052657365B7
:102B9000740020536F6674776172652052657365A7
:102BA000740020536F667477617265205265736597
:102BB000740020536F667477617265205265736587
:102BC0007400205761746368646F67205265736591
:102BD0007400205761746368646F67205265736581
:102BE0007400205761746368646F67205265736571
:102BF0007400205761746368646F67205265736561
:102C00007400205761746368646F67205265736550
:102C100074002042726F776E206F75742052657356
:102C20006574002042726F776E206F757420526554
:102C3000736574002042726F776E206F7574205236
:102C400065736574002042726F776E206F75742013
:102C50005265736574002042726F776E206F7574D1
:102C6000205265736574002045787465726E616CDE
:102C7000205265736574002045787465726E616CCE
:102C8000205265736574002045787465726E616CBE
:102C9000205265736574002045787465726E616CAE
:102CA000205265736574002045787465726E616C9E
:102CB00020526573657400506F77657255700050CF
:102CC0006F776572557000506F7765725570005060
:102CD0006F776572557000506F776572557000653B
:102CE0006E717565696E67202200656E7175656924
:102CF0006E67202200656E717565696E672022001F
:102D0000656E717565696E67202200656E71756507
:102D1000696E672022007770726F772E207A6D6956
:102D2000616E007061726120746F6D617220656602
:102D30006563746F0020706572206D6F73747261CB
:102D4000726520692063616D622E002070726F20B1
:102D500070726F6A6576656E69207A6D656E0020A7
:102D6000666F722074616B652065666665637400CA
:102D700052657374617274206472756B61726B69F1
:102D8000005265696E6963696172206C6120696DCA
:102D9000702E005269617676696F206C61207374C1
:102DA000616D702E0052657374617274756A74651A
:102DB000207469736B61726E75005265626F6F7417
:102DC00020746865207072696E746572004D6F645E
:102DD000205B7720777964616A6E6F73635D004D65
:102DE0006F646F205B6D617320667565727A615DDB
:102DF000004D6F646F205B70697520666F727A6139
:102E00005D004D6F6420205B7679732E2076796BA0
:102E10006F6E5D004D6F6465205B68696768207048
:102E20006F7765725D004D6F642020202020202088
:102E30005B63696368795D004D6F646F20202020BB
:102E4000205B73696C656E63696F5D004D6F646FC5
:102E500020202020205B73696C656E7A696F736F28
:102E60005D004D6F64202020202020205B7469636A
:102E700068795D004D6F646520202020205B7369B8
:102E80006C656E745D0057796D69616E612066696D
:102E90006C616D656E74750043616D6269616E642D
:102EA0006F2066696C2E21004D757465766F6C65B8
:102EB0002066696C2E210056796D656E6120666909
:102EC0006C616D656E747521004368616E67696E33
:102ED000672066696C616D656E7421005770726F52
:102EE0007761647A2066696C616D656E7400496E05
:102EF00073657274612066696C616D656E746F00D4
:102F0000496E7365726972652066696C616D656E84
:102F1000746F00566C6F7A74652066696C616D65BC
:102F20006E7400496E736572742066696C616D65BC
:102F30006E74004E616369736E696A2070727A798B
:102F40006369736B00592070756C736520656C2024
:102F50006D616E646F00592070756C736520656CCF
:102F6000206D616E646F004120737469736B6E65D0
:102F7000746520746C616369746B6F00416E6420CA
:102F8000707265737320746865206B6E6F62005792
:102F9000796D69616E61206F6B210043616D6269BB
:102FA0006172206269656E210043616D6269612E04
:102FB00020726975736369746F21005A6D656E6163
:102FC0002075737065736E6121004368616E67657B
:102FD00020737563636573732100437A79737A6331
:102FE0007A2E206B6F6C6F72750043617267616E31
:102FF000646F20636F6C6F720043617267616E640F
:103000006F20636F6C6F720043697374656E692023
:103010006261727679004C6F6164696E6720636FDC
:103020006C6F720050726F737A6520637A656B61A2
:1030300063004573706572610041737065747461FB
:103040000050726F73696D2063656B656A7465000B
:10305000506C656173652077616974005770726F99
:10306000772E2066696C616D656E747500436172C0
:1030700067616E646F2066696C2E004361726761E0
:103080006E646F2066696C2E005A61766164656EAD
:10309000692066696C616D656E7475004C6F616462
:1030A000696E672066696C616D656E74004B6F6C4C
:1030B0006F72207A616E6965637A79737A2E004344
:1030C0006F6C6F72206E6F20636C61726F00436F64
:1030D0006C6F72206E6F20636C61726F0042617260
:1030E0007661206E656E6920636973746100436F59
:1030F0006C6F72206E6F7420636C65617200427237
:10310000616B2066696C616D656E74750046696CF3
:103110002E206E6F206361726761646F0046696C78
:103120002E206E6F206361726761646F0046696C68
:10313000616D656E74206E657A61766564656E009A
:1031400046696C616D656E74206E6F74206C6F6182
:10315000646564004E6965004E6F004E6F004E65F9
:10316000004E6F0054616B00536900536900416E5B
:103170006F005965730057796D69616E61206F6BDF
:103180003F0043616D626961646F20636F727265B5
:10319000632E3F0043616D626961746F20636F72DB
:1031A000722E3F0056796D656E61206F6B3F004354
:1031B00068616E67656420636F72726563746C79B1
:1031C0003F00506F6D6F6300537570706F727400C5
:1031D000537570706F727400506F64706F7261001D
:1031E000537570706F7274004E6167727A656A20F1
:1031F0006479737A65210050726563616C2E206575
:1032000078747275736F7221005072657269732ED3
:10321000207567656C6C6F2100507265646568721B
:10322000656A746520747279736B752100507265DC
:103230006865617420746865206E6F7A7A6C6521A8
:1032400000424C41443A004552524F523A004552D6
:10325000524F523A0043485942413A004552524F68
:10326000523A00526563747261637400526563740C
:1032700072616374005265637472616374005265B5
:103280006374726163740052656374726163740085
:103290005770726F7761647A2066696C616D656ED4
:1032A0007400496E74726F64756369722066696C2C
:1032B000616D656E746F0043617269636172652050
:1032C00066696C616D656E746F005A6176657374C2
:1032D0002066696C616D656E74004C6F6164206678
:1032E000696C616D656E740057796A616320666907
:1032F0006C616D656E740053616361722066696C08
:10330000616D656E746F00536361726963617265AC
:103310002066696C2E0056796A6D6F757420666937
:103320006C616D656E7400556E6C6F6164206669CA
:103330006C616D656E740047727A616E69650050EC
:10334000726563616C656E7461720050726572695A
:103350007363616C64610050726564656872657660
:1033600000507265686561740055737461776965B2
:103370006E696100416A7573746500496D706F73A1
:1033800074617A696F6E69004E6173746176656EFF
:10339000690053657474696E6773004B616C696290
:1033A0007261636A61204F4B0043616C69627261B4
:1033B0006369C383C692C382C2B36E204F4B00437E
:1033C000616C6962726174757261204F4B004B6170
:1033D0006C696272616365204F4B0043616C696286
:1033E000726174696F6E20646F6E65004B616C6909
:1033F0006272756A65205A0043616C696272616E1F
:10340000646F205A0043616C696272616E646F2060
:103410005A004B616C696272756A69205A00436197
:103420006C6962726174696E67205A004B616C69E5
:103430006272756A205A0043616C6962726172201F
:103440005A0043616C69627261205A004B616C6979
:1034500062726F766174205A0043616C69627261B6
:103460007465205A005679626572746520767974A5
:1034700069736B0056796265727465207679746938
:10348000736B00567962657274652076797469731E
:103490006B00567962657274652076797469736B16
:1034A000005069636B207072696E74004175746FAF
:1034B000646F7374726F6963205A3F004175746F53
:1034C000204D6963726F7061736F205A3F004175C0
:1034D000746F207265676F6C617265205A203F00BF
:1034E0004175746F20646F6C61646974205A203F69
:1034F000004175746F2061646A757374205A203FAF
:1035000000456E6473746F702061626F7274004561
:103510006E6473746F702061626F727400456E64C4
:1035200073746F702061626F727400456E6473749F
:103530006F702061626F727400456E6473746F7097
:103540002061626F727400446F7374726F6A656E8B
:103550006965206F7379205A004D6963726F7061DD
:10356000736F205A004261627973746570205A004B
:10357000446F6C6164656E69206F7379205A004CEA
:103580006976652061646A757374205A00426162CD
:103590007973746570205900426162797374657043
:1035A000205900426162797374657020590042614C
:1035B0006279737465702059004261627973746531
:1035C000702059004261627973746570205800421E
:1035D0006162797374657020580042616279737416
:1035E00065702058004261627973746570205800DC
:1035F00042616279737465702058005A204F666684
:10360000736574005A204F6666736574005A204FC4
:103610006666736574005A204F6666736574005A57
:10362000204F666673657400486F6D6520582F598A
:10363000206265666F7265205A00486F6D6520587C
:103640002F59206265666F7265205A00486F6D655C
:1036500020582F59206265666F7265205A00486FA6
:103660006D6520582F59206265666F7265205A007B
:10367000486F6D6520582F59206265666F7265200E
:103680005A005A2070726F6265206F75742E206226
:103690006564005A2070726F6265206F75742E2009
:1036A000626564005A2070726F6265206F75742EB7
:1036B00020626564005A2070726F6265206F7574B5
:1036C0002E20626564005A2070726F6265206F75EB
:1036D000742E206265640056796D656E697420539E
:1036E00044004368616E67652053442063617264DF
:1036F000004368616E676520534420636172640013
:1037000056796D656E6974205344004368616E6735
:1037100065205344206361726400496E69632E2002
:10372000534400496E69742E2053442063617264CF
:1037300000496E69742E205344206361726400490D
:103740006E69632E20534400496E69742E205344E1
:1037500020636172640057796D69656E69632066E4
:10376000696C616D656E740043616D6269617220A0
:1037700066696C616D656E746F0043616D6269614D
:1037800072652066696C616D656E746F0056796D47
:10379000656E69742066696C616D656E740043685E
:1037A000616E67652066696C616D656E7400417558
:1037B000746F526574722E004175746F5265747225
:1037C0002E004175746F526574722E004175746FCE
:1037D000526574722E004175746F526574722E00BA
:1037E000556E52657420205600556E526574202027
:1037F0005600556E52657420205600556E52657401
:1038000020205600556E52657420205600532055D6
:103810006E5265742B6D6D005320556E5265742B7E
:103820006D6D005320556E5265742B6D6D005320E5
:10383000556E5265742B6D6D005320556E52657434
:103840002B6D6D00556E526574202B6D6D00556E9D
:10385000526574202B6D6D00556E526574202B6D72
:103860006D00556E526574202B6D6D00556E52655E
:1038700074202B6D6D00486F70206D6D00486F7067
:10388000206D6D00486F70206D6D00486F70206D69
:103890006D00486F70206D6D0052657472616374C5
:1038A00020205600526574726163742020560052C5
:1038B000657472616374202056005265747261638E
:1038C0007420205600526574726163742020560083
:1038D000537761702052652E6D6D005377617020B3
:1038E00052652E6D6D00537761702052652E6D6D9F
:1038F00000537761702052652E6D6D0053776170B3
:103900002052652E6D6D0052657472616374206D76
:103910006D0052657472616374206D6D0052657440
:1039200072616374206D6D005265747261637420FE
:103930006D6D0052657472616374206D6D00535437
:103940004F505045442E20005041524144410041C7
:10395000525245535441544F200053544F505045F8
:10396000442E200053544F505045442E20004B49C4
:103970004C4C45442E200050415241444120444586
:1039800020454D4552472E0055434349534F200093
:103990004B494C4C45442E20004B494C4C45442E41
:1039A00020004E6F206D6F76652E0053696E206D7E
:1039B0006F76696D69656E746F004E657373756EB1
:1039C000204D6F76696D656E746F004E6F206D6F60
:1039D00076652E004E6F206D6F76652E00447275F1
:1039E0006B2070727A657277616E79005072696EC1
:1039F000742061626F72746564005374616D7061EC
:103A00002061626F7274697461005469736B207015
:103A10007265727573656E005072696E74206162B2
:103A20006F7274656400577A6E6F7769656E696549
:103A3000206472756B7500526573756D69656E648F
:103A40006F20696D7072652E0052697072656E64C8
:103A500069205374616D7061004F626E6F76656EA0
:103A600069207469736B7500526573756D696E6753
:103A7000207072696E74005761697420666F7220DD
:103A8000757365722E2E2E004573706572616E64BB
:103A90006F206F7264656E657300417474656E6447
:103AA00069205574656E74652E2E2E0057616974F9
:103AB00020666F7220757365722E2E2E0057616915
:103AC0007420666F7220757365722E2E2E00536CF3
:103AD0006565702E2E2E005265706F736F2E2E2E20
:103AE00000536F7370656E73696F6E652E2E2E00B6
:103AF000536C6565702E2E2E00536C6565702E2EEE
:103B00002E004272616B206B617274792053440005
:103B10004E6F20686179207461726A657461205308
:103B200044004E6F205344204361727461005A6117
:103B3000646E61205344206B61727461004E6F208B
:103B400053442063617264004472756B207A205381
:103B500044004D656E75206465205344004D656ECC
:103B600075205344204361727461005469736B2063
:103B70007A205344005072696E742066726F6D2013
:103B80005344005A6174727A796D6163206472756E
:103B90006B00446574656E657220696D7072657343
:103BA000696F6E0041727265737461207374616D28
:103BB0007061005A61737461766974207469736B03
:103BC0000053746F70207072696E74004B6F6E7466
:103BD000796E756F776163005265616E75646172AD
:103BE00020696D707265732E0052697072656E6423
:103BF00069207374616D706100506F6B7261636FE7
:103C000076617400526573756D65207072696E74AB
:103C10000050727A6572776163206472756B005030
:103C2000617573617220696D70726573696F6E0082
:103C3000506175736100506F7A6173746176697455
:103C4000207469736B005061757365207072696EC2
:103C500074004E617374726F696300416A757374A6
:103C6000617200416461747461004C616469740044
:103C700054756E65005072697072617661005072A1
:103C80006570617265005072657061726500507296
:103C90006970726176610050726570617265004989
:103CA0006E666F726D61636A65004D6F6E69746FE9
:103CB00072697A61720047756172646100496E666B
:103CC0006F726D61636500496E666F207363726524
:103CD000656E004F626E6F7669740052656672653C
:103CE00073680052656672657368004F626E6F7626
:103CF00069740052656672657368004F626E6F7614
:103D0000697420767963686F7A6900526573746F9D
:103D10007265206661696C736166650052657374D3
:103D20006F7265206661696C73616665004F626ED3
:103D30006F76697420767963686F7A69005265736B
:103D4000746F7265206661696C7361666500556C9D
:103D50006F7A69742070616D6574004C6F616420C6
:103D60006D656D6F7279004C6F6164206D656D6F6C
:103D7000727900556C6F7A69742070616D6574009A
:103D80004C6F6164206D656D6F72790053746F7252
:103D900065206D656D6F72790053746F7265206D6B
:103DA000656D6F72790053746F7265206D656D6F0C
:103DB00072790053746F7265206D656D6F72790052
:103DC00053746F7265206D656D6F7279004C43445A
:103DD00020636F6E7472617374004C434420636F90
:103DE0006E7472617374004C434420636F6E74721E
:103DF000617374004C434420636F6E74726173741A
:103E0000004C434420636F6E7472617374004669A2
:103E10006C2E204469612E20330046696C2E2044AC
:103E200069612E20330046696C2E204469612E2082
:103E3000330046696C2E204469612E2033004669A8
:103E40006C2E204469612E20330046696C2E20447C
:103E500069612E20320046696C2E204469612E2053
:103E6000320046696C2E204469612E20320046697A
:103E70006C2E204469612E20320046696C2E20444D
:103E800069612E20320046696C2E204469612E2023
:103E9000310046696C2E204469612E20310046694C
:103EA0006C2E204469612E20310046696C2E20441E
:103EB00069612E20310046696C2E204469612E20F4
:103EC00031004520696E206D6D33004520696E20FC
:103ED0006D6D33004520696E206D6D33004520699E
:103EE0006E206D6D33004520696E206D6D33004688
:103EF000696C616D656E740046696C616D656E74A8
:103F00000046696C616D656E740046696C616D6533
:103F10006E740046696C616D656E7400506F6879EF
:103F200062004D6F74696F6E004D6F74696F6E0043
:103F3000506F687962004D6F74696F6E0054656DE3
:103F400070657261747572610054656D706572613F
:103F5000747572610054656D70657261747572611B
:103F6000005465706C6F74610054656D70657261AA
:103F700074757265004573746570732F6D6D0045BF
:103F800073746570732F6D6D004573746570732F56
:103F90006D6D004573746570732F6D6D004573749E
:103FA0006570732F6D6D005A73746570732F6D6D2E
:103FB000005A73746570732F6D6D005A7374657059
:103FC000732F6D6D005A73746570732F6D6D005A89
:103FD00073746570732F6D6D005973746570732FF2
:103FE0006D6D005973746570732F6D6D0059737426
:103FF0006570732F6D6D005973746570732F6D6DDF
:10400000005973746570732F6D6D0058737465700B
:10401000732F6D6D005873746570732F6D6D00583C
:1040200073746570732F6D6D005873746570732FA2
:104030006D6D005873746570732F6D6D00412D7236
:1040400065747261637400412D726574726163748A
:1040500000412D7265747261637400412D72657444
:104060007261637400412D72657472616374004102
:104070006D61782000416D61782000416D6178208C
:1040800000416D61782000416D61782000565472C6
:104090006176206D696E005654726176206D696E8E
:1040A000005654726176206D696E005654726176C6
:1040B000206D696E005654726176206D696E0056EF
:1040C0006D696E00566D696E00566D696E00566DB5
:1040D000696E00566D696E006500650065006500DB
:1040E00065007A007A007A007A007A007900790017
:1040F00079007900790078007800780078007800FD
:10410000566D61782000566D61782000566D61789B
:104110002000566D61782000566D6178200056654C
:104120002D6A65726B0056652D6A65726B00566567
:104130002D6A65726B0056652D6A65726B00566557
:104140002D6A65726B00567A2D6A65726B00567A1D
:104150002D6A65726B00567A2D6A65726B00567A0D
:104160002D6A65726B00567A2D6A65726B005678FF
:10417000792D6A65726B005678792D6A65726B00CD
:104180005678792D6A65726B005678792D6A65725A
:104190006B005678792D6A65726B00416363656CBC
:1041A00000416363656C00416363656C0041636358
:1041B000656C00416363656C005049442D430050B9
:1041C00049442D43005049442D43005049442D4358
:1041D000005049442D43005049442D440050494467
:1041E0002D44005049442D44005049442D44005072
:1041F00049442D44005049442D49005049442D491B
:10420000005049442D49005049442D49005049442B
:104210002D49005049442D50005049442D50005024
:1042200049442D50005049442D50005049442D50D0
:10423000004F6666004F6666004F6666004F666612
:10424000004F6666004F6E20004F6E20004F6E20BC
:10425000004F6E20004F6E20004175746F74656DC5
:1042600070004175746F74656D70004175746F7482
:10427000656D70004175746F74656D700041757483
:104280006F74656D70002002204661637400200227
:10429000204661637400200220466163740020029E
:1042A000204661637400200220466163740020028E
:1042B000204D6178002002204D6178002002204DC1
:1042C0006178002002204D6178002002204D617845
:1042D000002002204D696E002002204D696E0020F2
:1042E00002204D696E002002204D696E00200220E0
:1042F0004D696E004B6F6E74726F6C6100436F6E30
:1043000074726F6C00436F6E74726F6C004B6F6EE3
:1043100074726F6C6100436F6E74726F6C005072D8
:1043200075746F6B203200466C6F77203200466CDC
:104330006F77203200507275746F6B203200466CBC
:104340006F77203200507275746F6B203100466CAD
:104350006F77203100466C6F772031005072757492
:104360006F6B203100466C6F77203100507275748E
:104370006F6B203000466C6F77203000466C6F7793
:10438000203000507275746F6B203000466C6F7770
:1043900020300050727A65706C797700466C756ACF
:1043A0006F00466C7573736F00507275746F6B009D
:1043B000466C6F7700507265646B6F73632077652E
:1043C0006E742E0056656E74696C61646F7200566F
:1043D000656E746F6C6100527963686C6F737420E2
:1043E00076656E742E0046616E207370656564009C
:1043F00053746F6C696B004261736500506961743E
:10440000746F004265640042656400547279736B96
:104410006133004E6F7A7A6C6533004E6F7A7A6C36
:10442000653300547279736B6133004E6F7A7A6C26
:10443000653300547279736B6132004E6F7A7A6C17
:104440006532004E6F7A7A6C653200547279736B04
:104450006132004E6F7A7A6C6532004479737A610A
:10446000004675736F72005567656C6C6F0054720F
:1044700079736B61004E6F7A7A6C65005072656477
:104480006B6F73630056656C6F636964616400569B
:10449000656C636974C383C692C386E28099C383E3
:1044A000E2809AC382C2A000527963686C6F737411
:1044B00000537065656400506F73756E6F7574207E
:1044C0006F2031306D6D004D6F76652031306D6D30
:1044D000004D6F76652031306D6D00506F73756ED5
:1044E0006F7574206F2031306D6D004D6F766520D3
:1044F00031306D6D00506F73756E6F7574206F2065
:10450000316D6D004D6F766520316D6D004D6F76AC
:104510006520316D6D00506F73756E6F7574206F0F
:1045200020316D6D004D6F766520316D6D00506FDF
:1045300073756E6F7574206F20302E316D6D004D68
:104540006F766520302E316D6D004D6F76652030B1
:104550002E316D6D00506F73756E6F7574206F2006
:10456000302E316D6D004D6F766520302E316D6DC2
:10457000004578747275646572330045787472759D
:1045800064657233004578747275646572330045F2
:1045900078747275646572330045787472756465F9
:1045A00072330045787472756465723200457874B0
:1045B0007275646572320045787472756465723222
:1045C000004578747275646572320045787472754E
:1045D000646572320045787472756465720045785E
:1045E000747275736F72004573747275736F726550
:1045F00000457874727564657200457874727564EC
:1046000065720050727A6573756E6163205A004D51
:104610006F766572205A004D756F7669205A00508A
:104620006F73756E6F7574205A004D6F7665205AE2
:104630000050727A6573756E61632059004D6F7614
:1046400065722059004D756F7669205900506F735F
:10465000756E6F75742059004D6F76652059005046
:10466000727A6573756E61632058004D6F7665725E
:104670002058004D756F7669205800506F73756E25
:104680006F75742058004D6F766520580052756321
:1046900068206F7369004D6F76657220656A657377
:1046A000004D756F7669204173736500506F7375A7
:1046B0006E6F7574206F7375004D6F76652061782D
:1046C000697300526574726163740052657472613B
:1046D0006374005265747261637400526574726130
:1046E0006374005265747261637400457874727506
:1046F000646F7661740045787472756465004578FE
:104700007472756465004578747275646F7661744F
:104710000045787472756465005A61706E6F7574C7
:10472000207A64726F6A0053776974636820706FCF
:10473000776572206F6666005377697463682070CE
:104740006F776572206F6666005A61706E6F757460
:10475000207A64726F6A0053776974636820706F9F
:10476000776572206F6666005679706E6F7574207B
:104770007A64726F6A0053776974636820706F7728
:104780006572206F6E0053776974636820706F776D
:104790006572206F6E005679706E6F7574207A6442
:1047A000726F6A0053776974636820706F776572FF
:1047B000206F6E00577963686C6F647A6963004597
:1047C0006E667269617200526166667265646461E8
:1047D000005A63686C6164697400436F6F6C646F46
:1047E000776E005072656465687265762041425349
:1047F00020636F6E66005072656865617420414287
:104800005320636F6E660050726568656174204165
:10481000425320636F6E660050726564656872650E
:10482000762041425320636F6E6600507265686562
:1048300061742041425320636F6E6600507265645C
:10484000656872657620414253204265640050726B
:10485000656865617420414253204265640050726E
:10486000656865617420414253204265640050725E
:104870006564656872657620414253204265640034
:10488000507265686561742041425320426564003E
:104890005072656465687265762041425320416CB0
:1048A0006C00507265686561742041425320416C10
:1048B0006C00507265686561742041425320416C00
:1048C0006C005072656465687265762041425320C1
:1048D000416C6C00507265686561742041425320E0
:1048E000416C6C0050726564656872657620414267
:1048F0005320330050726568656174204142532033
:104900003300507265686561742041425320330062
:1049100050726564656872657620414253203300A9
:1049200050726568656174204142532033005072B3
:10493000656465687265762041425320320050728A
:104940006568656174204142532032005072656889
:10495000656174204142532032005072656465687D
:10496000726576204142532032005072656865615D
:10497000742041425320320050726564656872654C
:104980007620414253203100507265686561742081
:104990004142532031005072656865617420414284
:1049A000532031005072656465687265762041421B
:1049B0005320310050726568656174204142532074
:1049C000310050726564656872657620414253001B
:1049D0005072656865617420414253005072656889
:1049E0006561742041425300507265646568726568
:1049F00076204142530050726568656174204142DF
:104A0000530050726564656872657620504C412091
:104A1000636F6E66005072656865617420504C412A
:104A200020636F6E66005072656865617420504C3B
:104A30004120636F6E6600507265646568726576CA
:104A400020504C4120636F6E66005072656865614E
:104A50007420504C4120636F6E660050726564652F
:104A60006872657620504C41204265640050726542
:104A70006865617420504C41204265640050726545
:104A80006865617420504C41204265640050726535
:104A900064656872657620504C4120426564005020
:104AA00072656865617420504C4120426564005015
:104AB000726564656872657620504C4120416C6C6B
:104AC000005072656865617420504C4120416C6CE7
:104AD000005072656865617420504C4120416C6CD7
:104AE0000050726564656872657620504C412041C3
:104AF0006C6C005072656865617420504C412041B7
:104B00006C6C0050726564656872657620504C412B
:104B10002033005072656865617420504C41203329
:104B2000005072656865617420504C41203300501C
:104B3000726564656872657620504C412033005080
:104B400072656865617420504C4120330050726575
:104B500064656872657620504C4120320050726561
:104B60006865617420504C41203200507265686560
:104B7000617420504C412032005072656465687247
:104B8000657620504C412032005072656865617432
:104B900020504C4120320050726564656872657621
:104BA00020504C412031005072656865617420507E
:104BB0004C412031005072656865617420504C4151
:104BC00020310050726564656872657620504C41F2
:104BD0002031005072656865617420504C4120316D
:104BE0000050726564656872657620504C410050D3
:104BF00072656865617420504C410050726568654B
:104C0000617420504C41005072656465687265762D
:104C100020504C41005072656865617420504C41D1
:104C2000004E617374617620706F636174656B0010
:104C3000536574206F726967696E00536574206FE5
:104C4000726967696E004E617374617620706F637C
:104C50006174656B00536574206F726967696E00DB
:104C60004E617374617620706F636174656B206848
:104C70006F6D650053657420686F6D65206F6666A3
:104C8000736574730053657420686F6D65206F667B
:104C90006673657473004E617374617620706F6320
:104CA0006174656B20686F6D650053657420686F73
:104CB0006D65206F666673657473004175746F204F
:104CC000686F6D65004C6C6576617220616C206F59
:104CD000726967656E004175746F20486F6D65007D
:104CE0004175746F20686F6D65004175746F206841
:104CF0006F6D650057796C61637A79632073696CB5
:104D00006E696B6900417061676172206D6F746FCD
:104D1000726573004469736162696C697461204DE6
:104D20006F746F7269005679706E6F7574206D6F55
:104D3000746F72790044697361626C652073746585
:104D40007070657273004175746F73746172740072
:104D50004175746F7374617274004175746F73740C
:104D6000617274004175746F73746172740041757F
:104D7000746F7374617274004D656E7520676C6F2B
:104D8000776E65004D656E75207072696E6369702F
:104D9000616C004D656E75207072696E636970613B
:104DA0006C6500486C61766E69206E616269646B47
:104DB00061004D61696E004B617274612077796AA0
:104DC000657461005461726A65746120726574690A
:104DD0007261646100534420436172642072696DA2
:104DE0006F737361004B617274612076796A6D75BF
:104DF000746100436172642072656D6F7665640052
:104E00004B6172746120776C6F7A6F6E61005461D0
:104E1000726A65746120636F6C6F636164610053D3
:104E200044204361726420696E7365726974610025
:104E30004B6172746120766C6F7A656E61004361BC
:104E4000726420696E736572746564005072757364
:104E500061206933204D4B3220676F746F7761009A
:104E60005072757361206933204D4B32206C697329
:104E70007461005072757361206933204D4B32208C
:104E800070726F6E746F2E0050727573612069338B
:104E9000204D4B32206F6B00507275736120693367
:104EA000204D4B322072656164792E004D383420DC
:104EB000582059205A2045004D3234004D323320BD
:104EC0002573006175746F25692E67000A002F0035
:104ED0000A002E0044656C6574696F6E2066616916
:104EE0006C65642C2046696C653A200046696C65E7
:104EF0002064656C657465643A002E002E002E00F7
:104F00002E004E6F772066726573682066696C6547
:104F10003A20004E6F7720646F696E672066696C77
:104F2000653A20002220706F730022207061726544
:104F30006E743A2200535542524F5554494E452003
:104F400043414C4C207461726765743A220074725C
:104F500079696E6720746F2063616C6C2073756271
:104F60002D67636F64652066696C6573207769746B
:104F70006820746F6F206D616E79206C6576656C4A
:104F8000732E204D4158206C6576656C2069733A0C
:104F90000000002110422063308440A550C660E725
:104FA00070088129914AA16BB18CC1ADD1CEE1EFDE
:104FB000F13112100273325222B5529442F772D676
:104FC00062399318837BB35AA3BDD39CC3FFF3DE2E
:104FD000E36224433420040114E664C774A44485C6
:104FE000546AA54BB528850995EEE5CFF5ACC58D7E
:104FF000D55336722611163006D776F6669556B416
:10500000465BB77AA719973887DFF7FEE79DD7BCCD
:10501000C7C448E5588668A7784008611802282365
:1050200038CCC9EDD98EE9AFF9488969990AA92B1D
:10503000B9F55AD44AB77A966A711A500A333A12B5
:105040002AFDDBDCCBBFFB9EEB799B588B3BBB1A6D
:10505000ABA66C877CE44CC55C222C033C600C4105
:105060001CAEED8FFDECCDCDDD2AAD0BBD688D49BD
:105070009D977EB66ED55EF44E133E322E511E7055
:105080000E9FFFBEEFDDDFFCCF1BBF3AAF599F780D
:105090008F8891A981CAB1EBA10CD12DC14EF16FBE
:1050A000E18010A100C230E3200450254046706723
:1050B00060B9839893FBA3DAB33DC31CD37FE35E4F
:1050C000F3B1029012F322D2323542145277625673
:1050D00072EAB5CBA5A89589856EF54FE52CD50D5F
:1050E000C5E234C324A014810466744764245405C3
:1050F00044DBA7FAB79987B8975FE77EF71DC73CEF
:10510000D7D326F2369106B0165766767615463412
:10511000564CD96DC90EF92FE9C899E9898AB9ABFE
:10512000A94458654806782768C018E1088238A362
:10513000287DCB5CDB3FEB1EFBF98BD89BBBAB9A8E
:10514000BB754A545A376A167AF10AD01AB32A92B2
:105150003A2EFD0FED6CDD4DCDAABD8BADE89DC99E
:105160008D267C076C645C454CA23C832CE01CC102
:105170000C1FEF3EFF5DCF7CDF9BAFBABFD98FF82E
:105180009F176E367E554E745E932EB23ED10EF052
:105190001E22004D3232302053256900203A200073
:1051A000004C414E472053454C20464F5243454406
:1051B000002200205A3A0020593A0020453A0020A7
:1051C0005A3A0020593A00583A0020002E00204256
:1051D0003A0020453A00543A0020573A0020453A18
:1051E00000543A002042403A0020403A00202F006C
:1051F0003A00205400202F0020423A00202F006F58
:105200006B20543A002569206D696E2C2025692099
:1052100073656300496E646578206F7574206F66EE
:1052200020626F756E6473000A0042656420666FC9
:10523000756E642061743A200046696E64696E6719
:105240002062656420004D65736820626564206C8F
:105250006576656C696E67206E6F74206163746932
:1052600076652E000A002020000A4D656173757274
:10527000656420706F696E74733A000A5A20736512
:1052800061726368206865696768743A20002C0061
:105290004E756D20582C593A20004738300047325F
:1052A000380047383000256920686F7572732025F3
:1052B00069206D696E75746573004D313130004D34
:1052C0003239004D6179203330203230313600439D
:1052D0006F6D70696C65643A2000286E6F6E652C86
:1052E0002064656661756C7420636F6E66696729FA
:1052F000004D617920333020323031362031363A5A
:1053000032333A3037007374617274002200220025
:10531000FFFFFF0000A0400000A040000000400090
:10532000007F4300005643CDCC51430000000000F5
:105330000080C0CDCC4C3E00007F430000524300B3
:1053400000524300000000000080C0CDCC4C3E6500
:1053500063686F3A004572726F723A0047383000E6
:10536000473120452D38302046343030004D383319
:10537000004731205A313520463135303000473929
:1053800031004731205835302059313930204530EF
:1053900020463730303000473930004D3834004D2A
:1053A000383300473120453730204634303000470D
:1053B00031204534302046313030002E002020206E
:1053C00020202020202020202020002D2D3A2D2DAF
:1053D000002D2D2D003E555342005344002D2D002D
:1053E0000120000120004D36303000464C45582049
:1053F0002D20203233302F35300050502020202DEA
:1054000020203235342F3130300048495053202D80
:1054100020203232302F3130300050455420202DA2
:1054200020203234302F393000504C4120202D20A4
:10543000203231302F35300041425320202D2020A2
:105440003235352F313030004D3234004D3233207B
:10545000257300580059005A0045787472756465C8
:105460007200473238004D3834004D6179203330B6
:10547000203230313600446174653A20002D2D2DE4
:105480002D2D2D2D2D2D2D2D2D00453344763666B9
:10549000756C6C0052414D426F31336100315F37A2
:1054A000356D6D5F4D4B32002D2D2D2D2D2D2D2D5C
:1054B0002D2D2D2D004669726D77617265202D208E
:1054C000332E302E310048617264636F646564204E
:1054D00044656661756C742053657474696E677396
:1054E000204C6F616465640046696C616D656E7423
:1054F0002073657474696E67733A204469736162DE
:105500006C6564002020204D323030204400466914
:105510006C616D656E742073657474696E67733A3F
:10552000002020204D3230392053004175746F2DFA
:10553000526574726163743A20533D3020746F2059
:1055400064697361626C652C203120746F20696E10
:105550007465727072657420657874727564652DF7
:105560006F6E6C79206D6F76657320617320726544
:10557000747261637473206F72207265636F7665F5
:1055800072696573002046002020204D323038209B
:1055900053005265636F7665723A20533D457874C7
:1055A0007261206C656E67746820286D6D292046D5
:1055B0003A537065656420286D6D2F6D2900205A5F
:1055C000002046002020204D323037205300526505
:1055D00074726163743A20533D4C656E6774682041
:1055E000286D6D2920463A537065656420286D6DDD
:1055F0002F6D29205A3A205A4C69667420286D6D07
:1056000029002044002049002020204D3330312043
:1056100050005049442073657474696E67733A0092
:10562000205A0020590020204D32303620580048A2
:105630006F6D65206F666673657420286D6D293AFD
:1056400000204500205A002058002042002054002D
:1056500020204D323035205300416476616E636501
:1056600064207661726961626C65733A20533D4DC6
:10567000696E20666565647261746520286D6D2FA2
:1056800073292C20543D4D696E2074726176656CCF
:1056900020666565647261746520286D6D2F7329BD
:1056A0002C20423D6D696E696D756D207365676D67
:1056B000656E742074696D6520286D73292C2058DF
:1056C0003D6D6178696D756D205859206A65726B02
:1056D00020286D6D2F73292C20205A3D6D6178692B
:1056E0006D756D205A206A65726B20286D6D2F7361
:1056F000292C2020453D6D6178696D756D20452010
:105700006A65726B20286D6D2F732900205400206C
:10571000204D323034205300416363656C65726103
:1057200074696F6E3A20533D616363656C657261A5
:1057300074696F6E2C20543D7265747261637420BD
:10574000616363656C65726174696F6E002045000A
:10575000205A0020590020204D3230312058004D71
:105760006178696D756D20416363656C6572617404
:10577000696F6E20286D6D2F7332293A0020450025
:10578000205A0020590020204D3230332058004D3F
:105790006178696D756D20666565647261746573A5
:1057A00020286D6D2F73293A00204500205A0020D3
:1057B000590020204D3932205800537465707320F1
:1057C00070657220756E69743A0045303A20005A4F
:1057D0003A2000593A2000583A20004D53312C4DC0
:1057E00053322050696E730A005A00205A3A005909
:1057F0000020593A00580020583A0024F4D4305080
:10580000C38E20C2A24017828B7011127A910D8133
:105810006CD90AA861E108C7586607615143061EA2
:105820004B5D05C145A7041A411104093D98037158
:105830003931034036DB0265339102D430540280A3
:105840002E1D02632CEE01752AC501B028A001109F
:105850002781018F2564012B244B01E0223401AC08
:10586000211F018D200D01801FFC00841EED00977B
:105870001DDF00B81CD200E61BC600201BBC006464
:105880001AB200B219A8000A19A0006A189900D12A
:1058900017910040178B00B516840031167E00B3B7
:1058A0001579003A157300C7146F0058146A00EE9A
:1058B0001366008813630025135E00C7125B006C3B
:1058C00012570015125400C111510070114F0021E0
:1058D000114B00D61049008D1047004610440002BD
:1058E000104200C00F4000800F3E00420F3C0006F7
:1058F0000F3B00CB0E3800930E37005C0E350027AF
:105900000E3400F30D3200C10D3100900D300060F7
:105910000D2E00320D2D00050D2C00D90C2B00AEE4
:105920000C2900850C29005C0C2700350C27000E83
:105930000C2600E80B2400C40B2400A00B23007DE0
:105940000B23005A0B2100390B2100180B2000F803
:105950000A1F00D90A1E00BB0A1E009D0A1D0080F6
:105960000A1D00630A1C00470A1B002C0A1B0011B9
:105970000A1A00F7091A00DD091900C4091900AB59
:10598000091900920917007B091800630917004CD8
:1059900009160036091600200916000A091500F537
:1059A000081500E0081400CC081400B8081400A47E
:1059B000081400900813007D0812006B08130058AB
:1059C00008120046081200340811002308110012C2
:1059D00008110001081100F0071000E0071000D0C6
:1059E000071000C0071000B0070F00A107100091BA
:1059F000070E0083070F0074070F0065070E00579E
:105A0000070E0049070E003B070D002E070E002071
:105A1000070D0013070D0006070D00F9060C00ED39
:105A2000060D00E0060C00D4060C00C8060C00BCF5
:105A3000060C00B0060C00A4060B0099060C008DA5
:105A4000060B0082060B0077060B006C060B00614C
:105A5000060A0057060B004C060A0042060A0038E8
:105A6000060A002E060A0024060A001A060A00107A
:105A700006090007060A00FD050900F4050900EB08
:105A8000050900E2050900D9050900D0050900C78C
:105A9000050900BE050900B5050800AD050800A50B
:105AA0000509009C050800940508008C0508008481
:105AB0000508007C050800740508006C05070065F2
:105AC0000508005D050700560508004E050700475C
:105AD0000507004005080038050700310507002AC2
:105AE000050700230507001C050600160507000F23
:105AF0000507000805060002050700FB040600F57F
:105B0000040700EE040600E8040600E2040700DBD8
:105B1000040600D5040600CF040600C9040600C32D
:105B2000040600BD040600B7040600B1040500AC7D
:105B3000040600A6040600A00405009B04060095C8
:105B4000040500900406008A040500850405008011
:105B50000406007A04050075040500700405006B56
:105B600004050066040500610405005C0405005797
:105B7000040500520405004D0405004804050043D7
:105B80000405003E0404003A040500350405003015
:105B90000404002C04050027040400230405001E4F
:105BA0000404001A04040016040500110404000D86
:105BB000040400090405000404040000040400FCBB
:105BC000030400F8030400F4030400F0030400ECF1
:105BD000030400E8030400E4030400E0030400DC21
:105BE000030400D8030400D4030400D0030400CC51
:105BF000030400C8030300C503030024F404D920F0
:105C00001BC40C5C0E9804C4095F0265077101F4A3
:105C100005F900FB04B30048048700C1036900587C
:105C200003550003034500BE023A008402310053CD
:105C3000022A002902250004022000E4011C00C8F9
:105C4000011900AF011700980114008401130071BD
:105C50000110006101100051010E0043010D0036DA
:105C6000010B002B010B0020010B00150109000C9A
:105C700001090003010800FB000800F3000800EB25
:105C8000000700E4000600DE000600D8000600D28F
:105C9000000600CC000500C7000500C2000500BDDD
:105CA000000400B9000400B5000400B1000400AD18
:105CB000000400A9000400A5000300A20003009F47
:105CC0000004009B0003009800030095000200936D
:105CD000000300900003008D0002008B0003008889
:105CE0000002008600020084000300810002007FA1
:105CF0000002007D0002007B0002007900020077B4
:105D000000010076000200740002007200010071C0
:105D10000002006F0002006D0001006C0002006ACA
:105D200000010069000200670001006600010065D3
:105D300000010064000200620001006100010060D7
:105D40000001005F0002005D0001005C0001005BDB
:105D50000001005A000100590001005800010057DD
:105D600000010056000100550001005400010053DD
:105D700000000053000100520001005100010050DA
:105D80000001004F0001004E0000004E0001004DD8
:105D90000001004C0001004B0000004B0001004AD4
:105DA00000010049000100480000004800010047D0
:105DB00000010046000000460001004500000045CB
:105DC00000010044000100430000004300010042C4
:105DD00000000042000100410000004100010040BD
:105DE0000001003F0000003F0001003E0000003EB7
:105DF0000001003D0000003D0001003C0000003CAF
:105E00000000003C0001003B0000003B0001003AA4
:105E10000000003A0001003900000039000100389C
:105E20000000003800000038000100370000003793
:105E30000001003600000036000000360001003589
:105E4000000000350000003500010034000000347F
:105E50000000003400010033000000330000003374
:105E60000001003200000032000000320001003169
:105E7000000000310000003100010030000000305F
:105E8000000000300001002F0000002F0000002F54
:105E90000000002F0001002E0000002E0000002E48
:105EA0000001002D0000002D0000002D0000002D3D
:105EB0000001002C0000002C0000002C0000002C31
:105EC0000001002B0000002B0000002B0000002B25
:105ED0000001002A0000002A0000002A0000002A19
:105EE000000100290000002900000029000000290D
:105EF0000000002900010028000000280000002800
:105F000000000028000000280001002700000027F2
:105F100000000027000000270000002700010026E5
:105F200000000026000000260000002600000026D9
:105F300000010025000000250000002500000025CC
:105F400000000025000000250001002400000024BE
:105F500000000024000000240000002400010023B1
:105F600000000023000000230000002300000023A5
:105F70000000002300000023000100220000002296
:105F80000000002200000022000000220000002289
:105F9000000100210000002100000021000000217C
:105FA000000000210000002100000021000100206D
:105FB0000000002000000020000000200000002061
:105FC0000000002000000020000000200001001F51
:105FD0000000001F0000001F0000001F0000001F45
:105FE0000000001F0000001F0001001E0000001E36
:105FF0000000001E0000001E0000000000090A0250
:10600000080B0C0D0706030401000000000000004F
:106010000000000000000000000000000000000080
:106020000000000000000011100F00000000000040
:106030000000000000000000000000000000000060
:106040000000000000000000000000000000000050
:10605000000102102020080810204010204080027B
:10606000010201080402010102040810204080809E
:106070004020100804020180040201804020100822
:1060800004020108040201010204081020408001FA
:1060900002040810204080100804088010204004EA
:1060A0004080102040048005050505070508080804
:1060B00008020202020A0A08080404040401010199
:1060C00001010101010303030303030303040707A1
:1060D000070C0C0C0C0C0C0C0C020202020606063F
:1060E00006060606060B0B0B0B0B0B0B0B07070A22
:1060F0000A0A0A0A0A050505040404080800002023
:10610000002300260029002C002F0032000001008F
:106110000003010601090100002200250028002BD0
:10612000002E003100340002010000050108010BBF
:106130000100002100240027002A002D0030003338
:106140000001010000040107010A01024E414E490D
:106150004E495459494E46CDCCCC3D0AD7233C1725
:10616000B7D13877CC2B329595E6241FB14F0A0072
:106170000020410000C84200401C4620BCBE4CCA62
:106180001B0E5AAEC59D74009D973AB78FE984FBEC
:10619000A19711241FBECFEFD1E2DEBFCDBF00E03B
:1061A0000CBF1EE0A0E0B2E0ECECF4E202E00BBFBA
:1061B00002C007900D92AE3CB107D9F72FE1AEECCB
:1061C000BEE001C01D92A232B207E1F711E6C0E9BC
:1061D000D1E600E006C022970109FE010BBF0F9433
:1061E000B309C838D10780E00807A9F70E9488FFE3
:1061F0000D9454120C940000CF93DF93EC019C019A
:106200002C5F3F4F41E050E060E070E0898D9A8D57
:106210000E949E3B882399F04D895E896F89788D15
:10622000452B462B472B59F44C815D816E817F8134
:106230004D8B5E8B6F8B788F998190689983DF91FE
:10624000CF910895CF92DF92EF92FF920F931F9319
:10625000CF93DF93EC0189899A89AB89BC89803E11
:106260009F4FAF41B10510F080E06BC0CE01C4DF9D
:106270008823D1F30E94B239182F8823A9F3E98D1E
:10628000FA8DCC80DD80EE80FF8032E0C31AD10829
:10629000E108F108058404C0CC0CDD1CEE1CFF1CD9
:1062A0000A94D2F786859785A089B189C80ED91E30
:1062B000EA1EFB1E81E08093D40EC092D710D092CC
:1062C000D810E092D910F092DA1080E092E0E7ED79
:1062D000FEE0DF019C011D9221503040E1F701E01A
:1062E000E98DFA8D8481081790F427ED3EE0B7011F
:1062F000A601400F511D611D711D8091D50E909119
:10630000D60E0E9496628823E1F00F5FE9CFC12C80
:1063100082E0D82EE12CF12C058404C0CC0CDD1CCD
:10632000EE1CFF1C0A94D2F749895A896B897C8933
:106330004C0D5D1D6E1D7F1D498B5A8B6B8B7C8BAD
:10634000812FDF91CF911F910F91FF90EF90DF9000
:10635000CF900895CF93DF93EC0141E0611101C02C
:1063600040E06C857D858E859F850E94F23988236B
:1063700041F0888920E2829FC00111248952914F07
:1063800002C080E090E0DF91CF91089530E020E0FE
:106390004EE2DC015C91503271F0383029F4FB019F
:1063A000E20FF11D40832F5FFB01E20FF11DDC01C5
:1063B0005C9150832F5F3F5F01963B3051F7FB01AB
:1063C000E20FF11D10820895CF93DF93EB01FC01E2
:1063D0002381211102C080E00EC02250223020F41F
:1063E0008FE28883198206C060E0B4DF009799F3DA
:1063F000BE01CCDF81E0DF91CF910895FB012BE05E
:1064000030E231932150E9F7DC0190E027E03A2FA8
:10641000EB2F8D9181110AC0DA013C931196EC9318
:1064200081E0FB019081903239F525C08F32A1F3D4
:106430008E3219F0EEE8F1E008C02A30E1F098E081
:106440002AE0E5CF31963817B1F034913111FACF07
:10645000291788F03FED380F3E3568F431E0390FE9
:10646000FB01E90FF11D9FE9980F9A3108F4805262
:106470008083932FCCCF80E008950F931F93CF9309
:10648000DF93EC018B018B81882311F080E042C007
:10649000FB018789803139F18032C1F783E08B833A
:1064A000F801428D538D648D758D4D8B5E8B6F8B96
:1064B000788F9E012F5E3F4FC8010E94A93A882322
:1064C00029F31A8F098F81E089831C821D821E8225
:1064D0001F82188619861A861B861C861D861E86B4
:1064E0001F86188A17C082E08B831D8A1E8A1F8A26
:1064F000188EFB01408D518D60E070E095E0440FF7
:10650000551F661F771F9A95D1F7498B5A8B6B8B56
:106510007C8BD7CFDF91CF911F910F9108952F9250
:106520003F924F925F926F927F928F929F92AF9223
:10653000BF92CF92DF92EF92FF920F931F93CF9370
:10654000DF93EC015B016A018B81811103C08FEF46
:106550009FEFC7C0898180FFFACF49895A896B892B
:106560007C8988859985AA85BB852601612C712C3B
:106570008A019B01081B190B2A0B3B0B4016510685
:106580006206730618F06A01C81AD90A76013E013C
:1065900024E0620E711CE114F10409F476C0488510
:1065A00059856A857B854A0181E098222B811A01F1
:1065B0002B01E9E05694479437942794EA95D1F754
:1065C000898D9A8DFC01223049F4628D738D848D02
:1065D000958D620D731D841D951D3CC01481115055
:1065E000122181149104C1F4111116C0452B462BC0
:1065F000472B49F48D899E89AF89B88D8C839D8303
:10660000AE83BF8309C04C815D816E817F81930120
:1066100021D7882309F49BCFE98DFA8D6C817D8188
:106620008E819F816250710981099109058404C09E
:10663000660F771F881F991F0A94D2F72685378522
:1066400040895189620F731F841F951F610F711D4F
:10665000811D911D20E032E02819390987012E158E
:106660003F0508F489010115F2E01F0769F5209143
:10667000D7103091D8104091D9105091DA1062178C
:1066800073078407950719F41FC0C6012AC0950136
:10669000AB01BC018091D50E9091D60E0E94216273
:1066A000882309F454CFA00EB11E88859985AA8548
:1066B000BB85800F911FA11DB11D88879987AA876F
:1066C000BB87E01AF10A67CF40E08CD6882309F433
:1066D0003ECFB4016952714FA801C5010F94E40E79
:1066E000E2CFDF91CF911F910F91FF90EF90DF905C
:1066F000CF90BF90AF909F908F907F906F905F9062
:106700004F903F902F900895CF93DF931F92CDB776
:10671000DEB741E050E0BE016F5F7F4F00DF0197C1
:1067200019F4898190E002C08FEF9FEF0F90DF9105
:10673000CF910895CF92DF92EF92FF920F931F9324
:10674000CF93DF936C01EB017A01FC0183818230EE
:1067500060F000851185228533850F71112722276E
:106760003327012B022B032B11F08FEF5CC0411557
:10677000510511F0F70110821DE040E250E0BE012A
:10678000C601CDDE8032910539F021E0892B09F474
:1067900020E0822F819547C028812223C1F0253E29
:1067A00061F32E3251F33B853F733F3061F4E114C6
:1067B000F10449F04A8D5B8D452B29F42F713FEF91
:1067C000320F343030F02B8523FDD7CF2CC080E042
:1067D0002AC030E021503109129FC001139F900D53
:1067E0001124F701E80FF91F298120832B812183D0
:1067F0002D8122832F812383298524832E85258340
:10680000288926832A8927832C8920872E89218716
:10681000288D22872C8D23872E8D2487288126FF83
:10682000D2CF1586D0CFDF91CF911F910F91FF90DE
:10683000EF90DF90CF9008951F93CF93DF93EC01FB
:106840008B81823018F480E090E023C04885598520
:106850006A857B85A5E07695679557954795AA95B6
:10686000D1F7142F1F70CE014FDF97FDECCF488575
:1068700059856A857B85415E5F4F6F4F7F4F4887A3
:1068800059876A877B8720E2129FC00111248952B1
:10689000914FDF91CF911F9108954F925F926F9228
:1068A0007F92AF92BF92CF92DF92EF92FF920F93BF
:1068B0001F93CF93DF93EC016A017B012B8122238D
:1068C00049F089899A89AB89BC8984179507A607FD
:1068D000B70710F480E06BC0223009F463C0C11424
:1068E000D104E104F10449F41C821D821E821F823E
:1068F000188619861A861B8659C088859985AA85A7
:10690000BB85E98DFA8DE585F0E03996AC01BD01D6
:1069100041505109610971090E2E04C076956795A1
:10692000579547950A94D2F79701860101501109AE
:106930002109310904C03695279517950795EA95E1
:10694000D2F7041715072607370720F0892B8A2B63
:106950008B2B49F48D899E89AF89B88D8C839D835B
:10696000AE83BF8304C0041B150B260B370B280115
:1069700039015E0184E0A80EB11C41145104610488
:10698000710481F04C815D816E817F819501898DDB
:106990009A8D60D591E0491A5108610871088111FA
:1069A000ECCF05C0C886D986EA86FB8681E0DF91F8
:1069B000CF911F910F91FF90EF90DF90CF90BF90FC
:1069C000AF907F906F905F904F9008950F931F93BB
:1069D000CF93DF93EC018B818823D1F1898187FFED
:1069E00032C061E0CE01B6DC8C01009789F1FC0178
:1069F0008081853E69F18B81823040F449895A89D2
:106A00006B897C89448F558F668F778F4D895E891E
:106A10006F89788DF801538F428F758B648BE0916D
:106A2000CE0EF091CF0E309759F0B8016A5E7F4FCD
:106A3000C80148961995F801808D918D938B828BB2
:106A400089818F778983DF91CF911F910F918AC4BC
:106A500081E0888380E0DF91CF911F910F910895AD
:106A6000CF93DF93EC01B2DF1B82DF91CF910895CA
:106A7000FC0123812111F4CF08954F925F926F9210
:106A80007F92AF92BF92CF92DF92EF92FF920F93DD
:106A90001F93CF93DF9300D01F92CDB7DEB75C0179
:106AA0006A017B01FC0183818130E9F4818181FFEE
:106AB0001AC0F50181899289A389B4898417950741
:106AC000A607B70780F0892B8A2B8B2B09F472C09D
:106AD000F5014084518462847384B701A601C50125
:106AE000DCDE811102C080E066C0F501818D928DEF
:106AF000C114D104E104F10469F445895689678918
:106B0000708D25D7882379F3F501158A168A178A9F
:106B1000108E37C0F50144815581668177819E01D1
:106B20002F5F3F4F97D48823F1F249815A816B81BF
:106B30007C81F501818D928DFC012789203139F40A
:106B4000483FFFEF5F0761057105D8F407C0483F74
:106B50002FEF520762072FE0720798F4F8D68823C8
:106B600009F4C1CFF50144815581668177810FEF2A
:106B70001FEF2FEF3FE0818D928D51D5882309F4CF
:106B8000B2CFF501C18AD28AE38AF48A8181806812
:106B90008183C5011BDF882309F4A5CFB701A601B6
:106BA0004C145D046E047F0410F4B301A201C5010E
:106BB00074DE01C081E00F900F900F900F90DF9175
:106BC000CF911F910F91FF90EF90DF90CF90BF90EA
:106BD000AF907F906F905F904F900895FF920F93CA
:106BE0001F93CF93DF93EC01F42E80E2689FF001B6
:106BF0001124E952F14F8385817121F0842F827134
:106C000009F04EC08091D7109091D810A091D91062
:106C1000B091DA108C879D87AE87BF87688B4489D7
:106C2000558960E070E0BA0155274427028D138D25
:106C300020E030E0402B512B622B732B4D8B5E8B71
:106C40006F8B788F8385887151F4048D158D268D17
:106C5000378D098B1A8B2B8B3C8B81E00BC08031DD
:106C6000F9F49E012F5E3F4F898D9A8D72D488234F
:106C7000B9F084E08B838F2D8F7089831C821D82F5
:106C80001E821F82188619861A861B86F4FE0BC088
:106C900040E050E0BA01CE01F0DE811104C011C025
:106CA0001B8280E00EC0F5FE0BC049895A896B89B2
:106CB0007C89CE01DF91CF911F910F91FF90EDCD97
:106CC00081E0DF91CF911F910F91FF900895AF92D6
:106CD000BF92CF92DF92EF92FF920F931F93CF93C9
:106CE000DF937C01EB016A01B22E898D9A8DF70149
:106CF000928F818F40E050E0BA01CE01CEDDA12C11
:106D0000088519852A853B8589899A89AB89BC893B
:106D1000081719072A073B07A0F585E03695279540
:106D2000179507958A95D1F70F70CE0185DD0097ED
:106D300009F481C0FC012081222311F0253EB9F421
:106D4000A1100EC04091D7105091D8106091D91069
:106D50007091DA10F7014487558766877787008B33
:106D6000FC018081AA24A3948111CACF0AC04BE000
:106D700050E0BC01C6010F94D70E892B09F0C0CF9B
:106D800058C08B2D8274823409F055C0AA2049F076
:106D9000F701008961E0C701DDDAEC01009769F4D1
:106DA0004AC08B81823009F446C0CE014BDA882379
:106DB00009F441C0C7EDDEE000E080E2FE0111927F
:106DC0008A95E9F78BE0F601DE0101900D928A9534
:106DD000E1F7E091CE0EF091CF0E309739F0BE0181
:106DE000625F7F4FCE014096199508C081E298E21C
:106DF000998B888B80E098E09F878E878889998916
:106E00009B8B8A8B998F888F8E859F859F8B8E8B8E
:106E1000A9D2882381F04B2D602FC701DF91CF913C
:106E20001F910F91FF90EF90DF90CF90BF90AF90A8
:106E3000D5CEB7FEF0CF80E0DF91CF911F910F91BB
:106E4000FF90EF90DF90CF90BF90AF9008953F926A
:106E50004F925F926F927F928F929F92AF92BF926A
:106E6000CF92DF92EF92FF920F931F93CF93DF9316
:106E7000CDB7DEB7C354D1090FB6F894DEBF0FBE4D
:106E8000CDBF5C016B0124965FAF4EAF2497522EAD
:106E90001C8E1F8E19821C826115710511F410E081
:106EA00073C0FC0183818111FACF2496EEADFFAD52
:106EB000249780818F3211F076011DC02496EEADAB
:106EC000FFAD249780818F3231F431962496FFAF45
:106ED000EEAF2497F3CFF60183818250823060F3C6
:106EE000F601618D728DCE010196C7DA8823B9F261
:106EF000CE0101967C018E01045E1F4F3801FE0118
:106F000031964F01402E312E19C08823A9F121E07E
:106F1000AE01495C5F4FB701C801D9DE882309F48F
:106F2000BECFEC14FD0411F0C7019ADD061517055C
:106F300001F1942D832D7801092F182FAE014E5B9E
:106F40005F4FBE01695C7F4F24968EAD9FAD249745
:106F500055DA882309F4A3CF2496EEADFFAD24972C
:106F600080818F3291F631962496FFAFEEAF249751
:106F7000F3CF982D892DDFCF252DAE01495C5F4FD2
:106F8000B701C501A4DE182FCE01019671DDCE0137
:106F90004C966EDD812FCD5BDF4F0FB6F894DEBFD0
:106FA0000FBECDBFDF91CF911F910F91FF90EF905A
:106FB000DF90CF90BF90AF909F908F907F906F9019
:106FC0005F904F903F900895CF93DF93EC0140E0A6
:106FD00050E0BA0152DD882361F061E0CE01BAD9F8
:106FE000009739F025EEFC0120831B82DF91CF91C1
:106FF000B9C180E0DF91CF9108951F93CF93DF93C4
:10700000CDB7DEB76B970FB6F894DEBF0FBECDBF1E
:10701000AB0119821C8222E0BC01CE01019617DF70
:10702000182F882321F0CE010196CEDF182FCE0134
:1070300001961EDD812F6B960FB6F894DEBF0FBE52
:10704000CDBFDF91CF911F9108952F923F924F9224
:107050005F926F927F928F929F92AF92BF92CF92E8
:10706000DF92EF92FF920F931F93CF93DF9300D0A5
:107070001F921F92CDB7DEB78C015B013A01DC0194
:1070800013968C9113978130C1F411968C9181FFE6
:1070900014C082FF18C0F80141895289638974893C
:1070A00080859185A285B38584179507A607B707C4
:1070B00051F0C801F2DB811106C081E0F801808344
:1070C0008FEF9FEF37C1630183C0D80159968D912F
:1070D0009C915A97FC01F481F1501A012B0169E04F
:1070E00056944794379427946A95D1F7F221FD83FB
:1070F0004A0121E09222FF2309F476C080E092E069
:107100008819990976018C159D0508F47C01D80130
:107110005996ED91FC915A9714962D903D904D9073
:107120005C901797B2E02B1A31084108510805848A
:1071300004C0220C331C441C551C0A94D2F78685CB
:107140009785A089B189280E391E4A1E5B1EED81E4
:107150002E0E311C411C511CE114F2E0FF0609F017
:1071600089C08091D7109091D810A091D910B0917A
:10717000DA1082159305A405B50569F41092D40EB2
:107180008FEF9FEFDC018093D7109093D810A093DE
:10719000D910B093DA109501B201A1018091D50EFA
:1071A0009091D60E0E949662882309F486CFF8014A
:1071B00080859185A285B3858E0D9F1DA11DB11D72
:1071C00080879187A287B387AE0CBF1CCE18DF08DB
:1071D000D80118964D915D916D917C911B97C114CA
:1071E000D10409F072CF7AC08114910409F086CFDE
:1071F00014964D915D916D917C91179741155105B4
:107200006105710559F455968D919D910D90BC9134
:10721000A02D0097A105B10539F520C09E012F5F73
:107220003F4F18D1882309F448CF89819A81AB81D7
:10723000BC81F801218D328DF9012789203139F483
:10724000883FFFEF9F07A105B10540F40DC0883FBF
:107250002FEF9207A2072FE0B20730F0C8010E947B
:10726000FC3081114BCF29CFF80184839583A6830D
:10727000B78344CF8114910411F5D80118964D912C
:107280005D916D917C911B9751968D919D910D9083
:10729000BC91A02D481759076A077B0780F062D080
:1072A000882309F40ACF81E08093D40E2092D7106E
:1072B0003092D8104092D9105092DA1007C041E0B5
:1072C000C201B1018FD0882309F4F7CEA701B5011F
:1072D000C4018952914F0F94E40E69CF51968D915C
:1072E0009D910D90BC91A02DF801218184179507E7
:1072F000A607B70738F4418B528B638B748B2068D9
:1073000021830CC08091CE0E9091CF0E892B31F04D
:107310006114710419F02068F8012183D8011196D5
:107320008C9183FD02C0C30105C0C8014FDB8111F0
:10733000FACFC3CE0F900F900F900F900F90DF9168
:10734000CF911F910F91FF90EF90DF90CF90BF9062
:10735000AF909F908F907F906F905F904F903F90F5
:107360002F900895CF938091D40E8823B9F1409146
:10737000D7105091D8106091D9107091DA1027ED84
:107380003EE08091D50E9091D60E0E949662C82F55
:10739000811102C0C0E023C04091D00E5091D10EA7
:1073A0006091D20E7091D30E4115510561057105A2
:1073B00091F027ED3EE08091D50E9091D60E0E947F
:1073C0009662882339F31092D00E1092D10E10924B
:1073D000D20E1092D30E1092D40E01C0C1E08C2FA9
:1073E000CF910895CF92DF92EF92FF92CF936B01EE
:1073F0007C01C42F8091D7109091D810A091D91002
:10740000B091DA108C159D05AE05BF05C9F0AADF55
:10741000811102C080E018C027ED3EE0B701A6014F
:107420008091D50E9091D60E0E942162882391F30F
:10743000C092D710D092D810E092D910F092DA1002
:1074400081E0C1118093D40ECF91FF90EF90DF9037
:10745000CF9008958F929F92AF92BF92CF92DF927A
:10746000EF92FF920F931F93CF93DF93EC016A018A
:107470007B01890189859A85AB85BC850196A11D13
:10748000B11D84179507A607B70710F480E054C014
:107490008F89803129F49927872F762F652F0BC08C
:1074A0008032A1F7CB01BA0127E0969587957795B1
:1074B00067952A95D1F78B889C88AD88BE88680D22
:1074C000791D8A1D9B1D8090D7109090D810A09098
:1074D000D910B090DA10681579058A059B0581F4FA
:1074E0008F89803191F4DD24EE24FF24F601EE0F24
:1074F000FF1FE952F14F80819181A0E0B0E016C0FA
:1075000040E070DF8111ECCFC1CFE894C7F8DD24F3
:10751000EE24FF24F601EE0FFF1FEE0FFF1FE952CE
:10752000F14F80819181A281B381BF70F801808386
:107530009183A283B38381E0DF91CF911F910F915B
:10754000FF90EF90DF90CF90BF90AF909F908F9083
:1075500008954F925F926F927F92AF92BF92CF92B7
:10756000DF92EF92FF920F931F93CF93DF9300D0A0
:107570001F92CDB7DEB78C0149835A836B837C831E
:107580005901C12CD12C7601412C42E0542E612CA2
:10759000712C49815A816B817C819E012F5F3F4F05
:1075A000C80158DF882341F1D301C201F8010584E5
:1075B00004C0880F991FAA1FBB1F0A94D2F7C80ED8
:1075C000D91EEA1EFB1E49815A816B817C81878905
:1075D000803139F481E0483F5F4F6105710538F42F
:1075E000D8CF81E0483F5F4F6F4F7F4090F2F50169
:1075F000C082D182E282F3820F900F900F900F90A1
:10760000DF91CF911F910F91FF90EF90DF90CF907E
:10761000BF90AF907F906F905F904F9008954F9282
:107620005F926F927F928F929F92AF92BF92CF9212
:10763000DF92EF92FF920F931F93CF93DF93EC01B2
:107640004A015B012801390142305105610571058C
:1076500008F462C049855A856B857C854F5F5F4F12
:107660006F4F7F4F481559056A057B0508F454C0D4
:107670008F89803129F4FF24EB2CDA2CC92C0CC023
:10768000803209F049C07501640177E0F694E7940F
:10769000D794C7947A95D1F74B895C896D897E8997
:1076A000C40ED51EE61EF71E41E0C701B6019ADEE4
:1076B000882391F19F89903159F49924AA24BB24FD
:1076C000F401EE0FFF1FE952F14F5182408210C0CA
:1076D000E89487F89924AA24BB24F401EE0FFF1F35
:1076E000EE0FFF1FE952F14F408251826282738296
:1076F0009A89923090F04D815E816F8178854C0D32
:107700005D1D6E1D7F1D4093D00E5093D10E609372
:10771000D20E7093D30E01C080E0DF91CF911F9104
:107720000F91FF90EF90DF90CF90BF90AF909F9020
:107730008F907F906F905F904F9008952F923F921F
:107740004F925F926F927F928F929F92AF92BF9271
:10775000CF92DF92EF92FF920F931F93CF93DF931D
:10776000CDB7DEB72F970FB6F894DEBF0FBECDBFF3
:107770001C014C875D876E877F873B872A87DC01EA
:1077800019960D911D912D913C911C970F5F1F4FE4
:107790002F4F3F4F0D831E832F833887EA85FB854C
:1077A00080809180A280B38081149104A104B104EF
:1077B00031F0FFEF8F1A9F0AAF0ABF0A10C0DC0139
:1077C0008D909D90AD90BC90B1E0B9870C851D85E2
:1077D0002E853F85013011052105310509F01986F7
:1077E00075016401412C512C3201F1018185928592
:1077F000A385B485481659066A067B0608F04EC074
:107800000D811E812F8138850C151D052E053F0524
:1078100050F4F2E0CF2ED12CE12CF12CA2E08A2EF4
:10782000912CA12CB12C9E012F5F3F4FB701A601D7
:10783000C10110DE882391F149815A816B817C81DD
:10784000D701C6010196A11DB11D452B462B472B23
:1078500019F04C015D010FC0AC01BD014819590977
:107860006A097B090C851D852E853F8540175107C8
:107870006207730741F01FEF411A510A610A710A4A
:107880006C017D01B2CF0FEF1FEF2FEF3FE0B7018B
:10789000A601C101C4DE8D83811113C01D823DC0CC
:1078A0002601370121E0421A510861087108970149
:1078B0008601B301A201C101B2DE882379F373010D
:1078C00062018C149D04AE04BF0450F3AA85BB85ED
:1078D0004D915D916D917C91411551056105710549
:1078E000A9F4EA85FB8580829182A282B382F98520
:1078F000FF2399F00FEF801A900AA00AB00AD10175
:107900008D929D92AD92BC92139707C09501840110
:10791000C10185DE8111E5CFC1CF8D812F960FB6D4
:10792000F894DEBF0FBECDBFDF91CF911F910F91B5
:10793000FF90EF90DF90CF90BF90AF909F908F908F
:107940007F906F905F904F903F902F900895AF92EF
:10795000BF92CF92DF92EF92FF920F931F93CF933C
:10796000DF9300D01F92CDB7DEB75C016A017B01C7
:1079700082E090E0A0E0B0E0F50180839183A283F3
:10798000B3839E012F5F3F4FB701A601C50162DDA2
:10799000811102C080E023C000E010E09801B7012F
:1079A000A601C5013CDE8823A9F3C980DA80EB80FB
:1079B000FC80F5018789803149F481E0F8EFCF162A
:1079C000FFEFDF06E104F10450F4DBCF81E098EF34
:1079D000C9169FEFD906E9069FE0F90690F20F90CD
:1079E0000F900F900F90DF91CF911F910F91FF900B
:1079F000EF90DF90CF90BF90AF9008957F928F92DD
:107A00009F92AF92BF92CF92DF92EF92FF920F932D
:107A10001F93CF93DF93EC01142F7093D60E6093D6
:107A2000D50E1F8A82E090E0A0E0B0E088839983C1
:107A3000AA83BB831092D40E1092D00E1092D10E56
:107A40001092D20E1092D30E8FEF9FEFDC01809335
:107A5000D7109093D810A093D910B093DA10442384
:107A600049F1453008F0DEC040E060E070E0CB0155
:107A7000B9DC882309F4D6C020E1129FF00111245B
:107A8000EB57FF4E80818F7709F0CCC084859585B8
:107A9000A685B78584369105A105B10508F4C2C055
:107AA000C084D184E284F384C114D104E104F104DC
:107AB00021F4B8C0C12CD12C760140E0C701B60139
:107AC00091DC782E882309F4ADC08091E20E90916C
:107AD000E30E8115924009F0A5C03091E70E3323E3
:107AE00009F4A0C08091E50E9091E60E892B09F46F
:107AF00099C02091E40E222309F494C03A8B2C8380
:107B00001D8630E041E050E06D85062FCA01062E4B
:107B100002C0880F991F0A94E2F72817390731F03D
:107B200081E0860F8D87683078F37CC02091ED0E60
:107B30003091EE0E2115310519F040E050E008C0FB
:107B40002091FB0E3091FC0E4091FD0E5091FE0EE7
:107B50002D833E834F8358878091E50E9091E60EEA
:107B600046015701880E991EA11CB11C8B8A9C8A64
:107B7000AD8ABE8AE091E80EF091E90EF98FE88FA8
:107B8000A091E70EB0E00F94A309680D791D8A1D3E
:107B90009B1D6A8F7B8F8C8F9D8FB5E0EE0FFF1F33
:107BA000BA95E1F7E150FE4FEF2FFF27E695DC0194
:107BB000CB018E0F9F1FA11DB11D8E879F87A88BA4
:107BC000B98B8090EA0E9090EB0E8114910419F01D
:107BD000A12CB12C08C08090F70E9090F80EA090C8
:107BE000F90EB090FA0EA7019601281B390B4A0B2B
:107BF0005B0BDA01C901880D991DAA1DBB1D04C0CC
:107C0000B695A795979587950A95D2F789879A870C
:107C1000AB87BC87853F3FE09307A105B10520F402
:107C20008CE08F8B712C15C0853F9F4FA105B1054E
:107C300010F480E10DC08091030F9091040FA0918A
:107C4000050FB091060F8A8F9B8FAC8FBD8F80E29E
:107C50008F8B872DDF91CF911F910F91FF90EF9028
:107C6000DF90CF90BF90AF909F908F907F900895BE
:107C70004F925F926F927F928F929F92AF92BF923C
:107C8000CF92DF92EF92FF920F931F93CF93DF93E8
:107C90002C0127E034E081E090E0F9014591549116
:107CA000441655060CF062C0AC0141505109DA018E
:107CB000AA0FBB1FAA0FBB1FAB5FBB4FFD01659196
:107CC0007491440F551F440F551F4D5F5B4FFA01D0
:107CD00065907490FC01EE0FFF1FEE0FFF1FEB5F2E
:107CE000FB4FA590B490FD0105911491F901C59148
:107CF000D491FA0185909490882777FD8095982FEC
:107D00000F941D066B017C01B20166197709882763
:107D100077FD8095982F0F941D062B013C01B5012E
:107D2000601B710B882777FD8095982F0F941D0697
:107D30009B01AC01C301B2010F9450082B013C011F
:107D4000BE0168197909882777FD8095982F0F94CF
:107D50001D069B01AC01C301B2010F9482059B017A
:107D6000AC01C701B6010F94A20411C001962C5FAB
:107D70003F4F8D33910509F090CFE5EFF4E0659129
:107D80007491882777FD8095982F0F941D066B01BD
:107D90007C0120E030E040E252E4C701B6010F94DC
:107DA0007E0787FD1BC020E030E048E452E4C701B5
:107DB000B6010F947B0518168CF020E030E040E20D
:107DC00052E4C701B6010F94A10420E030E040E086
:107DD0005FE30F9450089B01AC013FC020E030E00E
:107DE00048E452E4C701B6010F947E0718163CF52B
:107DF00020E030E048EC52E4C701B6010F947B0567
:107E00001816ECF020E030E040EA50E4C701B6017B
:107E10000F94A2044B015C0120E030E048E452E4FE
:107E2000C701B6010F94A1042DEC3CEC4CEC5DE3D2
:107E30000F9450089B01AC01C501B40110C020E0B3
:107E400030E048EC52E4C701B6010F947E071816E3
:107E500054F420E030E040E251E4C701B6010F9451
:107E6000A2046B017C01C701B601DF91CF911F9184
:107E70000F91FF90EF90DF90CF90BF90AF909F90C9
:107E80008F907F906F905F904F9008954F925F9288
:107E90006F927F928F929F92AF92BF92CF92DF921A
:107EA000EF92FF920F931F93CF93DF932C016623E2
:107EB00071F1E5E5F3E58491882341F09091C000EC
:107EC00095FFFCCF8093C6003196F5CF70E04AE075
:107ED00050E08BE397E10E94C1DAECE6F2E0849196
:107EE000882341F09091C00095FFFCCF8093C6009D
:107EF0003196F5CF8091C00085FFFCCF8AE080935A
:107F0000C6000E94736F60E070E0CB017EC027E87E
:107F100033E081E090E0F901459154914416550613
:107F20000CF062C0AC0141505109DA01AA0FBB1F2D
:107F3000AA0FBB1FAB57BC4FFD0165917491440F55
:107F4000551F440F551F4D575C4FFA0165907490B3
:107F5000FC01EE0FFF1FEE0FFF1FEB57FC4FA5902C
:107F6000B490FD0105911491F901C591D491FA01E4
:107F700085909490882777FD8095982F0F941D0603
:107F80006B017C01B20166197709882777FD80951E
:107F9000982F0F941D062B013C01B501601B710B3E
:107FA000882777FD8095982F0F941D069B01AC01C3
:107FB000C301B2010F9450082B013C01BE016819A6
:107FC0007909882777FD8095982F0F941D069B01CE
:107FD000AC01C301B2010F9482059B01AC01C70142
:107FE000B6010F94A20411C001962C5F3F4F80325E
:107FF000910509F090CFE1E0F4E065917491882754
:1080000077FD8095982F0F941D06DF91CF911F91DA
:108010000F91FF90EF90DF90CF90BF90AF909F9027
:108020008F907F906F905F904F90089560E0809167
:108030004C1190914D112ADF6093481170934911B2
:1080400080934A1190934B11809146119091471162
:108050000FDE60934211709343118093441190930B
:1080600045118FB7F89410923A118FBF089520915F
:10807000200230912102409122025091230260E0BF
:1080800070E08FE793E40F94820560931A11709368
:108090001B1180931C1190931D112091100230919F
:1080A0001102409112025091130260E070E08FE7DC
:1080B00093E40F9482056093F9107093FA10809303
:1080C000FB109093FC10089597FF03C0809141111D
:1080D00004C0FC01E850FF4E808190E00895CF93EA
:1080E000DF93D82FC62FC19561E00E94E8FD6C2F69
:1080F0008D2F0E9421FE6C2F70E08D2FDF91CF918C
:108100000C94DEFCCF93C1E020E030E048E452E480
:10811000609148117091491180914A1190914B11D1
:108120000F947E0718160CF0C0E06C2F88E090E0EA
:10813000CF91D5CFCF93DF9310921E1110921F11C4
:1081400010922011109221112091200230912102D1
:10815000409122025091230260E070E08FE793E4A7
:108160000F94820560931A1170931B1180931C1158
:1081700090931D111092FD101092FE101092FF109E
:1081800010920011209110023091110240911202C0
:108190005091130260E070E08FE793E40F94820542
:1081A0006093F9107093FA108093FB109093FC1079
:1081B0006D9A809101018061809301019D9A809167
:1081C000010188608093010187ED80937A0010920D
:1081D0007E0010927D0080917E00816080937E0001
:1081E00080917E00826080937E0080917E0084601A
:1081F00080937E0080E888BD80916E0084608093CB
:108200006E006AEF70E080E090E00E94F7FE8FE081
:1082100090E09093F1108093F01060E080910A025A
:1082200090910B0233DE20E030E040E751E40F9400
:108230007B0587FF0AC080910A0290910B0240974C
:1082400090930B0280930A02E8CF81E391E0909330
:1082500009028093080260E08091F2109091F3107F
:1082600015DE20E030E848E953E40F947E07181645
:1082700054F48091F2109091F31040969093F31083
:108280008093F210E8CFC091EE10D091EF10CE01A4
:10829000EFDC20E030E046E153E40F947E0718164F
:1082A00034F46096D093EF10C093EE10ECCFDF91D2
:1082B000CF9108950895109251111092501110927B
:1082C0004F1110924E111092F810759810924F1194
:1082D00010924E1110924111A59808952F923F923D
:1082E0004F925F926F927F928F929F92AF92BF92C6
:1082F000CF92DF92EF92FF920F931F93CF93DF9372
:10830000CDB7DEB7AE970FB6F894DEBF0FBECDBFC8
:108310006B8F7C8F8D8F292E5A8749873CA72BA77F
:108320000E94C8FE6F8F78A389A39AA30E94C8FEFB
:108330006FA378A789A79AA729853A8512161306ED
:108340001CF0ECE1FDE017C0EFE2FDE08191882335
:1083500039F09091C00095FFFCCF8093C600F6CF16
:108360008091C00085FFFCCF1BC29091C00095FF9B
:10837000FCCF8093C60081918111F7CF8091C0001E
:1083800085FFFCCF8AE08093C60095DF49855A853A
:108390008FE7452B99F1809341118F8D98A1A9A169
:1083A000BAA1898B9A8BAB8BBC8B8D879E87AF874D
:1083B000B88B1D8290E4988FACE1A98FB6E4BA8F98
:1083C0001DA61D8A1E8A1F8A2FE730E040E050E07C
:1083D00029833A834B835C83EFE74E2E512C612C2B
:1083E000712C1BA21CA21DA21EA231E03E8F1C8676
:1083F0001B86312C00E010E01EA605C08093F8100B
:10840000CCCF0E9404AE80913A11882309F4F6C0C3
:108410000DDE49855A85452B51F03090421100916F
:10842000431110914411509145115EA709C030903D
:1084300048110091491110914A1180914B118EA75A
:10844000232D302F412F5EA56DA57D898E899F89B3
:108450000F947E0718162CF03DA60D8B1E8B9EA543
:108460009F8B232D302F412F5EA56D81788D898DB7
:108470009A8D0F947B0587FD05C03D82088F198F6B
:10848000AEA5AA8F0E94C8FE2FA138A549A55AA55E
:10849000621B730B840B950B653C7940810591053C
:1084A00038F030DE0E94C8FE6FA378A789A79AA78C
:1084B0004E8D442309F44FC02B8D3C8D4D8D522D94
:1084C000632D702F812F9EA50F947E0718160CF038
:1084D00095C00E94C8FE29893A894B895C89621B34
:1084E000730B840B950B693873418105910508F472
:1084F00085C0D301C20129813A814B815C81821BF5
:10850000930BA40BB50B49855A85B595A7959795FF
:108510008795452B19F08093411102C08093F81084
:108520000E94C8FE6D877E878F87988BDC01CB0108
:1085300029893A894B895C89821B930BA40BB50B63
:108540008BA39CA3ADA3BEA33B8D3DA74C8D4D8BB0
:108550005D8D5E8B2F8A2B8D3C8D4D8D522D632D25
:10856000702F812F9EA50F947B0587FFEEC20E947E
:10857000C8FE2D853E854F855889621B730B840B81
:10858000950B693873418105910508F4DEC20E949C
:10859000C8FE698B7A8B8B8B9C8BDC01CB012D8584
:1085A0003E854F855889821B930BA40BB50B4B85D9
:1085B0005C85452B09F010C189819A81AB81BC8112
:1085C000840D951DA61DB71D29853A85B595A795DE
:1085D00097958795232B09F4B5C2809341114B855C
:1085E0005C854F5F5F4F5C874B875B8D5D838C8DB8
:1085F000888F9D8D998F2A8EA1E0AE8F20E030E08C
:1086000040EA51E46B8D7C8D8D8D922D0F94A204E8
:108610009B01AC01632D702F812F9EA50F947E07C7
:10862000181694F4E2E1F3E08491882341F09091EC
:10863000C00095FFFCCF8093C6003196F5CF8091A6
:10864000C00085FFFCCFACC00E94C8FE2F8D38A1B2
:1086500049A15AA1621B730B840B950B613D7740B6
:108660008105910508F44FC049855A85452B81F055
:10867000E0904111F12CECE0F3E084918823C1F00B
:108680009091C00095FFFCCF8093C6003196F5CF46
:10869000E090F810F12CE6E0F3E08491882341F0BB
:1086A0009091C00095FFFCCF8093C6003196F5CF26
:1086B00022E030E0432D502F612F7EA58BE397E120
:1086C0000E9497DBE2E0F3E08491882341F09091EF
:1086D000C00095FFFCCF8093C6003196F5CF4AE0ED
:1086E00050E0B7018BE397E10E94C1DA8091C000AE
:1086F00085FFFCCF8AE08093C6000E94C8FE6F8F82
:1087000078A389A39AA30E94C8FE6B017C010E94F2
:10871000C8FE89889A88AB88BC882D853E854F85A0
:108720005889820E931EA41EB51EC818D908EA08DF
:10873000FB08C60ED71EE81EF91E31E8C3163FE43B
:10874000D30632E1E306F10490F0E5EEF2E0849125
:10875000882341F09091C00095FFFCCF8093C60024
:108760003196F5CF8091C00085FFFCCF19C04B85B5
:108770005C858BA59CA5841795070CF042CEE9E893
:10878000F2E08491882341F09091C00095FFFCCFE6
:108790008093C6003196F5CF8091C00085FFFCCF55
:1087A0008AE08093C600AE960FB6F894DEBF0FBE87
:1087B000CDBFDF91CF911F910F91FF90EF90DF9090
:1087C000CF90BF90AF909F908F907F906F905F9071
:1087D0004F903F902F9008958BA09CA0ADA0BEA07D
:1087E000880E991EAA1EBB1E2BA13CA14DA15EA105
:1087F000281B390B4A0B5B0BCA01B90129813A814D
:108800004B815C810F941609A50194010F947B099B
:10881000240D351D461D571D2431310541055105D7
:1088200004F129013A013CEE43165104610471043C
:108830002CF06BEE462E512C612C712C40E8441626
:10884000510461047104DCF08EEF90E0A0E0B0E030
:1088500084199509A609B70989839A83AB83BC83D8
:1088600012C054E1452E512C612C712C24E130E0D2
:1088700040E050E029833A834B835C8304C0498203
:108880005A826B827C82EBE7F3E08491882341F08B
:108890009091C00095FFFCCF8093C6003196F5CF34
:1088A0002AE030E0B301A2018BE397E10E9496DA5F
:1088B000E6E7F3E08491882341F09091C00095FFB2
:1088C000FCCF8093C6003196F5CF2AE030E0498195
:1088D0005A816B817C818BE397E10E9496DAEFE607
:1088E000F3E08491882341F09091C00095FFFCCF84
:1088F0008093C6003196F5CF22E030E04D81588D4F
:10890000698D7A8D8BE397E10E9497DBE8E6F3E0CF
:108910008491882341F09091C00095FFFCCF809313
:10892000C6003196F5CF22E030E04DA55D896E8915
:108930007F898BE397E10E9497DB8091C00085FFE0
:10894000FCCF8AE08093C6002B853C85233031051F
:108950000CF432CE69817A818B819C810F941D0643
:1089600020E030E040E850E40F9450086B017C01B7
:108970002D81388D498D5A8D6DA57D898E899F8970
:108980000F94A10420ED3FE049E450E40F94500817
:1089900020E030E040E05FE30F9450089B01AC0121
:1089A000C701B6010F9482056B017C01C501B401BA
:1089B0000F941D0620E030E04AE754E40F9482054E
:1089C0004B015C01E2E6F3E08491882341F0909151
:1089D000C00095FFFCCF8093C6003196F5CF22E012
:1089E00030E0B701A6018BE397E10E9497DBECE54D
:1089F000F3E08491882341F09091C00095FFFCCF73
:108A00008093C6003196F5CF22E030E0B501A40195
:108A10008BE397E10E9497DB8091C00085FFFCCF3C
:108A20008AE08093C6002AE939E949E15FE3C7019A
:108A3000B6010F9450086B017C019B01AC010F94AF
:108A4000A204A50194010F9482056D837E838F8318
:108A50009887A5019401C701B6010F94500820E042
:108A600030E040E05EE30F9450084B015C01EEE41F
:108A7000F3E08491882341F09091C00095FFFCCFF2
:108A80008093C6003196F5CF8091C00085FFFCCF62
:108A90008AE08093C600E8E4F3E08491882341F003
:108AA0009091C00095FFFCCF8093C6003196F5CF22
:108AB00022E030E0B701A6018BE397E10E9497DB4B
:108AC0008091C00085FFFCCF8AE08093C600E2E47D
:108AD000F3E08491882341F09091C00095FFFCCF92
:108AE0008093C6003196F5CF22E030E04D815E8163
:108AF0006F8178858BE397E10E9497DB8091C000BE
:108B000085FFFCCF8AE08093C600ECE3F3E084911C
:108B1000882341F09091C00095FFFCCF8093C60060
:108B20003196F5CF22E030E0B501A4018BE397E167
:108B30000E9497DB8091C00085FFFCCF8AE0809384
:108B4000C6003ACD8093F8104ACD1E8E57CD81E0F5
:108B5000809378130E949BE48091D013882339F08E
:108B60001092D01360E08EEC93E10E94C35A8CE522
:108B700092E00E9462AD9FDB179A10928E13169AB4
:108B800010928F13149A56D10E9404AE9FB7F89496
:108B9000809102018460809302019FBF84EF91E085
:108BA0000E941BFF9FB7F894809102018B7F8093F6
:108BB00002019FBF84E690E00C941BFF2F923F922E
:108BC0004F925F926F927F928F929F92AF92BF92DD
:108BD000CF92DF92EF92FF920F931F93CF93DF9389
:108BE000CDB7DEB728970FB6F894DEBF0FBECDBF66
:108BF0004C012A013B010D831E832F833887AA2055
:108C000039F0A12CB12C19821A821B821C820BC054
:108C10003DE2A32EB12C80E090E0A0E7B1E489838F
:108C20009A83AB83BC830E94C8FE0F941B06840109
:108C3000000F111F000F111FD801A65ABE4E1D01B3
:108C40002D913D914D915C910F94A10420E030E075
:108C50004AEF54E40F947E0718160CF0D2C00E941D
:108C6000C8FE0F941B06F101608371838283938396
:108C700020E030E0A901C701B6010F947B05811106
:108C800007C0F401EE0FFF1FEE5AFE4E1182108254
:108C9000980126593E4E1901A3019201D1016D910F
:108CA0007D918D919C910F947B05882321F120E08B
:108CB00030E0A901C301B2010F947E07F801E65824
:108CC000FE4E181674F480E090E0A0E8BFE38083C5
:108CD0009183A283B383F1014082518262827382C5
:108CE0000AC01082118212821382D1014D925D92CC
:108CF0006D927C921397A30192016D817E818F8189
:108D000098850F947E0787FD19C0F801E658FE4E3E
:108D10001F0120E030E040E85FE3608171818281E3
:108D200093810F947B05811109C080E090E0A0E061
:108D3000B0E4F10180839183A283B38320E030E02B
:108D4000A901C701B6010F947E0718160CF059C08F
:108D500029813A814B815C81C301B2010F94A10446
:108D60002D813E814F8158850F947B0587FF12C06E
:108D700029813A814B815C81C301B2010F94A20425
:108D80009B01AC016D817E818F8198850F947B055D
:108D900087FD37C0F801E658FE4E20E030E040E89D
:108DA0005FE360817181828193810F947E07181641
:108DB00044F5F401EE0FFF1FEE5AFE4E80819181C3
:108DC000019691838083880F991FA816B906CCF469
:108DD00028960FB6F894DEBF0FBECDBFDF91CF91BE
:108DE0001F910F91FF90EF90DF90CF90BF90AF90C9
:108DF0009F908F907F906F905F904F903F902F90BB
:108E0000A6CE28960FB6F894DEBF0FBECDBFDF9179
:108E1000CF911F910F91FF90EF90DF90CF90BF9077
:108E2000AF909F908F907F906F905F904F903F900A
:108E30002F9008952F923F924F925F926F927F9260
:108E40008F929F92AF92BF92CF92DF92EF92FF925A
:108E50000F931F93CF93DF93CDB7DEB728970FB64D
:108E6000F894DEBF0FBECDBF80913A11882309F47C
:108E70000AC3DCD86091F81070E080E090E00F94B5
:108E80001D066B017C014090481150904911609083
:108E90004A1170904B1160915011709151118827B7
:108EA00077FD8095982F0F941D06AB01BC01A12C76
:108EB0009301820181E090E081DE809048119090E2
:108EC0004911A0904A11B0904B110091501110918E
:108ED0005111B801882777FD8095982F0F941D06B2
:108EE000A50194010F94A1046B017C0160932211F0
:108EF00070932311809324119093251120E030E08A
:108F000040E251E40F947E07181624F481E0809328
:108F10001911F7C020E030E040E251ECC701B60182
:108F20000F947B0587FD02C0012B21F481E0809323
:108F300019110CC180911911882351F0109236112A
:108F40001092371110923811109239111092191194
:108F5000209124023091250240912602509127024F
:108F6000C701B6010F94500869837A838B839C8371
:108F700060932E1170932F118093301190933111C3
:108F8000209136113091371140913811509139119B
:108F9000C701B6010F94A2042B013C0120901E11C1
:108FA00030901F1110912011009121119101412F3A
:108FB000502F0F947B0587FD14C020901A1130901C
:108FC0001B1110911C1100911D119101412F502F67
:108FD000B201C3010F947E0718161CF01201162D62
:108FE000072DC101A12FB02F809336119093371117
:108FF000A0933811B09339112091200230912102B1
:109000004091220250912302B101812F902F0F94A1
:1090100050086D837E838F83988760932A117093A5
:109020002B1180932C1190932D112091321130919E
:1090300033114091341150913511C501B4010F9491
:10904000A10420911C0230911D0240911E025091FA
:109050001F020F94500820ED3CEC4CE45DE30F94AC
:1090600050082B013C0123E333E343E75FE36091C6
:1090700026117091271180912811909129110F9438
:1090800050089B01AC01C301B2010F94A2042B0153
:109090003C016093261170932711809328119093BF
:1090A00029112D813E814F81588569817A818B817B
:1090B0009C810F94A204A30192010F94A1042B019F
:1090C0003C0120E030E04FE753E40F947E0720E0BE
:1090D00030E0A9011816E4F4C701B6010F947E0729
:1090E00018167CF4A7019601B101812F902F0F94DF
:1090F000A1046093361170933711809338119093C7
:109100003911412C512CFFE76F2EF3E47F2E21C043
:10911000C301B2010F947B0587FF1BC020E030E044
:10912000A901C701B6010F947B0587FF0FC0A701F6
:109130009601B101812F902F0F94A10460933611F5
:10914000709337118093381190933911412C512C21
:1091500032018092321190923311A0923411B09268
:1091600035116091F0107091F110882777FD80958E
:10917000982F0F941D069B01AC01C501B4010F94FB
:109180007E071816DCF460910802709109028827A6
:1091900077FD8095982F0F941D069B01AC01C501AA
:1091A000B4010F947B0587FF09C0C301B2010F947E
:1091B000EA05759567956093F81002C01092F81053
:1091C0000E94C8FE0091F4101091F5102091F61045
:1091D0003091F710601B710B820B930B653C79404B
:1091E0008105910560F00E9482400E94C8FE609354
:1091F000F4107093F5108093F6109093F710809010
:10920000421190904311A0904411B090451160918B
:109210004E1170914F11882777FD8095982F0F94EC
:109220001D06A50194010F94A1046B017C016093BC
:1092300001117093021180930311909304112091F6
:1092400014023091150240911602509117020F94AA
:10925000500869837A838B839C8360930D1170938C
:109260000E1180930F1190931011209115113091D0
:1092700016114091171150911811C701B6010F94A2
:10928000A2048B011C016090FD107090FE105090A4
:10929000FF10409000119301452D542D0F947B0534
:1092A00087FD11C06090F9107090FA105090FB107B
:1092B0004090FC109301452D542DB801C1010F942D
:1092C0007E0718161CF48301252C342CC801D1010B
:1092D0008093151190931611A0931711B093181144
:1092E000209110023091110240911202509113020C
:1092F000B801C1010F9450086D837E838F839887D6
:109300006093091170930A1180930B1190930C11C3
:10931000209111113091121140911311509114119B
:10932000C501B4010F94A10420910C0230910D02EB
:1093300040910E0250910F020F94500820ED3CEC2A
:109340004CE45DE30F9450082B013C0123E333E32D
:1093500043E75FE360910511709106118091071159
:10936000909108110F9450089B01AC01C301B20108
:109370000F94A2042B013C01609305117093061118
:1093800080930711909308118092111190921211FD
:10939000A0921311B09214112D813E814F815885F6
:1093A00069817A818B819C810F94A204A30192012F
:1093B0000F94A1042B013C0120E030E04FE753E47F
:1093C0000F947E0720E030E0A9011816ACF4C70125
:1093D000B6010F947E0718166CF5A7019601B80127
:1093E000C1010F94A104609315117093161180931D
:1093F0001711909318111EC0C301B2010F947B0581
:1094000087FF22C020E030E0A901C701B6010F9418
:109410007B0587FF16C0A7019601B801C1010F9413
:10942000A1046093151170931611809317119093F6
:10943000181107C0412C512C5FE7652E53E4752E9F
:1094400003C0412C512C320120E030E040E751E4D0
:10945000C501B4010F947E0718169CF420E030E09B
:1094600046E153E4C501B4010F947B0587FF09C0B1
:10947000C301B2010F94EA05759567956093411198
:1094800002C01092411128960FB6F894DEBF0FBEAD
:10949000CDBFDF91CF911F910F91FF90EF90DF90A3
:1094A000CF90BF90AF909F908F907F906F905F9084
:1094B0004F903F902F900895CF93C82F0E945B410B
:1094C0000E942870811134C0E5E5F3E59491992359
:1094D00041F08091C00085FFFCCF9093C60031968B
:1094E000F5CF6C2F70E04AE050E08BE397E10E94EB
:1094F000C1DA8091C00085FFFCCF8AE08093C6006E
:10950000EFE2F2E08491882341F09091C00095FF52
:10951000FCCF8093C6003196F5CF8091C00085FFC7
:10952000FCCF8AE08093C60082E292E00E9462ADA6
:10953000CF910C94D06FCF93C82F0E945B410E94B3
:109540002870811134C0E5E5F3E59491992341F049
:109550008091C00085FFFCCF9093C6003196F5CF77
:109560006C2F70E04AE050E08BE397E10E94C1DA93
:109570008091C00085FFFCCF8AE08093C600E5EFB4
:10958000F1E08491882341F09091C00095FFFCCFD9
:109590008093C6003196F5CF8091C00085FFFCCF47
:1095A0008AE08093C60088EE91E00E9462ADCF9180
:1095B0000C94D06FA5980E942870811125C0E5E514
:1095C000F3E58491882341F09091C00095FFFCCF92
:1095D0008093C6003196F5CFEFEAF1E084918823BD
:1095E00041F09091C00095FFFCCF8093C60031966A
:1095F000F5CF8091C00085FFFCCF8AE08093C60044
:109600008EE991E00E9462AD0C94D06F1F920F9290
:109610000FB60F9211240BB60F920F931F932F9337
:109620003F934F935F936F937F938F939F93AF93EA
:10963000BF93CF93DF93EF93FF9380910702811144
:1096400012C08091F8108093ED10882311F0759A64
:1096500001C07598809141118093EC10882311F01E
:10966000A59A01C0A5989091ED10809107029817D6
:1096700008F475989091EC1080910702981708F4FF
:10968000A598809107028F5F8F7780930702809162
:10969000060290E08B30910508F093C0FC01EE5873
:1096A000FF4F0D94970910927B0080E480937C001B
:1096B00080917A00806480937A000E946BAD81E093
:1096C00019C020917800309179008091E810909134
:1096D000E910A091EA10B091EB10820F931FA11D29
:1096E000B11D8093E8109093E910A093EA10B09315
:1096F000EB1082E08093060264C010927B0082E44B
:1097000080937C0080917A00806480937A000E942C
:109710006BAD83E0EFCF209178003091790080919C
:10972000E4109091E510A091E610B091E710820F3F
:10973000931FA11DB11D8093E4109093E510A09399
:10974000E610B093E71084E0D5CF10927B0081E45F
:1097500080937C0080917A00806480937A000E94DC
:109760006BAD85E0C7CF2091780030917900809172
:10977000E0109091E110A091E210B091E310820FFF
:10978000931FA11DB11D8093E0109093E110A09351
:10979000E210B093E31086E0ADCF0E946BAD87E09E
:1097A000A9CF88E0A7CF0E946BAD89E0A3CF10922C
:1097B00006028091DF108F5F8093DF1002C010924D
:1097C00006028091DF10803108F463C080913A1165
:1097D000811110C08091E8109091E91090934D1183
:1097E00080934C118091E4109091E5109093471173
:1097F0008093461181E080933A111092DF1010920D
:10980000E8101092E9101092EA101092EB101092EA
:10981000E0101092E1101092E2101092E3101092FA
:10982000DB101092DC101092DD101092DE101092FE
:10983000E4101092E5101092E6101092E7102091BB
:109840004C1130914D118091F2109091F3108217CC
:10985000930714F080E030DE20914C1130914D11CF
:1098600080910A0290910B022817390714F080E0CA
:1098700062DE20914611309147118091EE10909157
:10988000EF10821793072CF010924F1110924E1187
:1098900091DE00E010E0E801CC0FDD1FC55CDE4E7C
:1098A000888199811816190644F461E0802F0E947E
:1098B000BDE488819981019709C0892B49F060E056
:1098C000802F0E94BDE488819981019699838883C5
:1098D0000F5F1F4F03301105F1F6FF91EF91DF91FC
:1098E000CF91BF91AF919F918F917F916F915F9138
:1098F0004F913F912F911F910F910F900BBE0F90A1
:109900000FBE0F901F9018952CEA35EC47E25EE3EE
:109910000D9450082CEA35EC47E25EE30D94820585
:109920002CEA35EC47E25EE30D9482052CEA35EC37
:1099300047E25EE30D945008CF93DF93EC0160E0C3
:109940008E810E9421FE81E090E00E941BFF61E079
:109950008E810E9421FE81E090E00E941BFF60E06A
:109960008E810E9421FE84E690E0DF91CF910C94DD
:109970001BFFCF92DF92EF92FF920F931F93CF9333
:10998000DF937C01C0E0D0E0C62ED12C87010C0F04
:109990001D1F61E0F80187810E94E8FDB6010C2ED1
:1099A00002C0759567950A94E2F76170F8018781A6
:1099B0000E9421FE2196C430D10541F7C701DF91F5
:1099C000CF911F910F91FF90EF90DF90CF90B4CF88
:1099D000CF92DF92EF92FF920F931F93CF93DF937B
:1099E0007C01C0E0D0E0C62ED12C87010C0F1D1FDA
:1099F00061E0F80187810E94E8FDB6010C2E02C0EB
:109A0000759567950A94E2F76170F80187810E9465
:109A100021FE2196C830D10541F7C701DF91CF91D2
:109A20001F910F91FF90EF90DF90CF9085CF1F9304
:109A3000CF93DF93EC01162F642F8C810E9421FEBF
:109A40008D818F3F19F060E00E9421FE8F85612F8C
:109A500084FF05C0CE01DF91CF911F91B9CF70E097
:109A600084E0759567958A95E1F7CE0182DF612FD5
:109A7000CE01DF91CF911F917CCF40E0D8CF61E044
:109A8000FCDF80E496E00C941BFF62E0F6DF80E4EC
:109A900096E00C941BFFCF93DF93CDB7DEB72897EA
:109AA0000FB6F894DEBF0FBECDBF28E0E7E9FCE0BB
:109AB000DE01119601900D922A95E1F7FC012389B0
:109AC000421710F04FEF420FFE013196E40FF11DE7
:109AD000E40FF11D2081260F2068622F28960FB613
:109AE000F894DEBF0FBECDBFDF91CF91C6CFFC0192
:109AF0006089262F2460208B6C60BFCFCF93DF93CB
:109B0000EC01423018F08F8588608F874B8B1C8A60
:109B1000222329F0413019F48F8584608F8780E5F6
:109B200093EC0E941BFF60E08C810E9421FE60E0AC
:109B30008E810E9421FE8D818F3F19F060E00E948E
:109B400021FE6F8564FD19C063E0CE0112DF84E958
:109B500091E10E941BFF63E0CE010BDF84E991E1FC
:109B60000E941BFF63E0CE0104DF86E990E00E94C3
:109B70001BFF62E0CE01FDDE13C06062CE017DDF1F
:109B800084E991E10E941BFF6F856062CE0175DF61
:109B900086E990E00E941BFF6F856062CE016DDF59
:109BA0006F856062CE0169DF8CE390E00E941BFF4D
:109BB00084E0888BCE019BDF8CE390E00E941BFF4A
:109BC000CE015DDF88EB9BE00E941BFF82E0898B6A
:109BD00066E0CE0152DF8CE390E0DF91CF910C94F0
:109BE0001BFF6F927F928F92AF92CF92EF920F9363
:109BF0001F93CF93DF93CDB7DEB73C01162F842F91
:109C00005E854F8538899989F3018483258306838E
:109C1000E782C086A18682865387448735879687E8
:109C200061E00E94E8FDF30185818F3F19F061E05A
:109C30000E94E8FD61E0F30186810E94E8FD1123A6
:109C400019F0F301178603C080E1F301878720E054
:109C500041E060E1C301DF91CF911F910F91EF903F
:109C6000CF90AF908F907F906F9048CF8F92AF92B0
:109C7000CF92EF920F93DC0113961C921E921297D3
:109C8000EDE5FDE0ED93FC931F921F921F921F9252
:109C90008C2CAE2CC02EE22E042F2FEF462F61E02D
:109CA000A0DF0F900F900F900F900F91EF90CF903B
:109CB000AF908F900895CF93DF93EC01423018F06E
:109CC0008F8588608F874B8B1C8A222329F0413037
:109CD00019F48F8584608F8780E593EC0E941BFFC9
:109CE00060E08C810E9421FE60E08E810E9421FE56
:109CF0008D818F3F19F060E00E9421FE6F8564FD29
:109D000019C063E0CE0135DE84E991E10E941BFFBA
:109D100063E0CE012EDE84E991E10E941BFF63E047
:109D2000CE0127DE86E990E00E941BFF62E0CE01B3
:109D300020DE13C06062CE01A0DE84E991E10E94C2
:109D40001BFF6F856062CE0198DE86E990E00E947D
:109D50001BFF6F856062CE0190DE6F856062CE0171
:109D60008CDE8CE390E00E941BFF84E0888BCE01A8
:109D7000BEDE8CE390E00E941BFFCE0186DE80E415
:109D800096E00E941BFF82E0898B66E0CE0175DEC3
:109D90008CE390E00E941BFF40E068E0CE017BDE98
:109DA00064E97EE0CE010F94310441E068E0CE0129
:109DB00072DE64E97EE0CE010F94310442E066E099
:109DC000CE0169DE62E97EE0CE01DF91CF910D9494
:109DD0003104CF92DF92EF92FF920F931F93CF93B4
:109DE000DF931F921F92CDB7DEB78C01677088E0BA
:109DF000689FB00111246064C80149835A833DDE25
:109E00004981C42E5A81D52EE12CF12CD6016D91B9
:109E10006D01D801ED91FC910190F081E02DC80118
:109E20001995BFEFEB1AFB0AE8E0EE16F10471F7A3
:109E30000F900F90DF91CF911F910F91FF90EF90B6
:109E4000DF90CF90089541E0F2DD81E090E0089549
:109E50000F931F93CF93DF93EC018B0144E150E00C
:109E6000BC018AE891E10F94AE0ECE010F948D0EE5
:109E7000992744E150E0481B590BB80186579E4E84
:109E80000F94AE0E8AE891E1DF91CF911F910F916F
:109E90000895AF92BF92CF92DF92EF92FF920F930D
:109EA0001F93CF93DF93EC015B017A01690144E1D9
:109EB00050E0BC018AE891E10F94AE0ECE010F9400
:109EC0008D0EEC01DD2704E110E0A8014C1B5D0BB9
:109ED000B501CE0186579E4E0F94AE0EC5010F946C
:109EE0008D0EC80FD91FDD27A8014C1B5D0BB701D4
:109EF000CE0186579E4E0F94AE0EC7010F948D0E65
:109F00008C0F9D1F9927A801481B590BB601865736
:109F10009E4E0F94AE0E8AE891E1DF91CF911F9192
:109F20000F91FF90EF90DF90CF90BF90AF9008958A
:109F30002F923F924F925F926F927F928F929F9259
:109F4000AF92BF92CF92DF92EF92FF920F931F9347
:109F5000CF93DF93CDB7DEB7CF54D1090FB6F894C6
:109F6000DEBF0FBECDBF1C017E8F6D8F4A012FABB0
:109F700009AF2896EFAE28972C96ACAEBDAECEAE0C
:109F8000DFAE2C9734E0239F50011124FC01EA0D31
:109F9000FB1D80819181A281B381898F9A8FAB8FC4
:109FA000BC8FDA01AA0DBB1DBCAFABAF4D905D906D
:109FB0006D907C90A3019201698D7A8D8B8D9C8D23
:109FC0000F94A20421966CAF7DAF8EAF9FAF219707
:109FD000B4E00B9F80011124F101E00FF11F2081FB
:109FE0003181428153812F8F38A349A35AA3A40101
:109FF000400F511F23965FAF4EAF2397DA01CD90EC
:10A00000DD90ED90FC90A70196016F8D78A189A15C
:10A010009AA10F94A20427966CAF7DAF8EAF9FAF2D
:10A0200027972896EFAD2897B4E0EB9FC001112445
:10A03000F101E80FF91F20813181428153812BA367
:10A040003CA34DA35EA3ED8DFE8DE80FF91F60814B
:10A050007181828193810F94A1046FA378A789A74E
:10A060009AA7AD8DBE8D1C968D919D910D90BC9142
:10A07000A02D60968CAF9DAFAEAFBFAF6097D10102
:10A080001C962D913D914D915C911F972BA73CA75C
:10A090004DA75EA7A301920150582D8B3E8B4F8B8D
:10A0A000588FD701C601B058898B9A8BAB8BBC8B6C
:10A0B000ED8DFE8DEA0DFB1D2081318142815381A2
:10A0C0002FA738AB49AB5AAB21962CAD3DAD4EAD69
:10A0D0005FAD21976FA578A989A99AA90F94A104CA
:10A0E0006B017C01ED8DFE8DE00FF11F8081918170
:10A0F000A281B3818BAB9CABADABBEAB27962CAD35
:10A100003DAD4EAD5FAD2797BC01CD010F94A104CD
:10A110004B015C01A70196016D897E898F89988D1D
:10A120000F9450082B013C01A501940169897A899B
:10A130008B899C890F9450089B01AC01C301B2012B
:10A140000F94A2042B013C01A50194016D897E8925
:10A150008F89988D0F9450084B015C01A7019601DF
:10A1600069897A898B899C890F9450089B01AC017D
:10A17000C501B4010F94A104A30192010F94150528
:10A180006B017C0120E030E0A9010F947B0587FF83
:10A190000AC02BED3FE049EC50E4C701B6010F9433
:10A1A000A2046B017C01AA968FADAA97882351F077
:10A1B0002BED3FE049EC50E4C701B6010F94A10438
:10A1C0006B017C012FA538A949A95AA9698D7A8DFF
:10A1D0008B8D9C8D0F947B0581111FC02BA93CA9F1
:10A1E0004DA95EA96F8D78A189A19AA10F947B05D5
:10A1F000811113C020E030E0A901C701B6010F941E
:10A200007B0581110AC02BED3FE049EC50E4C7010A
:10A21000B6010F94A2046B017C01A9962CAD3DAD53
:10A220004EAD5FADA997C701B6010F9450082FA19D
:10A2300038A549A55AA55F770F948B074B015C01A0
:10A240002FE632E143E85AE30F947B0587FDC8C14E
:10A25000C501B4010F9458060F94EF057A8F698FEA
:10A26000DB01AB2B21F4E1E0F0E0FA8FE98F298DDF
:10A270003A8DB90180E090E00F941B064B015C0120
:10A280009B01AC01C701B6010F9482052B013C0173
:10A29000A50194016FA178A589A59AA50F948205BF
:10A2A0006FA778AB89AB9AAB2BA53CA54DA55EA556
:10A2B00060966CAD7DAD8EAD9FAD60970F94A1049F
:10A2C000A50194010F9482056BAB7CAB8DAB9EAB6B
:10A2D00020E030E040E05FE3C301B2010F9450089A
:10A2E000A30192010F9450089B01AC0160E070E063
:10A2F00080E89FE30F94A1046FA378A789A79AA78A
:10A30000CE010196FC0128964FAD289734E0439F7B
:10A31000E00DF11D11242BA13CA14DA15EA12083D4
:10A320003183428353832BA53CA54DA55EA52D8784
:10A330003E874F87588BB12C41E050E058A34F8F98
:10A340001C01BFA9A4E0BA9F800D911D112498AFF4
:10A350008FAB910159AD44E0549F200D311D112464
:10A360003AAF29AFFCA7EBA74F8D58A1898D9A8DE5
:10A370004817590708F01AC188E18B150CF444C03E
:10A380002FA138A549A55AA569897A898B899C8905
:10A390000F9450086B017C01A30192016D897E89A5
:10A3A0008F89988D0F945008A70196010F94A204ED
:10A3B000A62E172F982E892E2FA138A549A55AA56C
:10A3C0006D897E898F89988D0F9450086B017C016F
:10A3D000A301920169897A898B899C890F9450081D
:10A3E0009B01AC01C701B6010F94A1046D8B7E8B5C
:10A3F0008F8B988FB3948A2D912FA92DB82D898B8F
:10A400009A8BAB8BBC8B6CC0AF8DB8A1BD0180E0CB
:10A4100090E00F941B06A30192010F9450086B016A
:10A420007C010F947F05698B7A8B8B8B9C8BC7018A
:10A43000B6010F94B3084B015C01EBADFCADC080DD
:10A44000D180E280F380F7FAF094F7F8F094239645
:10A45000AEADBFAD23972D913D914D915C912BA356
:10A460003CA34DA35EA329893A894B895C89C70126
:10A47000B6010F9450086D8B7E8B8F8B988FA50142
:10A4800094016BA17CA18DA19EA10F9450089B010A
:10A49000AC016D897E898F89988D0F94A2046D8B94
:10A4A0007E8B8F8B988FA5019401C701B6010F9405
:10A4B00050086B017C0129893A894B895C896BA121
:10A4C0007CA18DA19EA10F9450089B01AC01C701F6
:10A4D000B6010F94A104698B7A8B8B8B9C8BB12C6A
:10A4E0002D893E894F89588D21966CAD7DAD8EADFD
:10A4F0009FAD21970F94A204EFA9F8AD60837183FB
:10A500008283938329893A894B895C8927966CAD2C
:10A510007DAD8EAD9FAD27970F94A204A9ADBAADC6
:10A520006D937D938D939C9313972FA538A949A97B
:10A530005AA9EBA5FCA560817181828193810F945A
:10A54000A204ABA5BCA56D937D938D939C931397AB
:10A550002BA93CA94DA95EA96D857E858F8598891B
:10A560000F94A2046D877E878F87988BC1010E940C
:10A57000006AFE01E659FF4F6F012C96ECACFDAC72
:10A580000EAD1FAD2C979E01235F3F4FAE01475F7D
:10A590005F4FBE016B5F7F4FC1010E9498EF2F8D0F
:10A5A00038A12F5F3F4F38A32F8FDECE2D8D3E8DEC
:10A5B000245F3F4F4D8D5E8D485F5F4F6D8D7E8D6B
:10A5C0006C5F7F4FDE01A659BF4F6D012C96ECAC3E
:10A5D000FDAC0EAD1FAD2C978D8D9E8D0E9498EF1A
:10A5E000C15BDF4F0FB6F894DEBF0FBECDBFDF916A
:10A5F000CF911F910F91FF90EF90DF90CF90BF9080
:10A60000AF909F908F907F906F905F904F903F9012
:10A610002F900895FC01148217821382128289EB15
:10A620009EE091838083089529EB3EE0FC01318315
:10A6300020832781222319F004960C943035089545
:10A64000CF92DF92EF92FF920F931F93CF93DF93FE
:10A65000EC01875B9F4FDEDFCE0186599F4FDADF2B
:10A660007E0129E8E20EF11C87016E0131E4C31A74
:10A670003EEFD30AC801CEDF015E1F4F0C151D054A
:10A68000C9F7FE01EF53FE4F89E1818314823596AD
:10A69000178ACE018C519E4FBDDFFE01EB56FD4F58
:10A6A00010821182128213823896108211821282D5
:10A6B00013821A821B82188219826E0187E6C81AD9
:10A6C0008DEFD80AF6011082118212821382F801EE
:10A6D00011821082FE01ED5FFD4F108286E391E052
:10A6E000F7019C01119221503040E1F7FE01EF5536
:10A6F000FD4F81E08083C95BDF4F198218820E9481
:10A70000C8FE68577C4E8F4F9F4FF6016083718360
:10A7100082839383DF91CF911F910F91FF90EF90F0
:10A72000DF90CF900895FC0120E03EE2DB014C91E8
:10A73000403241F0283011F430833196DB014C91E6
:10A74000408331962F5F6F5F7F4F2B3079F71082F8
:10A7500008952F923F924F925F926F927F928F92C5
:10A760009F92AF92BF92CF92DF92EF92FF920F93A0
:10A770001F93CF93DF93CDB7DEB7CA58D1090FB679
:10A78000F894DEBF0FBECDBF8C016B017A01490189
:10A79000CA57DF4F1882C658D04084E0E80EF11C3B
:10A7A000180191E1290E311CF801EA5BFF4FC957EE
:10A7B000DF4FF983E883C758D0403801FEE56F1AB0
:10A7C000FDEF7F0A58018CE5A81A8DEFB80A90E4D6
:10A7D000492E512C4C0E5D1E94E0490E511CA101D6
:10A7E000BE016F5F7F4FC7010E949A3318160CF0AD
:10A7F0004AC12C85322F3871303109F0ACC0F301D9
:10A80000808191810197029708F4A5C0BE016F5F16
:10A810007F4FCE0187589F4F86DFA0961FAEA0972F
:10A82000F6018081811107C061E67DE0CE01815A89
:10A830009F4F0F94070FB601CE01815A9F4F0F947F
:10A84000070FBE0167587F4FCE01815A9F4F0F946B
:10A85000070F61E67DE0CE01815A9F4F0F94070FED
:10A86000CE01805C9F4FD6DE21E0AE0147585F4F9E
:10A87000B701C2010E942737811147C0F3018081CF
:10A880009181892B09F041C0EFE4F3E5849188239D
:10A8900041F09091C00095FFFCCF8093C6003196A7
:10A8A000F5CFE091BB13F0E0EE0FFF1FE85DFD4F29
:10A8B0000190F081E02DE457FE4F0190F081E02DF2
:10A8C0008191882339F09091C00095FFFCCF80934F
:10A8D000C600F6CF8091C00085FFFCCF8AE0809350
:10A8E000C600FE01E758FF4F8191882339F090910F
:10A8F000C00095FFFCCF8093C600F6CF8091C000CA
:10A9000085FFFCCF8AE08093C6008BE1FE01EC5B03
:10A91000FF4FDE01959601900D928A95E1F72496FE
:10A920008EAD9FAD24979CA38BA389EB9EE09AA349
:10A9300089A320E030E0AE014F5D5F4FBE01615A58
:10A940007F4FC80106DFCE0181966EDECE01805CAE
:10A950009F4F6ADE44CF8981882309F494C08E32E8
:10A9600009F43DCF8F3509F43ACFF80181898E3251
:10A9700009F435CF8F3509F432CF23FD30CF81E094
:10A98000303109F080E0C957DF4FE881F981C758BD
:10A99000D0408083811108C08985873409F01FCF9A
:10A9A0008A858E3709F41BCF98012C5F3F4FBE017B
:10A9B0006F5F7F4FC901C757DF4F2883C958D04009
:10A9C000C657DF4F3883CA58D040ADDEF3018081CF
:10A9D0009181C757DF4F2881C958D040C657DF4FF4
:10A9E0003881CA58D0400097F1F4F601819188234C
:10A9F00039F09091C00095FFFCCF8093C600F6CF50
:10AA0000F9018191882339F09091C00095FFFCCF26
:10AA10008093C600F6CF8091C00085FFFCCF8AE00E
:10AA20008093C600DCCE8130910539F4F501808138
:10AA30009181019691838083D2CE029709F0CFCE87
:10AA40008114910439F0B901C4010F94F40E892BDB
:10AA500071F419C0CA57DF4FF881C658D0402F2F64
:10AA600030E0F501808191812817390761F0CA57DC
:10AA7000DF4FF881C658D040FF5FCA57DF4FF883D9
:10AA8000C658D040ACCEC657DF4F0FB6F894DEBFE5
:10AA90000FBECDBFDF91CF911F910F91FF90EF902F
:10AAA000DF90CF90BF90AF909F908F907F906F90EE
:10AAB0005F904F903F902F9008950F931F93CF93E7
:10AAC000DF93CDB7DEB76F970FB6F894DEBF0FBE3A
:10AAD000CDBF8C01FC01EE55FD4F1182108240E08C
:10AAE00050E0BA01835B9F4F0E944D34C801875BE1
:10AAF0009F4F2BE1FC013496DE01159601900D92DB
:10AB00002A95E1F7FC01828193819C838B8389EBF9
:10AB10009EE09A83898320E030E0AE014F5F5F4F73
:10AB20006AE97EE0C80115DECE0101967DDD6F96F3
:10AB30000FB6F894DEBF0FBECDBFDF91CF911F914E
:10AB40000F9108952BE1FB013496DC0114960190DE
:10AB50000D922A95E1F7FB0122813381FC013383B9
:10AB600022830895EF92FF920F931F93CF93DF9369
:10AB7000EC011B82FC01E05BFF4F8081882329F000
:10AB8000CE01835B9F4F0E9430357E018FE3E81A30
:10AB90008EEFF80A45E360E0C7010E946E61811103
:10ABA0002CC0EFE4F3E58491882341F09091C0003C
:10ABB00095FFFCCF8093C6003196F5CFE091BB1393
:10ABC000F0E0EE0FFF1FE85DFD4F0190F081E02DFA
:10ABD000E257FE4F0190F081E02D8491882341F0EF
:10ABE0009091C00095FFFCCF8093C6003196F5CFC1
:10ABF0008091C00085FFFCCF9EC08E010A531E4F7E
:10AC000041E0B701C8010E94FE3C811133C040E021
:10AC1000B701C8010E94FE3C81112CC0E5E5F3E5B7
:10AC20008491882341F09091C00095FFFCCF8093E0
:10AC3000C6003196F5CFE091BB13F0E0EE0FFF1F99
:10AC4000E85DFD4F0190F081E02DE057FE4F01904F
:10AC5000F081E02D8491882341F09091C00095FF10
:10AC6000FCCF8093C6003196F5CF8091C00085FF60
:10AC7000FCCF61C0B801CE01835B9F4F0E943D3283
:10AC800081112CC0E5E5F3E58491882341F0909192
:10AC9000C00095FFFCCF8093C6003196F5CFE091C0
:10ACA000BB13F0E0EE0FFF1FE85DFD4F0190F08158
:10ACB000E02DEE56FE4F0190F081E02D8491882327
:10ACC00041F09091C00095FFFCCF8093C600319673
:10ACD000F5CF8091C00085FFFCCF2DC081E08B8334
:10ACE000EFE4F3E58491882341F09091C00095FF53
:10ACF000FCCF8093C6003196F5CFE091BB13F0E016
:10AD0000EE0FFF1FE85DFD4F0190F081E02DEC5646
:10AD1000FE4F0190F081E02D8491882341F09091C5
:10AD2000C00095FFFCCF8093C6003196F5CF80918F
:10AD3000C00085FFFCCF8AE08093C6008E01075BD0
:10AD40001F4FB801CE0186599F4FFCDEC859DF4F17
:10AD500019830883DF91CF911F910F91FF90EF909E
:10AD60000895FC01128213820895FC01238122239D
:10AD700011F021E022830895FC0122812111128229
:10AD80000895AF92BF92CF92DF92EF92FF920F930E
:10AD90001F93CF93DF931F92CDB7DEB78C018FE265
:10ADA000FB0181935F01D12C41E07801F1E4EF1ABE
:10ADB000FEEFFF0A6FE1C62E2D2D30E0F7018081F6
:10ADC000918128173907D8F4C29EC001C39E900D07
:10ADD000112483579F4FB501800F911F49830E9413
:10ADE000E431C50149815C010196F50120812223EE
:10ADF00021F04D3810F44F5FF6CFD394DDCF47FDEF
:10AE000011C0B501C80188519E4F0F90DF91CF91BD
:10AE10001F910F91FF90EF90DF90CF90BF90AF9078
:10AE20000C94E431F50110820F90DF91CF911F91C6
:10AE30000F91FF90EF90DF90CF90BF90AF9008956B
:10AE40003F924F925F926F927F928F929F92AF92BA
:10AE5000BF92CF92DF92EF92FF920F931F93CF9307
:10AE6000DF93CDB7DEB7AC970FB6F894DEBF0FBE59
:10AE7000CDBF7C015B01FC018381882309F408C1FB
:10AE8000C70188519E4F0E943035F7011282CE01D2
:10AE900001966C01BFDB270198E6490E511CC701E2
:10AEA000875B9F4FF20191838083F50180818F3210
:10AEB00009F084C06FE270E0C5010F94120F8C019D
:10AEC0000F5F1F4F7AE0372E0115110509F47CC082
:10AED0006FE270E0C8010F94120F4C01009709F463
:10AEE00074C00817190708F070C03C01601A710A95
:10AEF000A301B801CE0180960F943B0FE0E2F0E091
:10AF0000EC0FFD1FE60DF71D1082FE01B09681913A
:10AF1000882339F09091C00095FFFCCF8093C60044
:10AF2000F6CF8091C00085FFFCCF3092C600F201C1
:10AF3000608171816115710519F06C5F7F4F02C0EE
:10AF400060E070E021E0AE01405E5F4FCE0105960B
:10AF50000E94273781112BC0E3E6FDE0849188230E
:10AF600041F09091C00095FFFCCF8093C6003196D0
:10AF7000F5CFFE01B0968191882339F09091C00001
:10AF800095FFFCCF8093C600F6CFEAEFFEE48491F4
:10AF9000882341F09091C00095FFFCCF8093C600BC
:10AFA0003196F5CF8091C00085FFFCCF6CC0F201D7
:10AFB000D182C08284010F5F1F4F86CFC70186599F
:10AFC0009F4FF201918380838501F20180819181FD
:10AFD000009711F0049602C080E090E0B8010E9452
:10AFE000FD37882339F1ECEEFEE48491882341F0AB
:10AFF0009091C00095FFFCCF8093C6003196F5CFAD
:10B00000F8018191882339F09091C00095FFFCCF21
:10B010008093C600F6CF8091C00085FFFCCF8AE008
:10B020008093C600F701E356FD4F10821182128211
:10B0300013822CC0E4EDFEE48491882341F09091CA
:10B04000C00095FFFCCF8093C6003196F5CFF80184
:10B050008191882339F09091C00095FFFCCF8093B7
:10B06000C600F6CFE2EDFEE48491882341F0909192
:10B07000C00095FFFCCF8093C6003196F5CF80913C
:10B08000C00085FFFCCF8AE08093C600C601CCDA01
:10B09000AC960FB6F894DEBF0FBECDBFDF91CF9157
:10B0A0001F910F91FF90EF90DF90CF90BF90AF90E6
:10B0B0009F908F907F906F905F904F903F900895FA
:10B0C0008F929F92AF92BF92CF92DF92EF92FF92B8
:10B0D000CF93DF931F92CDB7DEB77C01FC01828155
:10B0E000882309F4BCC071968191882339F090912E
:10B0F000C00095FFFCCF8093C600F6CFE0EDFEE4E4
:10B100008491882341F09091C00095FFFCCF8093FB
:10B11000C6003196F5CFE091BB13F0E0EE0FFF1FB4
:10B12000E85DFD4F0190F081E02DEE55FE4F01905E
:10B13000F081E02D8491882341F09091C00095FF2B
:10B14000FCCF8093C6003196F5CFF701E356FD4F53
:10B1500040815181628173812AE030E08BE397E185
:10B160000E94EDDAEEECFEE48491882341F09091A8
:10B17000C00095FFFCCF8093C6003196F5CFF70154
:10B18000EB56FD4F40815181628173812AE030E0AE
:10B190008BE397E10E94EDDA8091C00085FFFCCF40
:10B1A0008AE08093C6000E94C8FEE0E6CE2EEAEE5A
:10B1B000DE2EE12CF12CA70196010F9459094901CB
:10B1C0005A016091AB117091AC118091AD119091C9
:10B1D000AE11A70196010F945909821A930AC4016E
:10B1E0006CE370E00F9432096983CE0101960E94EE
:10B1F000EEAEFC012191CF01222339F03091C00045
:10B2000035FFFCCF2093C600F4CF40E050E06AE366
:10B210008BE397E10E94A5DAC4016CE370E00F9420
:10B2200032098983CE0101960E94EEAEFC01219184
:10B23000CF01222339F03091C00035FFFCCF20939D
:10B24000C600F4CFECECFEE484918823E1F0909109
:10B25000C00095FFFCCF8093C6003196F5CFE7E79D
:10B26000FDE08491882341F09091C00095FFFCCFD0
:10B270008093C6003196F5CF8091C00085FFFCCF4A
:10B280008AE08093C6000F90DF91CF91FF90EF90FE
:10B29000DF90CF90BF90AF909F908F900895AF9226
:10B2A000BF92CF92DF92EF92FF920F931F93CF93B3
:10B2B000DF935C01EB01FB0101900020E9F78F01B6
:10B2C00001501109061B170B6C01F8E1CF1AFEEFB4
:10B2D000DF0AF60110826EE470E0CE010F94120FC7
:10B2E0007C01009729F4F8013197EC0FFD1F0DC088
:10B2F00060E270E00F94120FEC0121966AE270E0B8
:10B30000C7010F94120FFC0131978DE081838AE011
:10B3100082831382BE01C5018C519E4F0E94AADB1D
:10B32000F6018081882371F1E5E5F3E584918823B6
:10B3300041F09091C00095FFFCCF8093C6003196FC
:10B34000F5CFE091BB13F0E0EE0FFF1FE85DFD4F7E
:10B350000190F081E02DEA55FE4F0190F081E02D43
:10B360008491882341F09091C00095FFFCCF809399
:10B37000C6003196F5CF8091C00085FFFCCF8AE0F2
:10B380008093C600DF91CF911F910F91FF90EF90B6
:10B39000DF90CF90BF90AF9008952F923F924F9241
:10B3A0005F926F927F928F929F92AF92BF92CF9255
:10B3B000DF92EF92FF920F931F93CF93DF93CDB75E
:10B3C000DEB7CC55D1090FB6F894DEBF0FBECDBFA6
:10B3D0004C018C010F551D4F662339F0F801108286
:10B3E000F401838181111DC015C0F801808188237B
:10B3F00009F4AFC0F401E756FD4FC080D180E28070
:10B40000F3800E94C8FEC616D706E806F90608F4BF
:10B41000A0C0E4CFC401A6DBF4018381882309F432
:10B4200098C07401F7E4EF0EF11CF70181818F934E
:10B4300080818F9383EC9EE49F938F938E01015CB8
:10B440001F4F1F930F930F944A0F0F900F900F9061
:10B450000F900F900F90B12CF80101900020E9F7A8
:10B460003197E01BF10BBE1684F46801CB0CD11CA4
:10B47000B7FCDA94F6018081992787FD90950F94A7
:10B480007E0EF6018083B394E7CFFDE48F0E911C0E
:10B4900040E050E0BA01C4010E944D34512CCE016D
:10B4A00001966C018CEB682E8EE4782E5E0191E2A1
:10B4B000A90EB11C40E050E0B601C4010E949A33CD
:10B4C0001816DCF5412CF60101900020E9F73197C0
:10B4D000EC19FD094E1674F41601240C311C47FCBE
:10B4E0003A94F101808190E00F947E0EF101808307
:10B4F0004394E9CF8A858E37E9F245E050E0B80100
:10B50000C6010F942D0F892BA9F61F930F937F92DD
:10B510006F92BF92AF920F944A0FC5010E94A76528
:10B5200088EB9EE40E9427660F900F900F900F907B
:10B530000F900F9055245394BDCF511004C08FEF3E
:10B540009FEFF70104C0F7018081918101969183FB
:10B550008083C45ADF4F0FB6F894DEBF0FBECDBF55
:10B56000DF91CF911F910F91FF90EF90DF90CF90DF
:10B57000BF90AF909F908F907F906F905F904F9013
:10B580003F902F9008950F931F93CF93DF93EC017B
:10B590008C0108511E4FC8010E94E634C8010E9468
:10B5A000303518821982DF91CF911F910F91089544
:10B5B000CF92DF92EF92FF920F931F93CF93DF937F
:10B5C000CDB7DEB76F970FB6F894DEBF0FBECDBF15
:10B5D0008C016A017C0188E6E80EF11CC8018659DD
:10B5E0009F4FF70191838083E65CFD4F22E030E0BE
:10B5F0003183208332967183608340E050E0BA014A
:10B6000004960E944D34F701808191812BE1FC0169
:10B610003496DE01159601900D922A95E1F7FC0112
:10B62000828193819C838B8389EB9EE09A838983BB
:10B630009601AE014F5F5F4F6AE97EE0C80189D88D
:10B64000CE0101960E9414536F960FB6F894DEBF98
:10B650000FBECDBFDF91CF911F910F91FF90EF9063
:10B66000DF90CF9008952F923F924F925F926F920A
:10B670007F928F929F92AF92BF92CF92DF92EF9282
:10B68000FF920F931F93CF93DF93CDB7DEB7AC97A5
:10B690000FB6F894DEBF0FBECDBF8C016B01342E08
:10B6A000DC0113968C91882309F449C3F801E55114
:10B6B000FE4F8081882309F4F5C02111C1C07801B3
:10B6C000BDEFEB1AFB0AF7018081882361F1E5E504
:10B6D000F3E58491882341F09091C00095FFFCCF61
:10B6E0008093C6003196F5CFEEE4FFE48491882381
:10B6F00041F09091C00095FFFCCF8093C600319639
:10B70000F5CF4AE050E061E070E08BE397E10E9402
:10B71000C1DA8091C00085FFFCCF8AE08093C6002B
:10B720000E94736F0CC3EFE4F3E58491882341F02A
:10B730009091C00095FFFCCF8093C6003196F5CF65
:10B74000E5E3FFE48491882341F09091C00095FFE8
:10B75000FCCF8093C6003196F5CFF6018191882306
:10B7600039F09091C00095FFFCCF8093C600F6CFD2
:10B77000EAE2FFE48491882341F09091C00095FFB4
:10B78000FCCF8093C6003196F5CFD7018C91FDE8B0
:10B79000BF2EB801B89E600D711D1124685F7D4FEA
:10B7A000C801EFDAF7018081F801B89EE00DF11DC4
:10B7B0001124E85FFD4F8191882339F09091C000FA
:10B7C00095FFFCCF8093C600F6CFE4E2FFE48491BE
:10B7D000882341F09091C00095FFFCCF8093C60074
:10B7E0003196F5CF5801F3E6AF1AFDEFBF0AD50148
:10B7F0004D915D916D917C912AE030E08BE397E172
:10B800000E94EDDA8091C00085FFFCCF8AE0809332
:10B81000C600F7012081F80184E0289FE00DF11DAA
:10B820001124EC5FFD4FD5014D915D916D917C919F
:10B8300040835183628373832F5FF70120832CC081
:10B84000EFE4F3E58491882341F09091C00095FFE7
:10B85000FCCF8093C6003196F5CFE3E1FFE48491FD
:10B86000882341F09091C00095FFFCCF8093C600E3
:10B870003196F5CFF6018191882339F09091C0007F
:10B8800095FFFCCF8093C600F6CF8091C00085FF66
:10B89000FCCF8AE08093C600C80188519E4F0E9469
:10B8A000303530C0F801ED5FFD4F1082EFE4F3E575
:10B8B0008491882341F09091C00095FFFCCF809344
:10B8C000C6003196F5CFE2E0FFE48491882341F091
:10B8D0009091C00095FFFCCF8093C6003196F5CFC4
:10B8E000F6018191882339F09091C00095FFFCCF3B
:10B8F0008093C600F6CF8091C00085FFFCCF8AE020
:10B900008093C600D80112961C92FE0131965F0109
:10B91000CF010E940A532801F8E64F0E511CC801BE
:10B92000875B9F4FD2018D939C93F60180818F326C
:10B9300009F091C06FE270E0C6010F94120F0196FA
:10B940007C01EAE02E2EE114F10409F48AC06FE2D2
:10B9500070E0C7010F94120F4C01009709F482C0E8
:10B96000E816F90608F07EC03C016E187F08A301B6
:10B97000B701CE0180960F943B0FE0E2F0E0EC0FB0
:10B98000FD1FE60DF71D1082FE01B0968191882300
:10B9900039F09091C00095FFFCCF8093C600F6CFA0
:10B9A0008091C00085FFFCCF2092C600D2016D912E
:10B9B0007C916115710519F06C5F7F4F02C060E0EA
:10B9C00070E021E0AE01405E5F4FCE0105960E941F
:10B9D0002737811138C0E091BB13F0E0EE0FFF1F55
:10B9E000E85DFD4F0190F081E02DE856FE4F01909B
:10B9F000F081E02D8491882341F09091C00095FF63
:10BA0000FCCF8093C6003196F5CFFE01B0968191B0
:10BA1000882339F09091C00095FFFCCF8093C60039
:10BA2000F6CFE0E0FFE48491882341F09091C000DC
:10BA300095FFFCCF8093C6003196F5CF8091C00072
:10BA400085FFFCCF43C1F201B182A0827401FFEFF8
:10BA5000EF1AFF0A78CFC80186599F4FD2018D9304
:10BA60009C937601F801E851FE4F4F01332009F411
:10BA7000E5C0D2016D917C916115710519F06C5F83
:10BA80007F4F02C060E070E021E0A701C4010E9486
:10BA900027372091BB13882309F49AC0F4018189C8
:10BAA0009289A389B489F801EB56FD4F8083918375
:10BAB000A283B383E22FF0E0EE0FFF1FE85DFD4F9E
:10BAC0000190F081E02DE656FE4F0190F081E02DCF
:10BAD0008491D801AB56BD4F882349F09091C000A6
:10BAE00095FFFCCF8093C60031968491F5CFF70186
:10BAF0008191882339F09091C00095FFFCCF80930D
:10BB0000C600F6CFE091BB13F0E0EE0FFF1FE85D3B
:10BB1000FD4F0190F081E02DE456FE4F0190F08141
:10BB2000E02D8491882341F09091C00095FFFCCFD7
:10BB30008093C6003196F5CF4D915D916D917C91CA
:10BB40002AE030E08BE397E10E94EDDA8091C000BB
:10BB500085FFFCCF8AE08093C600F801E356FD4FD5
:10BB60001082118212821382E091BB13F0E0EE0F7B
:10BB7000FF1FE85DFD4F0190F081E02DE256FE4F82
:10BB80000190F081E02D8491882341F09091C000D4
:10BB900095FFFCCF8093C6003196F5CF8091C00011
:10BBA00085FFFCCF8AE08093C600A70160E070E0CB
:10BBB000C801FEDCD80151968C91882319F0C80188
:10BBC000419601C0C7010E945EAB84E89DE0B2C00F
:10BBD000E22FF0E0EE0FFF1FE85DFD4F0190F081D6
:10BBE000E02DE856FE4F0190F081E02D84918823EE
:10BBF00041F09091C00095FFFCCF8093C600319634
:10BC0000F5CFF7018191882339F09091C00095FF1D
:10BC1000FCCF8093C600F6CFEEEFFEE4849188233C
:10BC200041F09091C00095FFFCCF8093C600319603
:10BC3000F5CF8091C00085FFFCCF48C0F201608144
:10BC400071816115710519F06C5F7F4F02C060E072
:10BC500070E026E5A701C4010E94273781113AC090
:10BC6000E091BB13F0E0EE0FFF1FE85DFD4F019088
:10BC7000F081E02DE856FE4F0190F081E02D849197
:10BC8000882341F09091C00095FFFCCF8093C600BF
:10BC90003196F5CFF7018191882339F09091C0005A
:10BCA00095FFFCCF8093C600F6CFECEFFEE48491C5
:10BCB000882341F09091C00095FFFCCF8093C6008F
:10BCC0003196F5CF8091C00085FFFCCF8AE080934C
:10BCD000C60032C081E0D8018C93E091BB13F0E044
:10BCE000EE0FFF1FE85DFD4F0190F081E02DE05663
:10BCF000FE4F0190F081E02D8491882341F09091D6
:10BD0000C00095FFFCCF8093C6003196F5CFF601B9
:10BD10008191882339F09091C00095FFFCCF8093EA
:10BD2000C600F6CF8091C00085FFFCCF8AE08093EB
:10BD3000C600C7010E945EABC5010E941453AC96B9
:10BD40000FB6F894DEBF0FBECDBFDF91CF911F912C
:10BD50000F91FF90EF90DF90CF90BF90AF909F90AA
:10BD60008F907F906F905F904F903F902F900895AD
:10BD700021E0FC01218340E076CCCF92DF92EF926C
:10BD8000FF920F931F93CF93DF93CDB7DEB76F97DB
:10BD90000FB6F894DEBF0FBECDBF8C016C0128E654
:10BDA000C20ED11C86599F4FF60191838083E65CB9
:10BDB000FD4F21E030E0318320837801FCE5EF1A6C
:10BDC000FDEFFF0AF7011182108240E050E0BA0156
:10BDD00004960E944D34F601808191812BE1FC0193
:10BDE0003496DE01159601900D922A95E1F7FC013B
:10BDF000828193819C838B8389EB9EE09A838983E4
:10BE000020E030E0AE014F5F5F4F6AE97EE0C8019D
:10BE10000E94A953CE0101960E941453F70180811C
:10BE200091816F960FB6F894DEBF0FBECDBFDF9144
:10BE3000CF911F910F91FF90EF90DF90CF900895D9
:10BE4000AF92BF92CF92DF92EF92FF920F931F9328
:10BE5000CF93DF93CDB7DEB76F970FB6F894DEBF01
:10BE60000FBECDBF8C017B01CE0101960E940A530B
:10BE7000F801EF58FF4F80816801811104C029E467
:10BE8000C20ED11C03C08AE6C80ED11C21E0A70156
:10BE9000B6016C5F7F4FCE0105960E942737811156
:10BEA0003AC0EFE4F3E58491882341F09091C0001B
:10BEB00095FFFCCF8093C6003196F5CFE091BB1380
:10BEC000F0E0EE0FFF1FE85DFD4F0190F081E02DE7
:10BED000E855FE4F0190F081E02D8491882341F0D8
:10BEE0009091C00095FFFCCF8093C6003196F5CFAE
:10BEF000F7018191882339F09091C00095FFFCCF24
:10BF00008093C600F6CF8091C00085FFFCCF8AE009
:10BF10008093C60036C0F801E154FE4F80819181C4
:10BF20008A30910530F59C012F5F3F4F318320838C
:10BF30002FE1289F7001299FF00C112429E8E20EBF
:10BF4000F11CE00EF11E5C01B701C7014F960E9483
:10BF5000A25581E0A81AB1082FE1E21AF1088FEF8B
:10BF6000A816B80689F7B601C80187579F4F0E94E7
:10BF7000A255BE016F5F7F4FC80186599F4F0E9437
:10BF8000A255CE0101960E9414536F960FB6F894F5
:10BF9000DEBF0FBECDBFDF91CF911F910F91FF90FC
:10BFA000EF90DF90CF90BF90AF900895EF92FF9207
:10BFB0000F931F93CF93DF93EC01C154DE4F288181
:10BFC000398121153105F9F0215031093983288350
:10BFD0008C0107571F4FB80186599F4F0E94A255E9
:10BFE000C80100E010E07C012FE1E20EF11C288185
:10BFF00039810217130738F40F5F1F4FB7010E94F2
:10C00000A255C701F0CFDF91CF911F910F91FF9003
:10C01000EF900895EF92FF920F931F93CF93DF93CA
:10C02000EC010E9415E48E010D5F1D4FF801808127
:10C030009E0128513E4F79018823A1F1C9010E9438
:10C040003035F801808181508083BE01FDE88F9FEB
:10C05000600D711D1124685F7D4F21E041E0CE012C
:10C0600002DBF8018081FE0124E0829FE00DF11DDA
:10C070001124EC5FFD4F4081518162817381FE018B
:10C08000E356FD4F4083518362837383C7010E944F
:10C090004D34CE01DF91CF911F910F91FF90EF9022
:10C0A0000C94B5560E949BE4C7010E9430351A8259
:10C0B0008CEA9EE4DF91CF911F910F91FF90EF905A
:10C0C000C6C58FEF8EBD0DB407FEFDCF8EB50895AA
:10C0D0008EBD0DB407FEFDCF089561E0FC018081A7
:10C0E0000C9421FEFC012281322F306A36953CBD32
:10C0F00020FD06C031E0263009F430E0232F01C0D6
:10C1000020E02DBD60E0FC0180810C9421FECF92E7
:10C11000DF92EF92FF920F931F93CF93DF93EC0187
:10C120008B017A010E94C8FE6B01CBDF8B838F3FAE
:10C1300049F40E94C8FE6C197D096D327140A8F364
:10C1400081E144C08E3F11F08FE040C0E114F10462
:10C15000D9F0C70101972FEF2EBDF8014FEF9F01D6
:10C16000201B310B2817390738F40DB407FEFDCF1B
:10C170002EB521934EBDF3CF0DB407FEFDCF2EB5E6
:10C18000F801E80FF91F2083D801E00EF11EC12C41
:10C19000D12CAE15BF0579F08D91ED2DFF27E82745
:10C1A000EE0FFF1FEF56F04B85919491DC2CCC24C1
:10C1B000C826D926EECF85DF082F10E0102F0027E4
:10C1C00080DF082BC016D10631F080E28983CE01D2
:10C1D00084DF80E003C0CE0180DF81E0DF91CF917A
:10C1E0001F910F91FF90EF90DF90CF9008950F93E4
:10C1F0001F93CF93DF93EB010E94C8FE8B0161DF99
:10C200008F3F49F00E94C8FE601B710B6C177D07C1
:10C21000B0F380E001C081E0DF91CF911F910F91D9
:10C220000895CF92DF92FF920F931F93CF93DF93E6
:10C2300000D01F92CDB7DEB76C01F62E29833A836A
:10C240004B835C834FDF6CE271E0C601D0DF8F2D42
:10C2500080643EDF08E110E05C814B813A812981F6
:10C26000DA01C901002E04C0B695A7959795879568
:10C270000A94D2F729833A834B835C8329DF0850E1
:10C28000110929813A814B815C81083F8FEF1807A2
:10C2900039F7FF2029F0E8E0FE1621F08FEF03C008
:10C2A00085E901C087E814DFFCE0FF1201C009DF67
:10C2B00010E007DFF601838387FF04C01F3F11F002
:10C2C0001F5FF7CF0F900F900F900F90DF91CF91DE
:10C2D0001F910F91FF90DF90CF900895BF92CF9262
:10C2E000DF92EF92FF920F931F93CF93DF93EC01B6
:10C2F000B62E1C82198248830E94C8FE8B0161E021
:10C3000088810E94E8FDCE01E8DE60E082E30E94C1
:10C31000E8FD61E083E30E94E8FD61E084E30E94C0
:10C32000E8FD61E085E30E94E8FD61E085E30E94AD
:10C3300021FE85E08A8382E58CBD1DBC6AE0F62E75
:10C340008FEFC6DEFA94E1F720E030E0A90160E06B
:10C35000CE0167DFF82E8B8381E0F81649F00E944A
:10C36000C8FE601B710B613D774070F381E046C0F1
:10C370002AEA31E040E050E068E0CE0152DF82FF7F
:10C3800002C0FC820CC054E0F52E9BDE8B83FA9435
:10C39000E1F78A3A11F082E031C082E08C838C812F
:10C3A000823031F4C12CD12CE12C40E4F42E03C0B6
:10C3B000C12CD12C760120E030E0A90167E3CE0149
:10C3C00030DFA701960169E2CE012BDF8B83882342
:10C3D00049F00E94C8FE601B710B613D774058F325
:10C3E0008AE00CC08C818230B1F420E030E0A901F9
:10C3F0006AE3CE0116DF882329F088E08983CE0125
:10C400006CDE14C05EDE807C803C11F483E08C83A3
:10C4100058DE57DE56DECE0160DE86E08B1518F45E
:10C4200088E1898303C0BA8281E001C080E0DF91A6
:10C43000CF911F910F91FF90EF90DF90CF90BF9021
:10C440000895AF92BF92CF92DF92EF92FF920F9337
:10C450001F93CF93DF93EC016A017B0189018C81EB
:10C46000833039F0F9E0CC0CDD1CEE1CFF1CFA9592
:10C47000D1F773E0B72EE4E0AE2EBA94A70196018F
:10C4800061E1CE01CEDE882311F0A98207C040E031
:10C4900052E0B801CE013BDE81110EC0CE01BB20BF
:10C4A00049F01BDE20E030E0A9016CE0CE01B9DEEE
:10C4B0001982E3CF12DE80E0DF91CF911F910F91BF
:10C4C000FF90EF90DF90CF90BF90AF900895CF9303
:10C4D000DF93EC016EBD20E030E00DB407FEFDCF30
:10C4E000FA01E20FF31F80818EBD0DB407FEFDCF70
:10C4F00081818EBD2E5F3F4F211582E0380769F79D
:10C500000DB407FEFDCF8FEFE3DD8FEFE1DDD9DD69
:10C510008B838F71853031F083E18983CE01DDDD3E
:10C5200080E001C081E0DF91CF9108950F931F93C8
:10C53000CF93DF93EC0189018C81833039F0B9E02E
:10C54000440F551F661F771FBA95D1F79A01AB01AB
:10C5500068E1CE0166DE882311F086E01EC0A801E6
:10C560006EEFCE01B4DF8823C9F068E572E0CE013A
:10C570003EDE182F811102C087E10FC020E030E0BD
:10C58000A9016DE0CE014DDE811106C09ADD811159
:10C5900003C0CE01A2DD05C086E18983CE019DDD09
:10C5A00010E0812FDF91CF911F910F910895FC0131
:10C5B000659175918591949108958091190C909150
:10C5C0001A0CA0911B0CB0911C0C809354139093E7
:10C5D0005513A0935613B09357138091550C909117
:10C5E000560C9093C3138093C21384E690E090930B
:10C5F000560C8093550C0E94C8FE6093B311709343
:10C60000B4118093B5119093B61181E00C9495DC30
:10C6100080E00E9495DC8091541390915513A09175
:10C620005613B09157138093190C90931A0CA09342
:10C630001B0CB0931C0C8091C2139091C313909368
:10C64000560C8093550C0E94C8FE6093B3117093F2
:10C65000B4118093B5119093B6110895AF92BF9223
:10C66000CF92DF92EF92FF920F931F93CF93DF93BE
:10C6700000D01F92CDB7DEB78FE5A82E8CE0B82E84
:10C68000F50160817181828193816093190C7093AF
:10C690001A0C80931B0C90931C0CC12CD12C20E203
:10C6A000E22E21ECF22EC982DA82EB82FC8220E0BB
:10C6B00030E040E752E40F94820539E8C32E33E1BD
:10C6C000D32E7B018C0129EA33E1AE014F5F5F4F2E
:10C6D00061EA73E18DE993E10E9498EF0E9415E40D
:10C6E00082E00E947FE469837A838B839C8329EABA
:10C6F00033E1AE014F5F5F4F61EA73E18DE993E192
:10C700000E94A6F98BE193E552DF9B01AC016981A0
:10C710007A818B819C810F94A20469837A838B83B5
:10C720009C8320E030E040E752E46091190C709166
:10C730001A0C80911B0C90911C0C0F9482057B01AC
:10C740008C0129EA33E1AE014F5F5F4F61EA73E18B
:10C750008DE993E10E9498EF0E9415E420E030E01B
:10C7600040E85EE3F50160817181828193810F94DD
:10C7700050086B017C016093190C70931A0C809324
:10C780001B0C90931C0C8BE193E511DF9B01AC011A
:10C790000F94A2049B01AC0169817A818B819C81F9
:10C7A0000F94A10469837A838B839C8320E030E01B
:10C7B00040E752E4C701B6010F94820549E8C42E50
:10C7C00043E1D42E7B018C0129EA33E1AE014F5FB6
:10C7D0005F4F61EA73E18DE993E10E9498EF0E9457
:10C7E00015E482E00E947FE46093A5137093A61382
:10C7F0008093A7139093A81329EA33E145EA53E104
:10C8000061EA73E18DE993E10E94A6F90F900F9020
:10C810000F900F90DF91CF911F910F91FF90EF90AC
:10C82000DF90CF90BF90AF9008952F923F924F929C
:10C830005F926F927F928F929F92AF92BF92CF92B0
:10C84000DF92EF92FF920F931F93CF93DF9300D06D
:10C8500000D0CDB7DEB71C01FC01E05FFC4A1491AB
:10C860009C01220F331F220F331F3E832D8323563B
:10C870003C4E4901F901108211821282138229EA89
:10C8800033E145EA53E161EA73E18DE993E10E9406
:10C89000A6F98D819E81815E9C4A89DE6B017C01B7
:10C8A000612F772767FD7095872F972F0F941D06AF
:10C8B0002B013C012D813E8128593C4E590120E03D
:10C8C00030E040EC5FE3C701B6010F945008A301CC
:10C8D00092010F945008F5016083718382839383E2
:10C8E0002D813E81295A334F3C832B83F90160818E
:10C8F0007181828193816093190C70931A0C8093DB
:10C900001B0C90931C0C20E030E040E752E40F94A5
:10C910008205E9E8CE2EE3E1DE2E7B018C0124E7DF
:10C9200033E140E753E16CE673E188E693E10E946E
:10C9300098EF0E9415E4F401108211821282138292
:10C9400029EA33E145EA53E161EA73E18DE993E1D4
:10C950000E94A6F92D813E812D5E3C4A3A832983AF
:10C96000C90125DE9058A30192010F945008F501EA
:10C97000608371838283938320E030E040E752E458
:10C980006091190C70911A0C80911B0C90911C0CE9
:10C990000F9482057B018C0124E733E140E753E1EA
:10C9A0006CE673E188E693E10E9498EF0E9415E43B
:10C9B00089819A81FCDD9B01AC010F94A204A30143
:10C9C00092010F945008F5016083718382839383F1
:10C9D00020E030E040E05FE3EB81FC816081718129
:10C9E000828193810F9450086093190C70931A0CF4
:10C9F00080931B0C90931C0C20E030E040E752E445
:10CA00000F9482057B018C0124E733E140E753E179
:10CA10006CE673E188E693E10E9498EF0E9415E4CA
:10CA20008D819E81855D9C4AC2DD0D811E810F56E0
:10CA30001C4EF80120813181428153810F94A20460
:10CA4000F40160837183828393838D819E818D5BEA
:10CA50009C4AADDD2D813E81255C334F7901F80183
:10CA600020813181428153810F94A204F7016083B8
:10CA70007183828393838D819E81895C9C4A97DD3B
:10CA80002D813E81215D334F7901F8012081318173
:10CA9000428153810F94A204F701608371838283E2
:10CAA0009383F40180819181A281B381F501808318
:10CAB0009183A283B3831092190C10921A0C1092D6
:10CAC0001B0C10921C0C0E948EDCF101E257FC4EF4
:10CAD00081E0808326960FB6F894DEBF0FBECDBFEF
:10CAE000DF91CF911F910F91FF90EF90DF90CF904A
:10CAF000BF90AF909F908F907F906F905F904F907E
:10CB00003F902F900895FC012491222341F0309111
:10CB1000C00035FFFCCF2093C6000196F4CF22E081
:10CB200030E08BE397E10C9497DBFC012491222306
:10CB300041F03091C00035FFFCCF2093C600019634
:10CB4000F4CF2AE030E08BE397E10C94EDDA20910A
:10CB5000BD113091BE11243031050CF077C04091E9
:10CB6000BF115091C01160E6649F9001659F300D28
:10CB70001124BC01C90189539E4E0F94260FEFE486
:10CB8000F3E58491882341F09091C00095FFFCCF9C
:10CB90008093C6003196F5CFE091BB13F0E0EE0F25
:10CBA000FF1FE85DFD4F0190F081E02DE45DFE4F39
:10CBB0000190F081E02D8491882341F09091C00094
:10CBC00095FFFCCF8093C6003196F5CF8091BF11C1
:10CBD0009091C01120E6289FF001299FF00D1124AB
:10CBE000E953FE4E8191882339F09091C00095FF62
:10CBF000FCCF8093C600F6CFEEE0F3E58491882366
:10CC000041F09091C00095FFFCCF8093C600319613
:10CC1000F5CF8091C00085FFFCCF8AE08093C600ED
:10CC20008091BF119091C011019664E070E00F9463
:10CC300046099093C0118093BF118091BD119091CE
:10CC4000BE1101969093BE118093BD11089520915D
:10CC5000BD113091BE11243031050CF077C04091E8
:10CC6000BF115091C01160E6649F9001659F300D27
:10CC70001124BC01C90189539E4E0F94860EEFE426
:10CC8000F3E58491882341F09091C00095FFFCCF9B
:10CC90008093C6003196F5CFE091BB13F0E0EE0F24
:10CCA000FF1FE85DFD4F0190F081E02DE45DFE4F38
:10CCB0000190F081E02D8491882341F09091C00093
:10CCC00095FFFCCF8093C6003196F5CF8091BF11C0
:10CCD0009091C01120E6289FF001299FF00D1124AA
:10CCE000E953FE4E8191882339F09091C00095FF61
:10CCF000FCCF8093C600F6CFECE0F3E58491882367
:10CD000041F09091C00095FFFCCF8093C600319612
:10CD1000F5CF8091C00085FFFCCF8AE08093C600EC
:10CD20008091BF119091C011019664E070E00F9462
:10CD300046099093C0118093BF118091BD119091CD
:10CD4000BE1101969093BE118093BD1108959B9AD8
:10CD5000A3980895FCDF40E052EC61E070E08BE3C3
:10CD600097E10E94A5D9E6E0F3E58491882341F09C
:10CD70009091C00095FFFCCF8093C6003196F5CF0F
:10CD80008091C00085FFFCCF8AE08093C6002FE42D
:10CD900033E5F9018491882341F09091C00095FF1B
:10CDA000FCCF8093C6003196F5CF84B780FF20C0BA
:10CDB000A091BB13B0E0AA0FBB1FA85DBD4FED91C2
:10CDC000FC91E25DFE4F0190F081E02D949199235A
:10CDD00041F04091C00045FFFCCF9093C6003196D2
:10CDE000F5CF9091C00095FFFCCF9AE09093C600DC
:10CDF00081FF20C0A091BB13B0E0AA0FBB1FA85DAC
:10CE0000BD4FED91FC91E05DFE4F0190F081E02D72
:10CE10009491992341F04091C00045FFFCCF90933D
:10CE2000C6003196F5CF9091C00095FFFCCF9AE0F7
:10CE30009093C60082FF20C0A091BB13B0E0AA0F60
:10CE4000BB1FA85DBD4FED91FC91EE5CFE4F0190C4
:10CE5000F081E02D9491992341F04091C00045FF6D
:10CE6000FCCF9093C6003196F5CF9091C00095FF0E
:10CE7000FCCF9AE09093C60083FF20C0A091BB1323
:10CE8000B0E0AA0FBB1FA85DBD4FED91FC91EC5C1B
:10CE9000FE4F0190F081E02D9491992341F0409153
:10CEA000C00045FFFCCF9093C6003196F5CF90911E
:10CEB000C00095FFFCCF9AE09093C60085FF20C08C
:10CEC000A091BB13B0E0AA0FBB1FA85DBD4FED91B1
:10CED000FC91EA5CFE4F0190F081E02D8491882363
:10CEE00041F09091C00095FFFCCF8093C600319631
:10CEF000F5CF8091C00085FFFCCF8AE08093C6000B
:10CF000014BEF9018491EFE4F3E5882349F0909190
:10CF1000C00095FFFCCF8093C60031968491F5CF79
:10CF2000A091BB13B0E0AA0FBB1FA85DBD4FED9150
:10CF3000FC91E65CFE4F0190F081E02D8491882306
:10CF400041F09091C00095FFFCCF8093C6003196D0
:10CF5000F5CFE1EFF2E58491882341F09091C00094
:10CF600095FFFCCF8093C6003196F5CFA091BB13FF
:10CF7000B0E0AA0FBB1FA85DBD4FED91FC91E85C2E
:10CF8000FE4F0190F081E02D4491442341F05091F7
:10CF9000C00055FFFCCF4093C6003196F5CFEAEDB7
:10CFA000F2E58491882341F09091C00095FFFCCF79
:10CFB0008093C6003196F5CF8091C00085FFFCCFED
:10CFC0008AE08093C600EFECF2E58491882341F07B
:10CFD0009091C00095FFFCCF8093C6003196F5CFAD
:10CFE000E3ECF2E58491882341F09091C00095FF35
:10CFF000FCCF8093C6003196F5CF8091C00085FFAD
:10D00000FCCF8AE08093C600F9012491EFE4F3E5B8
:10D01000222349F08091C00085FFFCCF2093C600F9
:10D0200031962491F5CFE091BB13F0E0EE0FFF1F96
:10D03000E85DFD4F0190F081E02DE45CFE4F019032
:10D04000F081E02D8491882341F09091C00095FFFC
:10D05000FCCF8093C6003196F5CF0E9496E74AE058
:10D0600050E0BC018BE397E10E94C1DAE091BB1371
:10D07000F0E0EE0FFF1FE85DFD4F0190F081E02D25
:10D08000E25CFE4F0190F081E02D8491882341F015
:10D090009091C00095FFFCCF8093C6003196F5CFEC
:10D0A0004AE050E060ED74E08BE397E10E94C1DA62
:10D0B0008091C00085FFFCCF8AE08093C60010926B
:10D0C000C3111092C4111092C5111092C6110E9482
:10D0D000C8D70E949AD30E949A400E9448EF0E94AB
:10D0E00087E60E94C9AD8091000186FD29C0FFEF4F
:10D0F00023ED80E3F15020408040E1F700C00000C4
:10D100008091000186FD25C080910101846080939B
:10D1100001019FB7F894809102018460809302011D
:10D120009FBF0E9439AB8091000186FFFCCF9FB763
:10D13000F894809102018B7F809302019FBF09C008
:10D140009FEFE3EDF0E39150E040F040E1F700C0E5
:10D150000000159808958091B7119091B81160E082
:10D1600070E001960D94DD0B8091B7119091B8118C
:10D170004AE050E060E070E001960D94450D682FA4
:10D18000772767FD70952091C1113091C21140E65B
:10D19000429FC001439F900D112489539E4E0F94CE
:10D1A000120F9093B8118093B71121E0892B09F4E5
:10D1B00020E0822F08950E94C8FE6093B3117093FF
:10D1C000B4118093B5119093B61108950E94C8FED2
:10D1D0006093B3117093B4118093B5119093B6110D
:10D1E000E091C111F091C211ED53FE4E8081811189
:10D1F00021C0E091BB13F0E0EE0FFF1FE85DFD4F93
:10D200000190F081E02DE05CFE4F0190F081E02D77
:10D210008491882341F09091C00095FFFCCF8093CA
:10D22000C6003196F5CF8091C00085FFFCCF8AE023
:10D230008093C60008958BE397E10E94F7D9E091AF
:10D24000BB13F0E0EE0FFF1FE85DFD4F0190F08192
:10D25000E02DE059FE4F0190F081E02D849188236C
:10D2600041F09091C00095FFFCCF8093C6003196AD
:10D27000F5CF40914C1350914D1360914E13709126
:10D280004F134F5F5F4F6F4F7F4F2AE030E08BE3CC
:10D2900097E10E9496DA8091C00085FFFCCF8AE07A
:10D2A0008093C60093CF8F929F92AF92BF92CF92FE
:10D2B000DF92EF92FF920F931F93CF93DF9348E299
:10D2C000E42E4EE0F42E0DE913E1C8E6D3E154EC70
:10D2D000C52E53E1D52EF70181917F0150DF8823C0
:10D2E00011F139DF4B015C01F6018081811103C02E
:10D2F0006091471301C061E070E080E090E00F941E
:10D300001D06F80120813181428153810F9450081C
:10D310009B01AC01C501B4010F94A2046883798319
:10D320008A839B8309C0F80180819181A281B381A6
:10D3300088839983AA83BB830C5F1F4F2496FFEFDA
:10D34000CF1ADF0A8CE2E8168EE0F80621F686E4B2
:10D3500016DF8823D1F0FFDE6B017C016093581348
:10D360007093591380935A1390935B1320E030E02D
:10D37000A9010F947E07181644F4C092190CD0929C
:10D380001A0CE0921B0CF0921C0CDF91CF911F91B4
:10D390000F91FF90EF90DF90CF90BF90AF909F9054
:10D3A0008F90089580DF89E4EADE882351F0D3DE90
:10D3B00060935C1370935D1380935E1390935F137F
:10D3C00008C010925C1310925D1310925E131092BD
:10D3D0005F138AE4D4DE882351F0BDDE60936013CE
:10D3E0007093611380936213909363130895109266
:10D3F00060131092611310926213109263130895D8
:10D40000CF92DF92EF92FF92CF93DF93EC01C09027
:10D410003B0CD0903C0CE0903D0CF0903E0CA701F2
:10D420009601688179818A819B810F947B0587FFB2
:10D4300004C0C882D982EA82FB82C0903F0CD0909F
:10D44000400CE090410CF090420CA70196016C81D9
:10D450007D818E819F810F947B0587FF04C0CC82E4
:10D46000DD82EE82FF8220E030E0A9016091430C72
:10D470007091440C8091450C9091460C0F94A2043D
:10D480006B017C019B01AC01688579858A859B8550
:10D490000F947B0587FF04C0C886D986EA86FB8681
:10D4A000C0902F0CD090300CE090310CF090320CEA
:10D4B000A7019601688179818A819B810F947E07FB
:10D4C000181624F4C882D982EA82FB82C090330CF9
:10D4D000D090340CE090350CF090360CA7019601FA
:10D4E0006C817D818E819F810F947E07181624F4B4
:10D4F000CC82DD82EE82FF82C090370CD090380C57
:10D50000E090390CF0903A0CA70196016885798576
:10D510008A859B850F947E07181624F4C886D986C1
:10D52000EA86FB86DF91CF91FF90EF90DF90CF905E
:10D5300008952F923F924F925F926F927F928F92B7
:10D540009F92AF92BF92CF92DF92EF92FF920F9392
:10D550001F93CF93DF93CDB7DEB7AF970FB6F89495
:10D56000DEBF0FBECDBF9BA38AA37DA36CA35FA329
:10D570004EA339A728A71BA70AA7E98ADC016D914A
:10D580007D918D919C9120919D1330919E1340919E
:10D590009F135091A013ECA1FDA180809180A280E7
:10D5A000B3804090A1135090A2136090A313709089
:10D5B000A413AEA1BFA1ED90FD900D911C91EA8A3C
:10D5C000FB8A0C8B1D8BE090A513F090A6130091A5
:10D5D000A7131091A813EE8EFF8E08A319A3E09154
:10D5E0000C18E11135C0AAA5BBA5ED90FD900D91D9
:10D5F0001C91FE0171966F0128A539A54EA15FA16E
:10D600006CA17DA18AA19BA10E9498EF80E1E8E630
:10D61000F3E1ADE9B3E101900D928A95E1F7AF96A0
:10D620000FB6F894DEBF0FBECDBFDF91CF911F9133
:10D630000F91FF90EF90DF90CF90BF90AF909F90B1
:10D640008F907F906F905F904F903F902F900895B4
:10D650000F94A1046E8B7F8B888F998F20E030E030
:10D66000A9010F947E07CE88DF88E88CF98C181604
:10D6700024F0F7FAF094F7F8F094A3019201C501B1
:10D68000B4010F94A1046A8F7B8F8C8F9D8F20E053
:10D6900030E0A9010F947E078A8C9B8CAC8CBD8CEA
:10D6A000181624F0B7FAB094B7F8B0942E8D3F8DC9
:10D6B00048A159A16A897B898C899D890F94A1040D
:10D6C0002B013C01A5019401C701B6010F94A204EE
:10D6D0006B017C0120E030E0A901C301B2010F948D
:10D6E0007E07A301920118160CF05058C701B6012D
:10D6F0000F94A2046B017C0120E030E0A9010F949B
:10D700007E0718160CF06FCF20E030E040EF51E4B8
:10D71000C701B6010F9482050F9458060F94EA05CD
:10D720007B8B6A8B8B01623071050CF45CCF20918E
:10D73000A9133091AA134091AB135091AC13A8A533
:10D74000B9A56D917D918D919C910F94A1046E8FDF
:10D750007F8F88A399A322242394312C780100275A
:10D76000F7FC0095102FECA6FDA60EA71FA7B10190
:10D77000882777FD8095982F0F941D066B017C01FB
:10D780006CA57DA58EA59FA50F941D069B01AC01E0
:10D79000C701B6010F9482056B017C01AAA5BBA548
:10D7A0008D909D90AD90BC902E8D3F8D48A159A13C
:10D7B0000F9450089B01AC016091A9137091AA13BA
:10D7C0008091AB139091AC130F94A20469837A8378
:10D7D0008B839C83A3019201C701B6010F9450086B
:10D7E0009B01AC016091A5137091A6138091A713C2
:10D7F0009091A8130F94A2046D837E838F839887E2
:10D800002A8D3B8D4C8D5D8DC701B6010F9450085C
:10D810009B01AC016091A1137091A2138091A3139D
:10D820009091A4130F94A20469877A878B879C87B1
:10D830002E893F89488D598DC701B6010F94500834
:10D840009B01AC0160919D1370919E1380919F1379
:10D850009091A0130F94A2046D877E878F87988B79
:10D86000FE0171966F01850174019E012F5F3F4F8C
:10D87000AE014B5F5F4FBE01675F7F4FCE010D96DC
:10D880000E9498EFFFEF2F1A3F0AEA88FB882E14B8
:10D890003F0409F06CCFA7CEEF920F931F93CF9365
:10D8A000DF9300D01F92CDB7DEB788E693E1A8DD05
:10D8B0000E94C8FE6093B3117093B4118093B511A8
:10D8C0009093B611209168133091691340916A13B7
:10D8D00050916B1360919D1370919E1380919F13D3
:10D8E0009091A0130F947B05E090891381117CC067
:10D8F00020916C1330916D1340916E1350916F1302
:10D900006091A1137091A2138091A3139091A4131D
:10D910000F947B05811168C020E030E040E752E4BD
:10D920006091190C70911A0C80911B0C90911C0C39
:10D930000F94820569837A838B839C838E010F5FAA
:10D940001F4F24E733E140E753E16CE673E188E6DB
:10D9500093E1EFDD8091681390916913A0916A13B0
:10D96000B0916B1380939D1390939E13A0939F137C
:10D97000B093A01380916C1390916D13A0916E13CE
:10D98000B0916F138093A1139093A213A093A3134C
:10D99000B093A4138091701390917113A09172139E
:10D9A000B09173138093A5139093A613A093A7131C
:10D9B000B093A8138091741390917513A09176136E
:10D9C000B09177138093A9139093AA13A093AB13EC
:10D9D000B093AC130F900F900F900F90DF91CF91F9
:10D9E0001F910F91EF9008956091550C7091560C16
:10D9F000882777FD8095982F0F941D062091190C8C
:10DA000030911A0C40911B0C50911C0C0F94500833
:10DA100020E030E040E752E40F94820520E030E05F
:10DA200048EC52E485CFCF92DF92EF92FF92CF93F2
:10DA3000C62FE0918913F0E0882309F4C2C0DF010A
:10DA4000AB57BC4E8C91811196C180919D139091E2
:10DA50009E13A0919F13B091A0138093681390938D
:10DA60006913A0936A13B0936B138091A1139091E3
:10DA7000A213A091A313B091A41380936C1390935D
:10DA80006D13A0936E13B0936F138091A5139091B3
:10DA9000A613A091A713B091A8138093701390932D
:10DAA0007113A0937213B0937313C090A913D09005
:10DAB000AA13E090AB13F090AC13C0927413D09201
:10DAC0007513E0927613F0927713EE0FFF1FEE0FAF
:10DAD000FF1FE95BF34F208131814281538166232F
:10DAE00049F06091270C7091280C8091290C90913D
:10DAF0002A0C08C060912B0C70912C0C80912D0C7D
:10DB000090912E0C0F9482059B01AC01C701B601C8
:10DB10000F94A2046093A9137093AA138093AB137C
:10DB20009093AC1389EA93E10E947AFAC090190CA1
:10DB3000D0901A0CE0901B0CF0901C0C20E030E010
:10DB400040E752E46091230C7091240C8091250CE5
:10DB50009091260C0F9450086093190C70931A0C36
:10DB600080931B0C90931C0CE0918913F0E0EB5711
:10DB7000FC4E81E0808390DE2091811330918213EE
:10DB800040918313509184136091A5137091A61353
:10DB90008091A7139091A8130F94A1046093A513EB
:10DBA0007093A6138093A7139093A81329EA33E1E7
:10DBB00045EA53E161EA73E18DE993E10E94A6F938
:10DBC000D1C0EB57FC4E8081882309F4D4C08091EA
:10DBD0009D1390919E13A0919F13B091A0138093D9
:10DBE000681390936913A0936A13B0936B13809199
:10DBF000A1139091A213A091A313B091A4138093A9
:10DC00006C1390936D13A0936E13B0936F13609188
:10DC1000A5137091A6138091A7139091A8136093F8
:10DC20007013709371138093721390937313C09059
:10DC3000A913D090AA13E090AB13F090AC13C0924C
:10DC40007413D0927513E0927613F09277132091AB
:10DC500081133091821340918313509184130F9458
:10DC6000A2046093A5137093A6138093A7139093B7
:10DC7000A81329EA33E145EA53E161EA73E18DE94A
:10DC800093E10E94A6F9F0908913CC2389F02091AA
:10DC9000791330917A1340917B1350917C136091EA
:10DCA000270C7091280C8091290C90912A0C10C09F
:10DCB00020917D1330917E1340917F1350918013FA
:10DCC00060912B0C70912C0C80912D0C90912E0C4E
:10DCD0000F94A20424E0F29EF0011124E95BF34FBB
:10DCE00020813181428153810F9482059B01AC01D7
:10DCF0006091A9137091AA138091AB139091AC130A
:10DD00000F94A1046093A9137093AA138093AB138B
:10DD10009093AC1389EA93E10E947AFAC090190CAF
:10DD2000D0901A0CE0901B0CF0901C0C20E030E01E
:10DD300040E752E460911F0C7091200C8091210CFF
:10DD40009091220C0F9450086093190C70931A0C48
:10DD500080931B0C90931C0CE0918913F0E0EB571F
:10DD6000FC4E108299DDC092190CD0921A0CE092F0
:10DD70001B0CF0921C0CCF91FF90EF90DF90CF9096
:10DD80000895AF92BF92CF92DF92EF92FF920F93DE
:10DD90001F93CF93DF93D82F20916013309161139D
:10DDA000409162135091631360915C1370915D1305
:10DDB00080915E1390915F130F948B07C62F172FDE
:10DDC000082FF92E6091550C7091560C882777FD1D
:10DDD0008095982F0F941D062091190C30911A0CE4
:10DDE00040911B0C50911C0C0F94500820E030E027
:10DDF00040E752E40F94820520E030E048EC52E422
:10DE00000F948205209189132F93DF93FF920F9334
:10DE10001F93CF935B016C01E2E0EE2E01E020E066
:10DE20004CE553E168E673E18DE993E10E94984F78
:10DE30008091681390916913A0916A13B0916B134C
:10DE400080939D1390939E13A0939F13B093A01360
:10DE500080916C1390916D13A0916E13B0916F131C
:10DE60008093A1139093A213A093A313B093A41330
:10DE70008091701390917113A0917213B0917313EC
:10DE80008093A5139093A613A093A713B093A81300
:10DE90008091741390917513A0917613B0917713BC
:10DEA0008093A9139093AA13A093AB13B093AC13D0
:10DEB0000E94C8FE6093B3117093B4118093B511A2
:10DEC0009093B6110F900F900F900F900F900F90AE
:10DED000DF91CF911F910F91FF90EF90DF90CF9046
:10DEE000BF90AF900895F8940E945B41179A1092EA
:10DEF0008E13169A10928F13149A60E087E40E9492
:10DF0000E8FDE5E5F3E58491882341F09091C000B8
:10DF100095FFFCCF8093C6003196F5CFE091BB13FF
:10DF2000F0E0EE0FFF1FE85DFD4F0190F081E02D66
:10DF3000E459FE4F0190F081E02D8491882341F057
:10DF40009091C00095FFFCCF8093C6003196F5CF2D
:10DF50008091C00085FFFCCF8AE08093C600E091ED
:10DF6000BB13F0E0EE0FFF1FE85DFD4F0190F08165
:10DF7000E02DE653FF4F808191810E9462AD78943D
:10DF8000C6E0D0E02197209749F068EC70E080E08F
:10DF900090E00E94F7FE0E9404AEF4CFF894FFCF09
:10DFA0000E945B418091A111811151C081E0809359
:10DFB000A11180914C1390914D13A0914E13B091EB
:10DFC0004F138093481390934913A0934A13B0932F
:10DFD0004B13E5E5F3E58491882341F09091C0006F
:10DFE00095FFFCCF8093C6003196F5CFE091BB132F
:10DFF000F0E0EE0FFF1FE85DFD4F0190F081E02D96
:10E00000E259FE4F0190F081E02D8491882341F088
:10E010009091C00095FFFCCF8093C6003196F5CF5C
:10E020008091C00085FFFCCF8AE08093C600E0911C
:10E03000BB13F0E0EE0FFF1FE85DFD4F0190F08194
:10E04000E02DE453FF4F808191810C946BAB0895D8
:10E050008091A1110895CF93DF93EC0180918913F2
:10E060008093A21184E58BD8811102C080E0B7C0F3
:10E0700072D80F94EF056093A2116623B9F3EFE411
:10E08000F3E58491882341F09091C00095FFFCCF87
:10E090008093C6003196F5CFCD36D10509F454C032
:10E0A000BCF4C836D10561F1C936D10509F087C085
:10E0B000E091BB13F0E0EE0FFF1FE85DFD4F019014
:10E0C000F081E02DEC5AFE4F0190F081E02D38C038
:10E0D000CA3DD10509F451C0CD3DD10509F06FC04D
:10E0E000E091BB13F0E0EE0FFF1FE85DFD4F0190E4
:10E0F000F081E02DE65AFE4F0190F081E02D5CC0EA
:10E10000E091BB13F0E0EE0FFF1FE85DFD4F0190C3
:10E11000F081E02DEE5AFE4F0190F081E02D8191CB
:10E12000882309F44CC09091C00095FFFCCF8093E8
:10E13000C600F5CF9091C00095FFFCCF8093C6003C
:10E1400081918111F7CF3BC0E091BB13F0E0EE0F5E
:10E15000FF1FE85DFD4F0190F081E02DE25AFE4F78
:10E160000190F081E02D8191882349F19091C000C8
:10E1700095FFFCCF8093C600F6CFE091BB13F0E093
:10E18000EE0FFF1FE85DFD4F0190F081E02DE85A92
:10E19000FE4F0190F081E02D8191882381F09091D4
:10E1A000C00095FFFCCF8093C600F6CF9091C000D1
:10E1B00095FFFCCF8093C60081918111F7CF40E09D
:10E1C00050E06091A2118BE397E10E94F8DA809110
:10E1D000C00085FFFCCF8AE08093C60081E0DF911C
:10E1E000CF9108954F925F926F927F928F929F92FC
:10E1F000AF92BF92CF92DF92EF92FF92CF93DF93D5
:10E2000000D01F92CDB7DEB72B013C0129833A83A2
:10E210004B835C838DEE9FE00F9466118F3F01F579
:10E220008EEE9FE00F9466118F3FD1F48FEE9FE04A
:10E230000F9466118F3FA1F480EF9FE00F94661159
:10E240008F3F71F440E050E0BA018DEE9FE00F94F3
:10E25000731140E050E0BA0181EF9FE00F94731119
:10E2600081EF9FE00F946E114B015C018DEE9FE0FA
:10E270000F946E116B017C0169817A818B819C8185
:10E280002CE330E040E050E00F945909C20ED31E59
:10E29000E41EF51EB701A6018DEE9FE00F947311E9
:10E2A000C301B20128EE33E040E050E00F94590979
:10E2B000BA01A901480D591D6A1D7B1D81EF9FE020
:10E2C0000F9473111092B7131092B8131092B913E0
:10E2D0001092BA130F900F900F900F90DF91CF9183
:10E2E000FF90EF90DF90CF90BF90AF909F908F9076
:10E2F0007F906F905F904F9008952F923F924F9232
:10E300005F926F927F928F929F92AF92BF92CF92C5
:10E31000DF92EF92FF920F931F93CF93DF93CDB7CE
:10E32000DEB76E970FB6F894DEBF0FBECDBF30E6F6
:10E33000B32E44E0E42EF12C5AE0952E6AE0C62E6E
:10E34000D12CAA24A3948091BC179091BD17209141
:10E35000BE173091BF17821B930B8F779927892B9C
:10E3600039F08091BD119091BE1104970CF448C012
:10E370008091D013882309F4E7C38091BA1190915A
:10E38000BB11892B09F0E0C38091BD119091BE11A2
:10E39000892B11F410929F11F8EE2F2EF3E03F2EEF
:10E3A000412C512CACE38A2E912CA12CB12C8E0146
:10E3B0000F5F1F4FE0E66E2E7724739440916B162B
:10E3C00050916C1660916D1670916E168091631667
:10E3D00090916416A0916516B0916616481759077A
:10E3E0006A077B0708F0B0C38091BD119091BE1100
:10E3F00004970CF0A9C380919F118111A5C36FC22E
:10E400008BE397E10E94DBD98093BC112091BA1174
:10E410003091BB118A3061F08D3051F08A3321F494
:10E420009091B911992321F02F3531050CF450C189
:10E430002115310509F46AC18091BF119091C01175
:10E44000B89E3001B99E700C1124F301E20FF31F46
:10E45000E953FE4E10822091B911211134C110925E
:10E46000B911FC01ED53FE4E1082830109531E4E7B
:10E470006EE470E0C8010F94120F0097F1F19093D1
:10E48000B8118093B711801B910B860D971D4AE040
:10E4900050E060E070E088539E4E0F94450D60930D
:10E4A00050137093511380935213909353134090D1
:10E4B0004C1350904D1360904E1370904F132FEFEC
:10E4C000421A520A620A720A0091BF111091C011D9
:10E4D000641575058605970509F41BC1B09EC0013A
:10E4E000B19E900D11246AEB72E589539E4E0F94F4
:10E4F000BD0E892B09F00DC1B8C16AE270E0C801F8
:10E500000F94120F892B09F451C0E5E5F3E58491CE
:10E51000882341F09091C00095FFFCCF8093C60006
:10E520003196F5CFE091BB13F0E0EE0FFF1FE85DF1
:10E53000FD4F0190F081E02DE65BFE4F0190F081F0
:10E54000E02D8491882341F09091C00095FFFCCF8D
:10E550008093C6003196F5CF40914C1350914D13E6
:10E5600060914E1370914F132AE030E08BE397E1F6
:10E570000E9496DA8091C00085FFFCCF8AE08093EC
:10E58000C6001092BB111092BA11DEC280915013D6
:10E5900090915113A0915213B091531380934C1347
:10E5A00090934D13A0934E13B0934F136090BF11EF
:10E5B0007090C011B69C8001B79C100D11240953B6
:10E5C0001E4E67E470E0C8010F94120F009709F423
:10E5D00056C09093B8118093B7112091D013211198
:10E5E00006C0D092BF13C092BE13A092C113801B6D
:10E5F000910BB69C9001B79C300D1124820F931F94
:10E6000060E070E088539E4E0F94DD0B0F94EA0596
:10E6100064307105A0F58091A111882381F1E0910A
:10E62000BB13F0E0EE0FFF1FE85DFD4F0190F0819E
:10E63000E02DE259FE4F0190F081E02D8491882376
:10E6400041F09091C00095FFFCCF8093C6003196B9
:10E65000F5CF8091C00085FFFCCF9092C600E0917D
:10E66000BB13F0E0EE0FFF1FE85DFD4F0190F0815E
:10E67000E02DE453FF4F808191810E946BAB0091AC
:10E68000BF111091C011B09EC001B19E900D112418
:10E6900069E97DE089539E4E0F941D0F892B09F483
:10E6A00022DCC8010196B7010F9446099093C0116E
:10E6B0008093BF118091BD119091BE1101969093EE
:10E6C000BE118093BD111092BB111092BA113BCEB6
:10E6D0008B3311F4A092B9119091B911911133CEED
:10E6E0004091BF115091C011B9016F5F7F4F70937E
:10E6F000BB116093BA11B49EF001B59EF00D1124C8
:10E70000E20FF31FE953FE4E80831DCE1092B91124
:10E710001BC2B09E3001B19E700C1124C3018953FD
:10E720009E4E1C016AE270E00F94120F009709F0F0
:10E730003FC0E5E5F3E58491882341F09091C00066
:10E7400095FFFCCF8093C6003196F5CFE091BB13C7
:10E75000F0E0EE0FFF1FE85DFD4F0190F081E02D2E
:10E76000E85BFE4F0190F081E02D8491882341F019
:10E770009091C00095FFFCCF8093C6003196F5CFF5
:10E7800040914C1350914D1360914E1370914F1363
:10E790002AE030E08BE397E10E9496DA8091C00096
:10E7A00085FFFCCF8AE08093C6000E941B69E9CEFA
:10E7B00020E010E0F301E20FF11DE953FE4E30813D
:10E7C0003A3219F02F5F1327F5CF9093B811809349
:10E7D000B71182199309860D971D60E070E0885388
:10E7E0009E4E0F94DD0B0F94EA05212F30E0261783
:10E7F000370709F4CBCEE5E5F3E58491882341F0B2
:10E800009091C00095FFFCCF8093C6003196F5CF64
:10E81000E091BB13F0E0EE0FFF1FE85DFD4F0190AC
:10E82000F081E02DEA5BFE4F0190F081E02D8491B4
:10E83000882341F09091C00095FFFCCF8093C600E3
:10E840003196F5CF40914C1350914D1360914E137A
:10E8500070914F132AE030E08BE397E10E9496DA43
:10E860008091C00085FFFCCF9DCFE5E5F3E5849165
:10E87000882341F09091C00095FFFCCF8093C600A3
:10E880003196F5CFE091BB13F0E0EE0FFF1FE85D8E
:10E89000FD4F0190F081E02DEC5BFE4F0190F08187
:10E8A000E02D8491882341F09091C00095FFFCCF2A
:10E8B0008093C6003196F5CF40914C1350914D1383
:10E8C00060914E1370914F132AE030E08BE397E193
:10E8D0000E9496DA8091C00085FFFCCF63CF8091C3
:10E8E000BE159091BF15A091C015B091C115809330
:10E8F0006B1690936C16A0936D16B0936E1686EB04
:10E9000095E10E948433482F8093BC118A30B9F07E
:10E910004D30A9F0433229F42091B911222379F026
:10E9200002C04A33C9F32091BA113091BB112F357F
:10E9300031052CF48F3F5FEF950709F0E7C0409158
:10E940006B1650916C1660916D1670916E168091D9
:10E95000631690916416A0916516B09166164817DB
:10E9600059076A077B0708F497C0E091BB13F0E0F2
:10E97000EE0FFF1FE85DFD4F0190F081E02DE45B9D
:10E98000FE4F0190F081E02D8491882341F0909119
:10E99000C00095FFFCCF8093C6003196F5CF8091E3
:10E9A000C00085FFFCCF8AE08093C6000E94C8FEAD
:10E9B0006093A7117093A8118093A9119093AA1145
:10E9C000C090AB11D090AC11E090AD11F090AE11B1
:10E9D0006C197D098E099F09A20191010F945909B3
:10E9E00069017A016091B7137091B8138091B913DE
:10E9F0009091BA13F7DBC701B601A50194010F94FA
:10EA00005909CA01B901A50194010F9459097F93CD
:10EA10006F93C701B60120E13EE040E050E00F9463
:10EA200059093F932F93A6EAB2E5BF93AF931F9383
:10EA30000F930F944A0FEFE4F3E584910FB6F89427
:10EA4000DEBF0FBECDBF882349F09091C00095FF77
:10EA5000FCCF8093C60031968491F5CFF801819167
:10EA6000882339F09091C00095FFFCCF8093C600B9
:10EA7000F6CF8091C00085FFFCCF3AE03093C6000E
:10EA8000C8010E945EAB8EEC93E10E940A6061E0D7
:10EA90008EEC93E10E94CD598091BC11833211F428
:10EAA00070929F112091BA113091BB11211531053F
:10EAB00009F42CCE8091BF119091C011689EF00195
:10EAC000699EF00D1124E20FF31FE953FE4E1082F0
:10EAD000FC01ED53FE4E70822091BD113091BE11AC
:10EAE0002F5F3F4F3093BE112093BD11019664E01C
:10EAF00070E00F9446099093C0118093BF1110925B
:10EB0000B9111092BB111092BA1158CC4B3311F4B9
:10EB10007092B9114091B91141114CCC4091BF1183
:10EB20005091C011B9016F5F7F4F7093BB1160931B
:10EB3000BA11649EF001659EF00D1124E20FF31FDF
:10EB4000E953FE4E80833ACC6E960FB6F894DEBF42
:10EB50000FBECDBFDF91CF911F910F91FF90EF902E
:10EB6000DF90CF90BF90AF909F908F907F906F90ED
:10EB70005F904F903F902F900895CF92DF92EF9249
:10EB8000FF920F931F93CF93C82F8091BD11909147
:10EB9000BE1103970CF4B1DB0E94C8FE0091AF11C7
:10EBA0001091B0112091B1113091B211C090B311F8
:10EBB000D090B411E090B511F090B6116C197D09A8
:10EBC0008E099F09061717072807390728F4012B14
:10EBD000022B032B09F087D94091150C5091160C8C
:10EBE0006091170C7091180C452B462B472B19F18F
:10EBF0000E94C8FE0091B3111091B4112091B5117B
:10EC00003091B611601B710B820B930B0091150CA8
:10EC10001091160C2091170C3091180C061717073D
:10EC20002807390740F49091D2188091D118981391
:10EC300002C0CC2349F0CF911F910F91FF90EF902C
:10EC4000DF90CF900C947CEF179A10928E13169A47
:10EC500010928F13149AEFCFCF92DF92EF92FF9220
:10EC60002091AD132223F1F020E030E040E05FE39B
:10EC70000F9450086B017C0120E030E0A9010F9453
:10EC80007B05882379F0A7019601C701B6010F948F
:10EC900050082BED3FE049E450E40F9450089B01ED
:10ECA000AC0104C020E030E040E85FE360E070E0E9
:10ECB00080E89FE30F948205FF90EF90DF90CF9064
:10ECC000089560914B0C70914C0C80914D0C90917B
:10ECD0004E0CC2DF6093470C7093480C8093490C34
:10ECE00090934A0C08952F923F924F925F926F92A9
:10ECF0007F928F929F92AF92BF92CF92DF92EF92CC
:10ED0000FF920F931F93CF93DF93CDB7DEB7C3541A
:10ED1000D1090FB6F894DEBF0FBECDBF81E40E94CB
:10ED2000BF68882309F455C082E70E94BF68882322
:10ED3000A9F0EEE9FDE08191882339F09091C000BF
:10ED400095FFFCCF8093C600F6CF8091C00085FF71
:10ED5000FCCF8AE08093C6000C94349386E70E942F
:10ED6000BF688823A9F0E4EAFDE08191882339F0A7
:10ED70009091C00095FFFCCF8093C600F6CF8091A4
:10ED8000C00085FFFCCF8AE08093C6000C943493CA
:10ED900087E60E94BF68882321F00E9439AB0C945B
:10EDA00034938AE70E94BF68882341F060E070E0F6
:10EDB00088EF9FE00E94A9A60C9434938CE60E94F1
:10EDC000BF68882311F40C9434930E94D0A60C944D
:10EDD000349387E40E94BF68882309F47CC50E94AD
:10EDE000AB680F94EA056135710509F4BDC34CF5B4
:10EDF0006430710509F4C8C054F46230710509F437
:10EE0000ABC00CF0B5C077FF4FC00C9434936B309F
:10EE1000710509F40DC15CF46A30710511F00C94B0
:10EE2000349360E081E00E94136D0C9434936C3154
:10EE3000710509F403C16035710509F492C10C94A0
:10EE400034936635710509F4EBC49CF463357105A0
:10EE500009F487C40CF441C46435710509F4D3C4C2
:10EE60006535710511F00C9434930E942ACB0C94F3
:10EE700034936A35710509F4DAC464F467357105B1
:10EE800011F00C94349361E087EF9FE00F947B11B5
:10EE90000C9434936B35710509F4CDC46C35710550
:10EEA00009F4CEC40C9434938091A11181110C9477
:10EEB00034930E9453696091B7137091B813809195
:10EEC000B9139091BA130F941B066B017C0120912A
:10EED000A9133091AA134091AB135091AC136091D8
:10EEE00074137091751380917613909177130F942A
:10EEF000A10420E030E048EC52E40F9450089B015C
:10EF0000AC01C701B6010F94A2040F94EF05609302
:10EF1000B7137093B8138093B9139093BA13809179
:10EF200086138823A9F088E50E94BF68811110C06C
:10EF300089E50E94BF6881110BC08AE50E94BF6805
:10EF4000811106C085E40E94BF6881110C9437933B
:10EF50000E944C6C0C9434938091A11181110C94FB
:10EF600034930E94D26981E00E94C16E0C94349364
:10EF70008091A11181110C9434930E94D26980E098
:10EF80000E94C16E0C943493E091BB13F0E0EE0F3D
:10EF9000FF1FE85DFD4F0190F081E02DE054FF4F31
:10EFA000808191810E946BAB80E50E94BF688823BD
:10EFB00039F00E94AB680F94EF054B015C0103C070
:10EFC000812C912C540183E50E94BF68882361F055
:10EFD0000E94AB6820E030E04AE754E40F94500808
:10EFE0000F94EF054B015C010E9415E40E94C8FEDE
:10EFF0006B017C01C80CD91CEA1CFB1C0E94C8FEDA
:10F000006093B3117093B4118093B5119093B611BE
:10F010000E94C8FE6C157D058E059F0510F00C94AE
:10F0200034930E941A4780E0A8DD0E9404AEF0CF1E
:10F0300060E080E00E94136D0C9434931092C01332
:10F0400010920C188091190C90911A0CA0911B0C25
:10F05000B0911C0C8093541390935513A0935613A6
:10F06000B09357138091550C9091560C9093C31305
:10F070008093C21384E690E09093560C8093550CD5
:10F080000E94C8FE6093B3117093B4118093B511C0
:10F090009093B61181E00E9495DC80919D13909130
:10F0A0009E13A0919F13B091A01380936813909327
:10F0B0006913A0936A13B0936B138091A11390917D
:10F0C000A213A091A313B091A41380936C139093F7
:10F0D0006D13A0936E13B0936F138091A51390914D
:10F0E000A613A091A713B091A813809370139093C7
:10F0F0007113A0937213B09373138091A91390911D
:10F10000AA13A091AB13B091AC1380937413909396
:10F110007513A0937613B09377131092190C109275
:10F120001A0C10921B0C10921C0C88E50E94BF68F0
:10F13000882311F090E00AC089E50E94BF68811120
:10F14000F9CF8AE50E94BF6891E0982790931D0C43
:10F15000992311F40C94669381E08093C0130C946E
:10F16000C5948091D01381110FC081E08093B213B8
:10F1700081E090E09093B1138093B01383E190E02D
:10F180009093AF138093AE1380918E13882341F038
:10F1900080918F13882321F08091901381110AC0F0
:10F1A0008EE992E50E9427668AE992E50E94276629
:10F1B0000C9434938CE098E10E94ADE780E090E0FD
:10F1C000A0E4B1E480939D1390939E13A0939F13AA
:10F1D000B093A01380E090E0A0E4B0EC8093A11382
:10F1E0009093A213A093A313B093A41320E030E054
:10F1F00040EF51E46091570C7091580C8091590C7C
:10F2000090915A0C0F948205F9E8CF2EF3E1DF2E8E
:10F210007B018C0129EA33E145EA53E161EA73E1BC
:10F220008DE993E10E9498EF80E090E0A0EAB0E4DD
:10F230008093A5139093A613A093A713B093A8133C
:10F2400020E030E040E752E460915F0C7091600C88
:10F250008091610C9091620C0F9482057B018C016E
:10F2600029EA33E145EA53E161EA73E18DE993E18B
:10F270000E9498EF0E9415E420E030E040EA51E45B
:10F280006091570C7091580C8091590C90915A0CC8
:10F290000F9482050F94EA058B0120E030E040E2F4
:10F2A00052E460915F0C7091600C8091610C9091C0
:10F2B000620C0F9482050F94EA057B010E94DD62C7
:10F2C00019AE18AEC701AA2797FDA095BA2F8CAF2B
:10F2D0009DAFAEAFBFAFC801AA2797FDA095BA2FCB
:10F2E00024968CAF9DAFAEAFBFAF249780E090E087
:10F2F000A0EAB0E48093A5139093A613A093A7135C
:10F30000B093A8136CAD7DAD8EAD9FAD0F941D066F
:10F310001B012C01E9E8CE2EE3E1DE2E7B018C01FE
:10F3200029EA33E145EA53E161EA73E18DE993E1CA
:10F330000E9498EF0E9415E488AD99AD63E070E0FB
:10F340000F9446097BAF6AAF3C019AAD90FF05C0B0
:10F35000A2E0B0E0A619B7093D01B301882777FD07
:10F360008095982F0F941D0620E030E04BEC52E47E
:10F370000F94500820E030E04CE052E40F94A204D7
:10F3800020E030E048EB51E40F94A10460939D131A
:10F3900070939E1380939F139093A013EAADFBADDF
:10F3A000BF01882777FD8095982F0F941D0620E0D8
:10F3B00030E044EC52E40F94500820E030E040ECA0
:10F3C00050E40F94A20420E030E040E151E40F94B7
:10F3D000A1046093A1137093A2138093A31390933D
:10F3E000A41324966CAD7DAD8EAD9FAD24970F9484
:10F3F0001D064B015C0169E8C62E63E1D62E85012E
:10F40000740129EA33E145EA53E161EA73E18DE9E8
:10F4100093E10E9498EF0E9415E40E942E6387E01A
:10F420002AAD3BAD829FF001839FF00D1124E60DC4
:10F43000F71DEE0FFF1FEE0FFF1FE45FF74E8091E9
:10F44000A5139091A613A091A713B091A81381833F
:10F450009283A383B4838091D013811109C08091DA
:10F46000AE139091AF1301979093AF138093AE13A7
:10F47000A8ADB9AD1196B9AFA8AF199709F036CFBD
:10F480000E94086380E090E0A0EAB0E48093A513B6
:10F490009093A613A093A713B093A81359E8C52E71
:10F4A00053E1D52E8201710129EA33E145EA53E1A6
:10F4B00061EA73E18DE993E10E9498EF8CE098E1B5
:10F4C0000E94C8E781E080930C188DEC9CECACE4C2
:10F4D000BEE380939D1390939E13A0939F13B093CC
:10F4E000A01343E353E363E770EC4093A1135093FD
:10F4F000A2136093A3137093A4138093A513909306
:10F50000A613A093A713B093A8138501740129EA49
:10F5100033E145EA53E16DE973E1CB010E9498EFD5
:10F520000E9415E48091D013811106C08091C1130F
:10F53000882311F40C94349387EF9FE00F946611A5
:10F54000813011F00C9434936CEC73E188EF9FE000
:10F550000E94BAA68091CC139091CD139093401144
:10F5600080933F110C94349380910C18882309F4F4
:10F570009EC0E0E9F2E58491882341F09091C000BB
:10F5800095FFFCCF8093C6003196F5CF4AE050E05E
:10F5900067E070E08BE397E10E94C1DAEEE8F2E504
:10F5A0008491882341F09091C00095FFFCCF809317
:10F5B000C6003196F5CF4AE050E067E070E08BE39B
:10F5C00097E10E94C1DAEBE7F2E58491882341F0EC
:10F5D0009091C00095FFFCCF8093C6003196F5CF87
:10F5E0004AE050E065E070E08BE397E10E94C1DA09
:10F5F000E9E6F2E58491882341F09091C00095FFFF
:10F60000FCCF8093C6003196F5CF8091C00085FF76
:10F61000FCCF8AE08093C60000E010E036E6A32E1F
:10F6200032E5B32E44E6842E42E5942EE12CF12CF3
:10F6300098012C54374E6901F5018491E6E6F2E514
:10F64000882349F09091C00095FFFCCF8093C600BD
:10F6500031968491F5CFF601EE0DFF1D4181528167
:10F660006381748125E030E08BE397E10E9497DBB2
:10F67000F4E0EF0EF11C2CE1E216F104E9F6F401DE
:10F680008491E4E6F2E5882349F09091C00095FF6B
:10F69000FCCF8093C60031968491F5CF0C511109AF
:10F6A0000C33FFEF1F0709F0C1CF0C943493E6E44D
:10F6B000F2E58491882341F09091C00095FFFCCF42
:10F6C0008093C6003196F5CF8091C00085FFFCCFB6
:10F6D0008AE08093C6000C943493E9E3F2E58491C8
:10F6E000882341F09091C00095FFFCCF8093C60025
:10F6F0003196F5CF8091C00085FFFCCF8AE08093E2
:10F70000C6000E94DD620E942E630E940863EAE246
:10F71000F2E58491882341F09091C00095FFFCCFE1
:10F720008093C6003196F5CF4091A5135091A61352
:10F730006091A7137091A81325E030E08BE397E167
:10F740000E9497DBE8E2F2E58491882311F40C949F
:10F7500034939091C00095FFFCCF8093C600319602
:10F76000F3CF83E50E94BF68882331F00E94AB6825
:10F770000F94EA058B0102C000E010E080E50E94D2
:10F78000BF68882311F10E94AB680F94EA05011548
:10F79000110511F40C94349365307105ECF0E4E13B
:10F7A000F2E58491882341F09091C00095FFFCCF51
:10F7B0008093C6003196F5CF8091C00085FFFCCFC5
:10F7C0008AE08093C6000C9434930115110511F45E
:10F7D0000C94349360E070E01093CD130093CC133D
:10F7E000CB01880F991F6CEC73E18B50904F0E94F6
:10F7F000A9A68091CC139091CD1390934011809342
:10F800003F110C9434938091CC139091CD1391952A
:10F81000819591099093401180933F110C943493FA
:10F820006FEF87EF9FE00F947B110C94349310924D
:10F8300047130C94349381E0809347130C943493D2
:10F8400085E40E94BF68811102C00E9415E408E2AD
:10F85000C02E0EE0D02E81E9E82E83E1F82E0DE9CE
:10F8600013E1B12CD6018D916D010E94BF688823F0
:10F8700039F1B3E0BB120CC00E94AB68F8016083A1
:10F8800071838283938389EA93E10E947AFA18C094
:10F890000E94AB68D7012D913D914D915C910F94E1
:10F8A000A204F801608371838283938329EA33E1A0
:10F8B00045EA53E161EA73E18DE993E10E94A6F91B
:10F8C000B394F4E0EF0EF11C0C5F1F4F24E0B21272
:10F8D000C9CF0C9434938DE40E94BF68882311F43F
:10F8E0000C943B920E94AB680F94EA056737710550
:10F8F00011F40C9484860CF0F7C06A32710509F497
:10F9000062C40CF07AC06731710509F4BBC20CF017
:10F9100044C06231710511F40C949B841CF577FF8F
:10F9200002C00C943493623071050CF4AFC16131A4
:10F93000710511F00C943493E091BB13F0E0EE0FDD
:10F94000FF1FE85DFD4F0190F081E02DE853FF4F70
:10F95000808191810E946BAB179816981598149826
:10F960000C9434936531710509F480C20CF084C2A3
:10F970006431710511F00C943493E091BB13F0E005
:10F98000EE0FFF1FE85DFD4F0190F081E02DE25B7F
:10F99000FE4F0190F081E02D38C26B31710509F402
:10F9A0009DC2B4F46931710509F484C20CF088C2B7
:10F9B0008EEC93E10E94B5560E94C8FE6093AB1195
:10F9C0007093AC118093AD119093AE110C9434935D
:10F9D0006E31710509F4BDC234F46C31710509F45E
:10F9E00083C20C9434936F31710509F48CC3603277
:10F9F000710509F4ECC20C9434936836710509F46E
:10FA000029C40CF043C06335710509F48FC714F5A0
:10FA10006135710509F455C70CF084C7603571056F
:10FA200011F00C9434939B9AA39881E080931E0C60
:10FA3000E091BB13F0E0EE0FFF1FE85DFD4F01907A
:10FA4000F081E02D808191810E946BAB0E9404AE19
:10FA50000C9434936535710509F4A0C70CF46BC799
:10FA60006C35710511F00C94349328E23EE039AF07
:10FA700028AF06E01EE126E1822E2EE1922E3AEC1E
:10FA8000A32E3DE1B32E312C0C944B856D367105C0
:10FA900009F41CC58CF46A36710509F4E2C60CF44D
:10FAA00008C46B36710511F00C94349310928813CE
:10FAB000109287130C9434936237710511F40C94EF
:10FAC0008D853CF46037710511F00C9434930E94DD
:10FAD000736F6337710509F4F0C76537710511F469
:10FAE0000C9479850C9434936C3231E0730711F4E3
:10FAF0000C94538B0CF053C06C3C710511F40C94B6
:10FB0000488924F56E3B710509F47CC574F46937A6
:10FB1000710511F40C947F8614F40C947A866C3879
:10FB2000710509F4B5C30C943493693C710511F463
:10FB30000C9409896B3C710511F40C942B89683C79
:10FB4000710511F00C9434930C948788603D710515
:10FB500011F40C941F8A54F46E3C710511F40C944A
:10FB6000CA8914F40C946A890C94E8896C3D710577
:10FB700011F40C94B88A3CF4613D710511F40C94B5
:10FB8000478A0C9434936D3D710511F40C94C98A25
:10FB9000623E710511F40C94F38A0C943493653F22
:10FBA00091E0790711F40C944F8D2CF56033B1E09E
:10FBB0007B0711F40C945C8C5CF46E32F1E07F07EF
:10FBC00011F40C94068D14F40C94898B0C94148D00
:10FBD0006F3531E0730711F40C94DF91603981E0E7
:10FBE000780711F40C944C8D6E35714011F00C9423
:10FBF00034930C94A8916835A2E07A0711F40C9420
:10FC0000978EA4F4673FE1E07E0711F40C94578DC2
:10FC100014F40C94548D6D3F714011F00C94349396
:10FC20000E9439ABEFE4F3E50C94618D6B3833E05F
:10FC3000730711F40C9482913CF46335734011F412
:10FC40000C94728D0C943493603AA3E07A0709F413
:10FC500027C2673E734011F00C9434931092A111A7
:10FC60000E9468AD8091481390914913A0914A1366
:10FC7000B0914B1380934C1390934D13A0934E135C
:10FC8000B0934F130E941B690C9434930091B711E9
:10FC90001091B8110E5F1F4F80E50E94BF68882346
:10FCA00079F00E94AB680F94EF056B017C01BB24D7
:10FCB000B394611571058105910531F4B12C04C02F
:10FCC000B12CC12CD12C760183E50E94BF6888231A
:10FCD00099F00E94AB6820E030E04AE754E40F94CA
:10FCE00050080F94EF056B017C01AA24A3946115C1
:10FCF00071058105910509F4A12C6AE270E0C80143
:10FD00000F94120F009711F0FC011082F801CF013F
:10FD100021912032E1F3B11007C0A11005C02223C8
:10FD200019F00E945EAB10C0E091BB13F0E0EE0F43
:10FD3000FF1FE85DFD4F0190F081E02DEE53FF4F76
:10FD4000808191810E946BAB81E00E943EAB0E945A
:10FD500015E40E94C8FE6093B3117093B4118093B0
:10FD6000B5119093B611C114D104E104F104A9F0C6
:10FD70000E94C8FE4B015C018C0C9D1CAE1CBF1C7C
:10FD80000E94C8FE681579058A059B05C0F40E948B
:10FD9000E8AE811114C00C94D8940E94E6AE88237A
:10FDA00011F40C9434930E94E8AE81110BC00E94B0
:10FDB0001A4780E00E94BD750E9404AEF4CF80E037
:10FDC0000E943EAB8091D013E091BB13F0E0EE0FA8
:10FDD000FF1FE85DFD4F0190F081E02D882341F089
:10FDE000EC53FF4F808191810E946BAB0C94349354
:10FDF000808191810E946BAB0C9434939091C000F0
:10FE000095FFFCCF8093C600319684918111F6CF87
:10FE10008091C00085FFFCCF8AE08093C6008EEC05
:10FE200093E10E945D55E091BB13F0E0EE0FFF1FE0
:10FE3000E85DFD4F0190F081E02DE05BFE4F019009
:10FE4000F081E02D8491882341F09091C00095FFCE
:10FE5000FCCF8093C6003196F5CF8091C00085FF1E
:10FE6000FCCF8AE08093C6000C9434938EEC93E12F
:10FE70000E94B2550C9434938EEC93E10E94B156DB
:10FE80000C9434930091B7111091B8110C5F1F4F6F
:10FE90006AE270E0C8010F94120F009711F0DC01C4
:10FEA0001C9221E041E0B8018EEC93E10E94335BAB
:10FEB0000C9434938EEC93E10E94BC560C943493D2
:10FEC0008091D113882311F40C94349383E50E941C
:10FED000BF6881110C94E1940C9434938EEC93E1FF
:10FEE0000E9460580C9434938091B7119091B8118E
:10FEF0006AE270E004960F94120F8C010097D9F01B
:10FF00002091C1113091C21140E6429FC001439F30
:10FF1000900D11246EE470E089539E4E0F94120FE1
:10FF200060E270E00F94120F01969093B8118093E5
:10FF3000B711F80110826091B7117091B8116C5F20
:10FF40007F4F21E040E08EEC93E10E94335B0C9404
:10FF500034938091D113882311F40C94349360E08E
:10FF60008EEC93E10E94C35A8091B7119091B81121
:10FF70006AE270E004960F94120F8C010097D9F09A
:10FF80002091C1113091C21140E6429FC001439FB0
:10FF9000900D11246EE470E089539E4E0F94120F61
:10FFA00060E270E00F94120F01969093B811809365
:10FFB000B711D8011C926091B7117091B8116C5FA4
:10FFC0007F4F8EEC93E10E9420570C9434938091E4
:10FFD000D01381110E9415E40091B7111091B8114E
:10FFE0000C5F1F4F6AE270E0C8010F94120F7C0192
:10FFF00061E270E0C8010F94120F009719F08C01B4
:020000021000EC
:100000000F5F1F4FE114F10411F0F701108280E53A
:100010000E94BF68F82E2091B7113091B8110217D5
:10002000130708F4F12C8091D113882311F40C9458
:10003000349321E02F2541E0B8018EEC93E10E943A
:10004000335B83E50E94BF688823B9F02091B71124
:100050003091B8112017310780F40E94B468AB01C9
:10006000BC0140936B1650936C1660936D167093A1
:100070006E1686EB95E10E944D348EEC93E10E9462
:10008000B556F1100C9434930E94C8FE6093AB11E6
:100090007093AC118093AD119093AE110C94349386
:1000A0008091B7119091B8116AE270E005960F94B3
:1000B000120F8C010097D9F02091C1113091C2111B
:1000C00040E6429FC001439F900D11246EE470E012
:1000D00089539E4E0F94120F60E270E00F94120F3E
:1000E00001969093B8118093B711D8011C9260913A
:1000F000B7117091B8116B5F7F4F8EEC93E10E9446
:10010000B85E0C9434930E94C8FE6093A71170935C
:10011000A8118093A9119093AA110091AB1110918D
:10012000AC112091AD113091AE11601B710B820B9F
:10013000930B28EE33E040E050E00F945909CA01D8
:10014000B9012CE330E040E050E00F9459097F936F
:100150006F933F932F9385E092E59F938F93CE010A
:1001600001969F938F930F944A0FEFE4F3E58491E8
:100170000FB6F894DEBF0FBECDBFEFE4F3E58823E2
:1001800049F09091C00095FFFCCF8093C600319656
:100190008491F5CFFE0131968191882339F09091B9
:1001A000C00095FFFCCF8093C600F6CF8091C000C1
:1001B00085FFFCCF8AE08093C600CE0101960E94A5
:1001C0005EAB0C94349383E50E94BF68882311F4DE
:1001D0000C9434930E94AB680F94EA05F62EE72E38
:1001E000862F9E2D8C0180E50E94BF68882331F008
:1001F0000F3F110509F010F40C94F2940DE010E09B
:10020000E0EFFDE0819191918017910711F40C943A
:1002100034932EE0E832F207A9F70630110539F4DD
:100220008F2D9E2D909388138093871304C017FF02
:1002300002C00C94349361E0802F0E94E8FD6F2D82
:10024000802F0E9421FE6F2D7E2D802F0E94DEFCCC
:100250000C94349388E690E00E942B7081110C94EA
:10026000349383E50E94BF68882371F00091A21146
:100270000E94AB6810E0000F111F005B1E4E0F9430
:10028000EA05D8016D937C930E945A410C943493F3
:1002900083E50E94BF68882311F40C9434930E9474
:1002A000AB680F94EA0570934F1160934E110C9454
:1002B000349389E690E00E942B7081110C94349362
:1002C000EFEFF1E58491882341F09091C00095FF14
:1002D000FCCF8093C6003196F5CFE091A211B4E037
:1002E000EB9FF0011124E85BFE4E40815181628159
:1002F000738121E030E08BE397E10E9497DBECEF24
:10030000F1E58491882341F09091C00095FFFCCFE6
:100310008093C6003196F5CFE091A211F0E0EE0F88
:10032000FF1FE05BFE4E60817181882777FD80951D
:10033000982F0F941D06AB01BC0121E030E08BE348
:1003400097E10E9497DBE8EFF1E58491882341F083
:100350009091C00095FFFCCF8093C6003196F5CFF9
:100360004091421150914311609144117091451197
:1003700021E030E08BE397E10E9497DBE5EFF1E5C8
:100380008491882341F09091C00095FFFCCF809329
:10039000C6003196F5CF60914E1170914F118827AC
:1003A00077FD8095982F0F941D06AB01BC0121E0CD
:1003B00030E08BE397E10E9497DBE2EFF1E5849177
:1003C000882341F09091C00095FFFCCF8093C60038
:1003D0003196F5CF4AE050E060E070E08BE397E1C2
:1003E0000E94C1DAE0EFF1E58491882341F0909119
:1003F000C00095FFFCCF8093C6003196F5CF4091A9
:1004000048115091491160914A1170914B1121E0AE
:1004100030E08BE397E10E9497DBEDEEF1E584910C
:10042000882341F09091C00095FFFCCF8093C600D7
:100430003196F5CF6091501170915111882777FD59
:100440008095982F0F941D06AB01BC0121E030E090
:100450008BE397E10E9497DBE9EEF1E58491882335
:1004600041F09091C00095FFFCCF8093C60031967B
:10047000F5CF8091A21190E00E9464404AE050E0E4
:10048000BC018BE397E10E94C1DAE4EEF1E58491CF
:10049000882341F09091C00095FFFCCF8093C60067
:1004A0003196F5CF8FEF9FEF0E9464404AE050E015
:1004B000BC018BE397E10E94C1DA8091C00085FF07
:1004C000FCCF8AE08093C6000C945B968DE690E0AA
:1004D0000E942B7081110C943493E091BB13F0E0D7
:1004E000EE0FFF1FE85DFD4F0190F081E02DE05A17
:1004F000FE4F808191810E946BAB81E090E09093F0
:10050000B6138093B51383E50E94BF68882391F0EA
:100510000091A2110E94AB6810E0000F111F005B58
:100520001E4E0F94EA05F8017183608381E0809389
:10053000140C15C082E50E94BF68882381F00091E9
:10054000A2110E94AB6810E0000F111F005B1E4E4D
:100550000F94EA05D8016D937C931092140C0E94BD
:100560005A410E94C8FE4B015C010091A21110E0AB
:10057000F801EE0FFF1FE05BFE4E6081718188275E
:1005800077FD8095982F0F941D06F801EE0FFF1F41
:10059000EE0FFF1FE85BFE4E11E0208131814281AA
:1005A00053810F947E0718160CF010E01093A011E1
:1005B00010927813CC24CA94DC2C760148EE442E99
:1005C00043E0542E612C712C5AE0352E8091781323
:1005D00081110C94F994BFEFCB16DB06EB06FB06FA
:1005E00011F40C942495F7FE02C00C94F9940E9427
:1005F000C8FE6C197D09683B7B4010F40C9424956F
:100600000C94F994E091BB13F0E0EE0FFF1FE85D4E
:10061000FD4F0190F081E02DEC59FE4F80819181DA
:100620000E946BAB83E090E09093B6138093B51378
:1006300083E50E94BF68882361F00E94AB680F9435
:10064000EA0570934F1160934E1181E08093140C72
:100650000FC082E50E94BF68882351F00E94AB68FA
:100660000F94EA0570934F1160934E111092140C81
:100670000E94C8FE4B015C011092781360914E11EC
:1006800070914F11882777FD8095982F0F941D0644
:1006900011E0209142113091431140914411509149
:1006A00045110F947E0718160CF010E01093A0115E
:1006B00006ED11E572EDE72E71E5F72EEEECCE2E8C
:1006C000E1E5DE2EFAE07F2E8091A01160914E11BF
:1006D00070914F11882309F48BC080917813811198
:1006E00087C0882777FD8095982F0F941D0620914D
:1006F00042113091431140914411509145110F9492
:100700007E0718160CF08BC00E94C8FE6819790984
:100710008A099B09693E73408105910508F460C010
:10072000E091891324E0E29FF0011124E85BFE4E82
:100730004081518162817381F8018491E6EDF1E598
:10074000882349F09091C00095FFFCCF8093C600AC
:1007500031968491F5CF22E030E08BE397E10E945F
:1007600097DBF7018491E2EDF1E5882349F0909160
:10077000C00095FFFCCF8093C60031968491F5CFE1
:100780006091891370E04AE050E08BE397E10E94AA
:10079000C1DAF6018491EEECF1E5882349F09091FD
:1007A000C00095FFFCCF8093C60031968491F5CFB1
:1007B0004091421150914311609144117091451143
:1007C00021E030E08BE397E10E9497DB8091C0004D
:1007D00085FFFCCF7092C6000E94C8FE4B015C01F1
:1007E0000E941A4780E00E94BD750E9404AE6CCF43
:1007F000882777FD8095982F0F941D062091421130
:100800003091431140914411509145110F947B0553
:1008100087FF05C08091140C882309F475CFE091FF
:10082000BB13F0E0EE0FFF1FE85DFD4F0190F0817C
:10083000E02DEA59FE4F808191810E946BAB84E0EC
:1008400090E09093B6138093B5130E94C8FE609316
:10085000B3117093B4118093B5119093B6110C94A9
:10086000349383E50E94BF68882319F10E94AB6826
:1008700020E030E0A9010F947B0587FD0FC00E94A6
:10088000AB6820E030E04FE753E40F947E07181682
:1008900044F00E94AB680F94EA0505C060E070E088
:1008A00002C06FEF70E070938813609387130C940D
:1008B00034938FEF90E090938813809387130C9478
:1008C00034930E945B410E9415E4149A0E9492E4C2
:1008D000109288131092871368EE73E080E090E026
:1008E0000E94F7FE9B9AA39A10921E0CE091BB13F4
:1008F000F0E0EE0FFF1FE85DFD4F0190F081E02D6D
:10090000E459FF4F408151812CEC31E56AEC71E5EF
:1009100081ED9DE00E94494F0E946BAB0E9404AEA6
:100920000C9434931092C7130C94349381E0809309
:10093000C7130C94349383E50E94BF688823A1F009
:100940000E94AB6820E030E04AE754E40F9450087E
:100950000F94EF056093150C7093160C8093170C91
:100960009093180C0C94349388E50E94BF68811111
:100970000C94389689E50E94BF6881110C943896D2
:100980008AE50E94BF6881110C94389685E40E9424
:10099000BF6881110C9438960C94559683E50E949B
:1009A000BF68882311F40C9434930E94AB6820E054
:1009B00030E04AE754E40F9450080F94EF05609339
:1009C000AF117093B0118093B1119093B2110C9448
:1009D0003493B3E03B1269C00E94AB686B017C01A9
:1009E00020E030E040EA51E40F947B0587FF3FC0F0
:1009F000A7019601F80160817181828193810F9432
:100A000082052B013C019B01AC016091DE1D7091C0
:100A1000DF1D8091E01D9091E11D0F9450086093BF
:100A2000DE1D7093DF1D8093E01D9093E11DA301F7
:100A30009201D4016D917D918D919C910F945008FC
:100A4000F4016083718382839383D5016D917D91DD
:100A50008D919C910F941B06A30192010F94500855
:100A60000F94EF05F5016083718382839383D8012E
:100A7000CD92DD92ED92FC92139733940C5F1F4F51
:100A8000F4E08F0E911C24E0A20EB11C34E033166A
:100A900011F40C943493A8ADB9AD8D91B9AFA8AF52
:100AA0000E94BF68882349F394CF0E94AB68F80185
:100AB0006083718382839383E0CFE091BB13F0E086
:100AC000EE0FFF1FE85DFD4F0190F081E02DE8592A
:100AD000FE4F0190F081E02D8491882311F40C9455
:100AE00034939091C00095FFFCCF8093C60031965F
:100AF000F3CF0091B7111091B8110B5F1F4F6AE24D
:100B000070E0C8010F94120F009711F0DC011C92E5
:100B1000C8010E945EAB0C943493E7ECF1E584913C
:100B2000882341F09091C00095FFFCCF8093C600D0
:100B30003196F5CF40919D1350919E1360919F1374
:100B40007091A01322E030E08BE397E10E9497DBE5
:100B5000E3ECF1E58491882341F09091C00095FF8A
:100B6000FCCF8093C6003196F5CF4091A1135091F0
:100B7000A2136091A3137091A41322E030E08BE3E1
:100B800097E10E9497DBEFEBF1E58491882341F038
:100B90009091C00095FFFCCF8093C6003196F5CFB1
:100BA0004091A5135091A6136091A7137091A813BB
:100BB00022E030E08BE397E10E9497DBEBEBF1E57D
:100BC0008491882341F09091C00095FFFCCF8093E1
:100BD000C6003196F5CF4091A9135091AA136091A8
:100BE000AB137091AC1322E030E08BE397E10E94ED
:100BF00097DBE091BB13F0E0EE0FFF1FE85DFD4FC8
:100C00000190F081E02DE659FE4F0190F081E02D3A
:100C10008491882341F09091C00095FFFCCF809390
:100C2000C6003196F5CF0E9471E40F941D06209105
:100C3000061E3091071E4091081E5091091E0F9408
:100C40008205AB01BC0122E030E08BE397E10E941A
:100C500097DBE7EBF1E58491882341F09091C000A8
:100C600095FFFCCF8093C6003196F5CF81E00E94BE
:100C700071E40F941D0620910A1E30910B1E4091C5
:100C80000C1E50910D1E0F948205AB01BC0122E099
:100C900030E08BE397E10E9497DBE3EBF1E5849191
:100CA000882341F09091C00095FFFCCF8093C6004F
:100CB0003196F5CF82E00E9471E40F941D062091D9
:100CC0000E1E30910F1E4091101E5091111E0F9458
:100CD0008205AB01BC0122E030E08BE397E10E948A
:100CE00097DB8091C00085FFFCCF8AE08093C6002F
:100CF0000C94349380E00E9495DC0C94349381E052
:100D00000E9495DC0C943493E091BB13F0E0EE0F5D
:100D1000FF1FE85DFD4F0190F081E02DEC57FE4F85
:100D20000190F081E02D8491882341F09091C000E2
:100D300095FFFCCF8093C6003196F5CF8091C0001F
:100D400085FFFCCF8AE08093C600E091BB13F0E002
:100D5000EE0FFF1FE85DFD4F0190F081E02DE85898
:100D6000FE4F0190F081E02D8491882341F0909115
:100D7000C00095FFFCCF8093C6003196F5CFE0917F
:100D8000BB13F0E0EE0FFF1FE85DFD4F1E9B13C08D
:100D90000190F081E02DEA57FE4F0190F081E02DA7
:100DA00084918823D9F09091C00095FFFCCF809367
:100DB000C6003196F5CF0190F081E02DE857FE4F47
:100DC0000190F081E02D8491882341F09091C00042
:100DD00095FFFCCF8093C6003196F5CF8091C0007F
:100DE00085FFFCCF8AE08093C600E091BB13F0E062
:100DF000EE0FFF1FE85DFD4F0190F081E02DE658FA
:100E0000FE4F0190F081E02D8491882341F0909174
:100E1000C00095FFFCCF8093C6003196F5CFE091DE
:100E2000BB13F0E0EE0FFF1FE85DFD4F029913C00A
:100E30000190F081E02DEA57FE4F0190F081E02D06
:100E400084918823D9F09091C00095FFFCCF8093C6
:100E5000C6003196F5CF0190F081E02DE857FE4FA6
:100E60000190F081E02D8491882341F09091C000A1
:100E700095FFFCCF8093C6003196F5CF8091C000DE
:100E800085FFFCCF8AE08093C600E091BB13F0E0C1
:100E9000EE0FFF1FE85DFD4F0190F081E02DE4585B
:100EA000FE4F0190F081E02D8491882341F09091D4
:100EB000C00095FFFCCF8093C6003196F5CFE0913E
:100EC000BB13F0E0EE0FFF1FE85DFD4F1D9B13C04D
:100ED0000190F081E02DEA57FE4F0190F081E02D66
:100EE00084918823D9F09091C00095FFFCCF809326
:100EF000C6003196F5CF0190F081E02DE857FE4F06
:100F00000190F081E02D8491882341F09091C00000
:100F100095FFFCCF8093C6003196F5CF8091C0003D
:100F200085FFFCCF8AE08093C600E091BB13F0E020
:100F3000EE0FFF1FE85DFD4F0190F081E02DE258BC
:100F4000FE4F0190F081E02D8491882341F0909133
:100F5000C00095FFFCCF8093C6003196F5CFE0919D
:100F6000BB13F0E0EE0FFF1FE85DFD4F019913C0CA
:100F70000190F081E02DEA57FE4F0190F081E02DC5
:100F800084918823D9F09091C00095FFFCCF809385
:100F9000C6003196F5CF0190F081E02DE857FE4F65
:100FA0000190F081E02D8491882341F09091C00060
:100FB00095FFFCCF8093C6003196F5CF8091C0009D
:100FC00085FFFCCF8AE08093C600E091BB13F0E080
:100FD000EE0FFF1FE85DFD4F0190F081E02DE0581E
:100FE000FE4F0190F081E02D8491882341F0909193
:100FF000C00095FFFCCF8093C6003196F5CFE091FD
:10100000BB13F0E0EE0FFF1FE85DFD4F1C9B13C00C
:101010000190F081E02DEA57FE4F0190F081E02D24
:1010200084918823D9F09091C00095FFFCCF8093E4
:10103000C6003196F5CF0190F081E02DE857FE4FC4
:101040000190F081E02D8491882341F09091C000BF
:1010500095FFFCCF8093C6003196F5CF8091C000FC
:1010600085FFFCCF8AE08093C600E091BB13F0E0DF
:10107000EE0FFF1FE85DFD4F0190F081E02DEE5770
:10108000FE4F0190F081E02D8491882341F09091F2
:10109000C00095FFFCCF8093C6003196F5CFE0915C
:1010A000BB13F0E0EE0FFF1FE85DFD4F379913C053
:1010B0000190F081E02DEA57FE4F0190F081E02D84
:1010C00084918823D9F09091C00095FFFCCF809344
:1010D000C6003196F5CF0190F081E02DE857FE4F24
:1010E0000190F081E02D8491882341F09091C0001F
:1010F00095FFFCCF8093C6003196F5CF8091C0005C
:1011000085FFFCCF8AE08093C6000C9434938091D5
:1011100089138093A21184E50E94BF68882381F11E
:101120000E94AB680F94EF056093A211662341F112
:10113000EFE4F3E58491882341F09091C00095FF9E
:10114000FCCF8093C6003196F5CFE091BB13F0E061
:10115000EE0FFF1FE85DFD4F0190F081E02DEA5A90
:10116000FE4F0190F081E02D8191882311F40C94C1
:1011700034939091C00095FFFCCF8093C600F4CFCC
:1011800084E40E94BF68882311F40C9434930E9475
:10119000AB6820E030E0A9010F947B05811103C00A
:1011A0001092AD1332C00091A21110E00E94AB6802
:1011B000F801EE0FFF1FEE0FFF1FE55BF34F60839B
:1011C000718382839383E0904B0CF0904C0C0091E0
:1011D0004D0C10914E0C20E030E0A901B701C80180
:1011E0000F947B05811104C0E12CF12C00E410E484
:1011F000C701D80180934B0C90934C0CA0934D0CDD
:10120000B0934E0C81E08093AD130E9461760C94F4
:10121000349308E21EE0A6EFEA2EADE1FA2EF801C3
:1012200081918F010E94BF68882351F00E94AB68B2
:101230000F94EF05D7016D937D938D939C93139736
:10124000B4E0EB0EF11CEEE00C321E0741F70E94F9
:10125000A7FA0C94349308E21EE0F6E1EF2EFEE1CB
:10126000FF2ED8018D918D010E94BF68882339F02F
:101270000E94AB68F7016083718382839383F4E0FB
:10128000EF0EF11C2EE00C32120759F70C94349338
:1012900083E50E94BF68882351F00E94AB68609389
:1012A000EE1D7093EF1D8093F01D9093F11D84E56A
:1012B0000E94BF68882311F40C9434930E94AB6899
:1012C0006093EA1D7093EB1D8093EC1D9093ED1DD0
:1012D0000C94349383E50E94BF68882351F00E94E8
:1012E000AB686093F21D7093F31D8093F41D90938F
:1012F000F51D84E50E94BF68882351F00E94AB6809
:101300006093DA1D7093DB1D8093DC1D9093DD1DCF
:1013100082E40E94BF68882361F00E94AB680F944A
:10132000EF056093261E7093271E8093281E9093CE
:10133000291E88E50E94BF68882351F00E94AB688F
:101340006093E61D7093E71D8093E81D9093E91D5F
:101350008AE50E94BF68882351F00E94AB686093C1
:10136000E21D7093E31D8093E41D9093E51D85E4D9
:101370000E94BF68882311F40C9434930E94AB68D8
:101380006093DE1D7093DF1D8093E01D9093E11D3F
:101390000C94349308E21EE0E1E9EE2EE3E1FE2E28
:1013A000D8018D918D010E94BF68882339F00E9479
:1013B000AB68F7016083718382839383F4E0EF0E5F
:1013C000F11C2EE00B32120711F40C943493E8CF89
:1013D00083E50E94BF68882351F00E94AB68609348
:1013E0002B0C70932C0C80932D0C90932E0C86E478
:1013F0000E94BF68882381F00E94AB6820E030E043
:1014000040E752E40F9482056093230C7093240C00
:101410008093250C9093260C8AE50E94BF68882350
:1014200011F40C9434930E94AB6860938113709311
:10143000821380938313909384130C94349383E5E5
:101440000E94BF68882351F00E94AB6860937D13AF
:1014500070937E1380937F139093801386E40E9491
:10146000BF68882311F40C9434930E94AB6820E089
:1014700030E040E752E40F94820560931F0C7093B4
:10148000200C8093210C9093220C0C94349383E5D0
:101490000E94BF68882311F40C9434930E94AB68B7
:1014A0000F94EA056115710551F06130710569F419
:1014B00081E080938613109285130C9434931092DC
:1014C0008613109285130C943493EFE4F3E5849122
:1014D000882341F09091C00095FFFCCF8093C60017
:1014E0003196F5CFE091BB13F0E0EE0FFF1FE85D02
:1014F000FD4F0190F081E02DEE58FE4F0190F081FC
:10150000E02D8491882341F09091C00095FFFCCF9D
:101510008093C6003196F5CF8091C1119091C21190
:1015200020E6289FF001299FF00D1124E953FE4E7B
:101530008191882339F09091C00095FFFCCF809372
:10154000C600F6CFE1EBF1E58491882341F090915C
:10155000C00095FFFCCF8093C6003196F5CF8091F7
:10156000C00085FFFCCF8AE08093C6000C943493C2
:1015700083E50E94BF68882311F40C9434930E9481
:10158000AB680F94EA057093560C6093550C0C945D
:10159000349383E50E94BF68882311F40C9434933C
:1015A0000E94AB680F94EA056B017C0184E50E9400
:1015B000BF68882391F08DED90E00E942B7081111F
:1015C0000C943493E091A211F0E0EE0FFF1FEF5A5C
:1015D000F34FD182C0820C943493D092540CC092B9
:1015E000530C0C94349380E50E94BF68882311F457
:1015F0000C9434930E94AB680F94EA05D62E062F04
:10160000172F83E50E94BF68882331F00E94AB68E2
:101610000F94EA057B0103C0EE24EA94FE2CC70177
:101620000196039710F00C943493E0EFFDE0819164
:1016300091918017910711F40C9434933EE0E832B5
:10164000F307A9F717FF02C00C9434930E9415E426
:10165000CD2C60E08D2D0E94E8FD8FEFE816F80696
:1016600031F0EA94EF2871F000E010E00DC08D2D0C
:101670000E9456FE31E020E0892B09F030E0032F74
:10168000122F02C001E010E08C2D0E9456FE801740
:10169000910709F4E9C70E941A4780E00E94BD75CE
:1016A0000E9404AEF1CF83E50E94BF68882331F029
:1016B0000E94AB680F94EA058B0102C00EE610E0B1
:1016C00080E50E94BF68882331F00E94AB680F94C8
:1016D000EA05CB0102C088EE93E06C01EE24D7FC52
:1016E000E094FE2C101611067CF420E030E0A901F5
:1016F000B80184E50E9494FFC701B6010E94F7FE7D
:1017000084E50F94AB02B0C7C701B6010E94F7FE93
:10171000ABC780E50E94BF68882351F00E94AB6888
:1017200060932402709325028093260290932702EF
:1017300089E40E94BF68882361F00E94AB680E9420
:10174000844C609320027093210280932202909334
:10175000230284E40E94BF68882361F00E94AB6882
:101760000E94904C60931C0270931D0280931E0295
:1017700090931F0283E40E94BF68882351F00E9467
:10178000AB68609318027093190280931A029093C9
:101790001B020E943740E091BB13F0E0EE0FFF1FE9
:1017A000E85DFD4F0190F081E02DE05CFE4F01907F
:1017B000F081E02D8191882339F09091C00095FF50
:1017C000FCCF8093C600F6CFEEEDFDE0819188233B
:1017D00039F09091C00095FFFCCF8093C600F6CF02
:1017E00040912402509125026091260270912702B7
:1017F00022E030E08BE397E10E9497DBE2EEFDE030
:101800008191882339F09091C00095FFFCCF80939F
:10181000C600F6CF609120027091210280912202D1
:10182000909123020E948A4CAB01BC0122E030E07F
:101830008BE397E10E9497DBE6EEFDE08191882340
:1018400039F09091C00095FFFCCF8093C600F6CF91
:1018500060911C0270911D0280911E0290911F02E6
:101860000E94964CAB01BC0122E030E08BE397E193
:101870000E9497DBEAEEFDE08191882339F0909198
:10188000C00095FFFCCF8093C600F6CF40911802B0
:101890005091190260911A0270911B0222E030E00F
:1018A0008BE397E10E9497DB8091C00085FFFCCF1E
:1018B0008AE08093C600D8C680E50E94BF6888236E
:1018C00051F00E94AB6860931402709315028093EC
:1018D00016029093170289E40E94BF68882361F082
:1018E0000E94AB680E94844C6093100270931102B6
:1018F000809312029093130284E40E94BF688823AD
:1019000061F00E94AB680E94904C60930C0270934F
:101910000D0280930E0290930F020E943740E091D7
:10192000BB13F0E0EE0FFF1FE85DFD4F0190F0816B
:10193000E02DE05CFE4F0190F081E02D8191882345
:1019400039F09091C00095FFFCCF8093C600F6CF90
:10195000EEEDFDE08191882339F09091C00095FF74
:10196000FCCF8093C600F6CF40911402509115022F
:10197000609116027091170222E030E08BE397E14C
:101980000E9497DBE2EEFDE08191882339F090918F
:10199000C00095FFFCCF8093C600F6CF6091100287
:1019A0007091110280911202909113020E948A4C50
:1019B000AB01BC0122E030E08BE397E10E9497DBB2
:1019C000E6EEFDE08191882339F09091C00095FF0B
:1019D000FCCF8093C600F6CF60910C0270910D028F
:1019E00080910E0290910F020E94964CAB01BC01B7
:1019F00022E030E08BE397E10E9497DB8091C0000A
:101A000085FFFCCF8AE08093C6002EC683E50E9446
:101A1000BF68882319F00E94AB6803C060E070E0E3
:101A2000CB010E949EFA20C685E40E94BF688823ED
:101A300041F00E94AB680F94EA058B0177FF03C069
:101A400009C000E010E0C12CD12C26E1E22E23E4F5
:101A5000F22E06C0C12CD12C9CE8E92E92E4F92E7E
:101A600083E50E94BF68882321F00E94AB686B0168
:101A70007C0183E40E94BF68882331F00E94AB6838
:101A80000F94EA059B0102C025E030E0A801C701E0
:101A9000B6010E946E41E8C50E9415E4E5C50E94AA
:101AA000C8D70E949AD3E0C50E94C8D7DDC50E945E
:101AB0009AD3DAC59091C00095FFFCCF8093C60001
:101AC000319684918111F6CFE1EAF1E58491882382
:101AD00009F4CAC59091C00095FFFCCF8093C60061
:101AE0003196F4CF8AE50E94BF68882309F4D6C0F6
:101AF0000E94AB686B017C0120E030E040E751ECD4
:101B00000F947E0787FD57C020E030E040EA50EC9C
:101B1000C701B6010F947B0518160CF44CC0F7FAF8
:101B2000F094F7F8F094C0928A13D0928B13E0925D
:101B30008C13F0928D13EFE4F3E58491882341F048
:101B40009091C00095FFFCCF8093C6003196F5CFF1
:101B5000E091BB13F0E0EE0FFF1FE85DFD4F8081C9
:101B60009181FC01E05CFE4F40815181E855F10913
:101B700020EA31E567E97EE0808191810E94494F4A
:101B8000FC012491222341F03091C00035FFFCCFAD
:101B90002093C6000196F4CF8091C00085FFFCCF52
:101BA0008AE08093C6008091C00085FFFCCF8AE068
:101BB0008093C60059C5EFE4F3E58491882341F092
:101BC0009091C00095FFFCCF8093C6003196F5CF71
:101BD000E091BB13F0E0EE0FFF1FE85DFD4F0190B9
:101BE000F081E02DE851FF4F0190F081E02D8491CC
:101BF000882341F09091C00095FFFCCF8093C600F0
:101C00003196F5CFE091BB13F0E0EE0FFF1FE85DDA
